:100000000C94AC120C94DB120C94DB120C94DB12EB
:100010000C94DB120C94DB120C94DB120C94DB12AC
:100020000C94DB120C94DB120C94CF180C944580CA
:100030000C9493840C9498800C94DB120C945C19AF
:100040000C94BD180C94DB120C94D48B0C948F89F7
:100050000C94DB120C94DB120C94DB120C94DB126C
:100060000C941A850C94A8190C9401810C94688541
:100070000C94DB120C94DB120C94AE7D0C94DB120E
:100080000C94DB120C94DB120C94DB127E1B831B92
:100090002E1B341B571B571B571B741B791B7E1BB6
:1000A000831BA01BA01B881B3A1B931B931B541C78
:1000B000591C201C261C2C1C2C1C2C1C4A1C4F1CA4
:1000C000541C591C681C681C5F1C182C182C182CFC
:1000D000182C812C3E2C3E2C3E2C3E2C3E2C3E2CB3
:1000E0003E2C282C302C302C482C482C8C2C8C2C42
:1000F0005A2C8C2C8C2C8C2C8C2C8C2C772C772C9C
:100100008C2C8C2C8C2C8C2C8C2C8C2C8C2C8C2C2F
:100110008C2C8C2C8C2C8C2C8C2C8C2C8C2C8C2C1F
:100120008C2C8C2C8C2C8C2C732C8C2C8C2C2B2C89
:100130008C2C282C282C842C223B2C3B423B8F3BA4
:10014000CE3B2C3C373C3A3C943C983C89419E4108
:100150003B42CE435744C942EB47D445D144D944EE
:100160006745D846555128512B512F51355139519A
:100170003E517B5C8A5C955CAB5CB25CB95CC85CF4
:10018000DF5CF75CC25DED5DF55DFD5D095E2A5EDD
:100190003A5E645EB15EBD5EF85E105F215F2D5F0A
:1001A000395F455F716287628762876274627A62D3
:1001B00087627762876280627D6283629862CD6EB9
:1001C0006D65FF6BEE65CD6ECD6E6B69CD6E656D49
:1001D000CD6ECD6ECD6EAF64A862F266217C127CCE
:1001E0000E7C147C187C1C7C107C1F7C297C7D83FD
:1001F00080839783B283B283978397839D869F86FC
:10020000A286A786B886C786D586DF86EF86FF8654
:1002100004871A871D872187238725872A872E87AA
:1002200039873D8745874C8750875287568758873F
:100230005A875C876087648769876E87738778874A
:100240007D87204F6C642056657273696F6E204500
:100250004550524F4D202020434845434B205345A5
:100260005454494E47532F43414C494200416C611D
:10027000726D732044697361626C6564004545501A
:10028000524F4D206C6F77206D656D004C4F41448F
:10029000494E470003426F6F746C6F616465720072
:1002A0004861726477617265204D656E7520456E98
:1002B00061626C6564006D537461636B206F666C82
:1002C0006F7700537769746368205761726E696E47
:1002D000671F506C656173652052657365742053A8
:1002E00077697463686573005468726F74746C65C1
:1002F000206E6F742069646C651F5265736574208D
:100300007468726F74746C65004D45535341474572
:1003100000707265737320616E79204B65790050AF
:100320007265737320616E79206B657920746F201C
:10033000736B6970004F46464F4E205448735448C3
:1003400025002D2D2D004348002D2D2D20002D2D75
:100350002D2D00000064281007030100000000019B
:1003600001010202020201010300040420414C4584
:1003700052540000010203000201030301020003C2
:10038000020100055275642000456C652000546828
:1003900072200041696C20004F4E20004F464600FD
:1003A00003544852525544454C4549443049443120
:1003B00049443241494C47454154524E4C31204CFE
:1003C00032204C33204C34204C35204C36204C37D6
:1003D000204C38204C39204C41204C42204C4320AA
:1003E0004C44204C45204C46204C47204C48204C47
:1003F0004920454C80454C2D454C815255805255E5
:100400002D52558141498041492D414981474580BF
:1004100047452D474581504231504232001B1E272F
:100420002D36394B4E636C7278878D939CB1B4C670
:10043000C9D2D8E1E453706C617368008040000059
:1004400000000000000000000000000000000000AC
:10045000000000000000000000000000000000009C
:10046000000000000000000000000000000000008C
:10047000000000000000000000000000000000007C
:1004800000000000000000000080C0E0E0F0F8F88C
:10049000FCFCFCF8F8F8F0400000000000808080D0
:1004A000000000000000000000000000000000004C
:1004B00000000080C0C0E0E0E0F0F0F0E0C000002C
:1004C000000000C0F8FFFF9F8783838383838383BB
:1004D000838383838383838383838383838383036C
:1004E00083808383838383838383838383838383DF
:1004F000838383838383838383C3E3733F1F0000EA
:10050000000080E0F0F8FCFEFFFFFFFF7F3F1F1FB1
:100510000F0783C3E1E1E0E0C0000E1F3F7F7FFFD4
:10052000F3E0E0800000000000000000000080F028
:10053000FCFEFFFFFFFF7F3F0F03010101000000F2
:1005400080F0FEFFFFC7C1C1C1C1C1C1C1C1C1C1EE
:10055000C1C1C1C1C1C1C1C1C1C1C1C101C1F0FEDF
:10056000FF3F0F070F0D0D0D1D19191919313131ED
:100570003171616161E1C1C1C18100000080E0F8B9
:10058000FCFFFFFFFF2F170F038180C0E0F0F8FC96
:10059000FEFFFFFFFFFFFF7F0100000000000000E3
:1005A00001010307070E1E1C3870E0F0F8FEFFFF84
:1005B0007F1F0F030001000000000000000000008A
:1005C000000000000000000000000000000000002B
:1005D000000000000000000000000000000000001B
:1005E000000000000000000000000000000000000B
:1005F0000000000000000000000000007EFFFFFF80
:10060000FFFFFFFBF8FCFCFEFF7F3F1F0F07C3FF50
:10061000FFFFFFFFFF7F0700000000000000000059
:100620000000000000C0E0F8FEFFFF7F1F0F1F3D2D
:100630007CF8F8F0E08000000000000000000000FE
:1006400000000000000000000000000000000000AA
:10065000000000000000000000000000000000009A
:10066000000000000000000000000000000000008A
:100670000000000000000000000000000000010178
:10068000010101030707070301000000E0FCFFFF71
:10069000FFFFFF1F0300000000000000000000003B
:1006A000C0F078DE2713090E0703000000000000E9
:1006B000000001030F7FFFFC7878F80000000000C5
:1006C00000000000000080808080808080808000AA
:1006D000808000808000000000000000808080801A
:1006E000808080808080808080808080808000000A
:1006F00000000000000000000000000000000000FA
:1007000000000000000000000080F0FEFFFFFFFF7F
:100710003F0F010000000000000000C0E0381E0F85
:1007200003000100000000000000000000000000C5
:1007300000000000000000000003030100000000B2
:100740000000000000000E0E02020202020303007D
:100750000F0F000F0F080808080808080F0F0808F7
:100760000808080F0F000000000F0F000000000035
:100770000000000000000000000000000000000079
:1007800000000000000000C0F8BFFFFFFF1F7F0156
:100790000000000000000000F0FCFF7F7830000047
:1007A0000000000000000000000000000000000049
:1007B0000000000000000000000000000000000039
:1007C0000000000000000000000000000000000029
:1007D0000000000000000000000000000000000019
:1007E0000000000000000000000000000000000009
:1007F00000000000000000000000000000000000F9
:100800000000000000301C070E0F07010000000070
:1008100000000000000000000000000000000000D8
:1008200000000000000000000000000000000000C8
:100830000000000000000000000000000000005662
:100840004552533A2056312E312D1F444154453ADA
:100850002033302E31322E323031351F54494D4540
:100860003A2031303A35383A31361F2053564E3A15
:1008700020657239782D723831391F204D4F443A36
:10088000204652534B592020203132382020003C42
:1008900006064F4E202020204F4646202020424F63
:1008A0005448202031355365637333305365637387
:1008B00036305365637356617269626C005653003B
:1008C00007203820536563733132205365637331D9
:1008D000362053656373001E030153415658004E82
:1008E000756D62657220566F69636520537700539A
:1008F0006166657479205377697463686573004332
:100900004F5059205452494D205B4D454E555D0086
:100910000D4F6E000D4F6E004C4F474943414C2028
:100920005357495443484553003C010A436F756E81
:100930007420446F776E436F756E7420557020205D
:100940000054696D65721F54726967676572411F53
:1009500054726967676572421F54696D65721F52F0
:1009600065736574205377697463680020547970E7
:10097000651F20436F756E7472791F42696E641F24
:1009800052616E6765003C02094C50342F4C503563
:10099000202044534D326F6E6C792044534D322FDA
:1009A00044534D580044534D205479706500014E16
:1009B00059000B4F7074696F6E0004486967684C8A
:1009C0006F7720003C00044E6F6E65003C010543CC
:1009D000473032335944383239003C0205475245DA
:1009E000454E424C554520444D303037003C0207BF
:1009F00053594D4158202053594D41583543003CDF
:100A0000040759443731372020534B59574C4B5228
:100A100053594D4158322058494E58554E204E4951
:100A20004855492020003C010444534D3244534D65
:100A300058003C01054869736B79484B33313000ED
:100A40003C0306466C79736B795639783920205609
:100A50003678362020563931322020003C0D0646AB
:100A60006C79736B7948756273616E4672736B79DA
:100A7000204869736B792056327832202044534DD8
:100A80003220204465766F20205944373137204B7F
:100A90004E2020202053796D615820534C54202043
:100AA000204358313020204347303233204261798F
:100AB000616E670050726F746F636F6C1F54797052
:100AC000651F506F7765721F42696E642020202079
:100AD000204175746F62696E641F52616E676500B4
:100AE000660103504F534E454700506F6C61726969
:100AF00074790050504D2046724C656E0D6D5365F3
:100B000063000C52784E756D000434434820364320
:100B1000482038434820313043483132434831344B
:100B200043483136434800137553000650504D205A
:100B3000202050585820202044534D32202050501F
:100B40004D31362050504D53494D4D554C54492050
:100B500053425553202000317374204368616E1F47
:100B600050726F746F000444521F024578706F1FFB
:100B70001F015765696768741F1F44725377311FDF
:100B8000447253773200034869204D6964204C6FEA
:100B900077006604042D2D2D2D3132302031323076
:100BA0005831343020393020200053776173682069
:100BB000547970651F436F6C6C6563746976651F4B
:100BC00053776173682052696E671F454C45204416
:100BD0006972656374696F6E1F41494C2044697284
:100BE000656374696F6E1F434F4C2044697265637F
:100BF00074696F6E0052455441313233005404061B
:100C0000457870202020457846696E6546696E6596
:100C100020204D656469756D436F61727365005482
:100C200072696D20496E631F5472696D2053771F7E
:100C300048692E52657320536C6F772F44656C6141
:100C4000791F547261696E65721F42656570204339
:100C50006E74005A01062020456E642043656E7450
:100C6000726500452E204C696D6974731F5468725B
:100C70002E2044656661756C741F5468726F7474BD
:100C80006C6520726576657273651F5468726F7447
:100C9000746C65204F70656E1F542D5472696D1F02
:100CA000542D4578706F2D4472006607032D2D2D4D
:100CB0005031205032205033204756344756354764
:100CC00056364756370044656661756C7420537715
:100CD0001F437573746F6D53746B4E616D65731F35
:100CE0004175746F204C696D6974731F566F6C7514
:100CF0006D6520436F6E74726F6C00566F6963652B
:100D000020496E646578114D454E55004D6F646500
:100D10006C204E616D65007016871892187F1879E7
:100D20001872186516431867185C1899185F161E14
:100D30001AB9165318564100566F696365004D4540
:100D40004E55204C4F4E470044656C657465005607
:100D50006F6963652046696C65005402062D2D2D70
:100D60002D2D2D4E756D62657220417564696F0081
:100D7000660104506C61794D757465005402064E2D
:100D80006F202020204265666F726541667465722F
:100D900020004E03072D2D2D2D2D2D2D4861707413
:100DA0006963314861707469633248617074696362
:100DB00033000776603D76616C20763D76616C206D
:100DC000200007280D2900506C617920536F75723F
:100DD00063651F4F6E206E6F2054656C656D657482
:100DE00072791F46696C655479706500536F75722E
:100DF00063651F46756E6374696F6E1F56616C750F
:100E0000651F5377697463681F526174651F486179
:100E10007074696300566F69636520416C61726D1F
:100E200000034D4F564520535449434B532F504FC9
:100E300054530005534554204D4944504F494E5496
:100E400000035B4D454E555D20544F205354415295
:100E500054006607044E4F4E45455854314558548A
:100E600032504330205047322050423720504735CF
:100E7000204C2D575200454C4520737769746368A8
:100E80001F41494C207377697463681F50423120B9
:100E90007377697463681F50423220737769746393
:100EA000681F50473220496E7075741F50423720BA
:100EB000496E7075741F4C2D575220496E707574B1
:100EC000004D27536F756E642053657269616C0025
:100ED0004672736B79204D6F6420446F6E650054C9
:100EE000656C656D657472455A3E3D7239300042DD
:100EF000616E644761700043616C004D756C74698C
:100F0000706C696572001802036F6666202B3D20C5
:100F10003A3D00036D6F64650A25207372632020DB
:100F200073770007536C6176650012424700414EAB
:100F300041000F504232000F504231005472696D2F
:100F40002D202B00204C6566741F52696768741F42
:100F50000355701F20446F776E1F20457869741FFA
:100F6000204D656E75004449414700537469636BB9
:100F70005363726F6C6C00506F745363726F6C6C60
:100F80000053706C617368204E616D650053706C26
:100F90006173682073637265656E004F776E65726A
:100FA000204E616D6500416C61726D205761726EFB
:100FB000696E67004D656D6F7279205761726E6959
:100FC0006E67005468726F74746C65205761726E3E
:100FD000696E670042617474657279207761726E20
:100FE000696E671F496E61637469766974792061FF
:100FF0006C61726D136D005275642000456C652044
:1010000000546872200041696C200043726F737352
:101010005472696D1F5468726F74746C65207265C8
:1010200076657273651F456E61626C652050504D28
:1010300053494D1F4368616E6E656C204F72646545
:10104000721F4D6F6465002048617074696320539E
:101050007472656E6774680042040A426565706563
:101060007220202020506953706B72202020204273
:1010700065657072566F696365506953706B566F22
:101080006963654D656761536F756E642000540632
:10109000065175696574204E6F4B657920785368E9
:1010A0006F727453686F7274204E6F726D20204C93
:1010B0006F6E672020784C6F6E672000566F6C75DE
:1010C0006D651F4265657065721F536F756E642094
:1010D0004D6F64651F20537065616B6572205069A8
:1010E000746368004C696768742073776974636817
:1010F0001F4261636B6C6967687420696E76657204
:10110000741F4C69676874206F6666206166746539
:10111000721F4C69676874206F6E2053746B204D8A
:10112000761F466C617368206F6E20626565700083
:10113000436F6E747261737400D1168816A916B964
:1011400016A0169416C916C1167E167616B0165A33
:1011500065726F20416C742E005A65726F204131A8
:10116000204F666673005A65726F204132204F66C9
:1011700066730052657365742047505300096D70A3
:1011800068004C61743D124864671F4C6F6E3D1FD0
:10119000416C743D096D2020204D61783D1F5370D6
:1011A000643D096B7473204D61783D1F56313D07D6
:1011B00056323D0E56333D1F56343D0756353D0ED3
:1011C00056363D000A52504D004675656C002204AB
:1011D0007C5E54546D0003457870457846466E65D4
:1011E0004D65644372730041323D0041313D00431F
:1011F00041502053504143452044454C20494E53D3
:101200000011544F541F01544D45115453571F01A1
:1012100053544B1153542500035B4D454E555D20EF
:10122000746F207265667265736800746D72314CFC
:101230006174206D61781275731F746D72314C6129
:1012400074206D696E1275731F746D7231204A6956
:10125000747465721275731F746D61696E126D73AB
:101260000053544154000966726565004D4F444572
:101270004C53454C0020464D300A524554410042E3
:1012800041434B555020444F4E45004241434B553E
:101290005000524553544F52454400534156494E15
:1012A0004700524553544F52494E47004C4F41441A
:1012B000494E4700526573746F7265004261636BFB
:1012C00075700020464D005377697463681F54722F
:1012D000696D731F4661646520496E1F46616465D0
:1012E000204F757400464C204D4F44450052414EEE
:1012F000474520434845434B20525353493A000643
:1013000042494E44494E47004475706C69636174AC
:10131000696E67206D6F64656C0044454C455445AB
:10132000204D4F44454C004455504C494341544591
:10133000204D4F44454C0054656D706C617465736D
:10134000104D454E5500012B2A52004D495845522B
:1013500000202020202020202020202020202000CD
:1013600044454C455445204D49583F00436C656108
:101370007220414C4C206D697865733F00035945DC
:10138000530B4E4F1F035B4D454E555D0B5B455850
:1013900049545D004D6178206D69786572732072E3
:1013A000656163683A2033321F1F50726573732082
:1013B0005B455849545D20746F2061626F72740000
:1013C0004E020841646420202020204D756C746911
:1013D000706C795265706C6163652000437572763C
:1013E0006500084469666600114578706F00015514
:1013F0007365204F75747075742020200001536F41
:10140000757263651F015765696768741F014F66D0
:10141000667365741F01466978204F66667365744C
:101420001F01456E61626C654578706F44521F0103
:101430005472696D1F1F1F015377697463681F0120
:101440004D4F4445531F015761726E696E671F010E
:101450004D756C7470781F0144656C617920446F20
:10146000776E1F0144656C61792055701F01536CC4
:101470006F772020446F776E1F01536C6F772020A9
:1014800055700045444954204D495820004F5000A4
:1014900054656D706C61746573005343092B0D2A9C
:1014A000122F00044C314C324C334C344C354C36FA
:1014B0004C374C384C394C414C424C434C444C45D5
:1014C0004C464C474C484C490048010546697273EC
:1014D000744C61737420005363616C6572204E61BB
:1014E0006D6500536F757263651F1F4F6666736588
:1014F000741F4D756C7469706C6965721F446976F0
:1015000069736F721F556E69741F5369676E1F444C
:101510006563696D616C731F4F6666736574204106
:1015200074006601034F46464F4E20005A07042DB3
:101530002D2D2D4131202041322020466173205332
:101540004331205343322053433320534334005319
:10155000696E6B20546F6E6573005A02042D2D2D39
:101560002D767370644132202000464153204F662F
:10157000667365741F566172696F3A20536F757296
:1015800063651F015377697463681F0153656E7348
:10159000697469766974791F1F43757272656E7418
:1015A00020536F7572636500437573746F6D2044CB
:1015B0006973706C617900477073416C744D616937
:1015C0006E004E756D20426C6164657300420303CA
:1015D0002D2D2D59656C4F7267526564005278004D
:1015E000547852535349616C726D00600301762D3B
:1015F0005641004120206368616E2E004801034D72
:101600006574496D7000480105467248756257530C
:101610004868690055737250726F746F1F556E6918
:101620007473005B2D3E5D00435600505245534598
:1016300054004355525645006A01032D2D2D494E45
:10164000560053575220003C0203443136443820A0
:101650004C52503C0203416D654A617045757256AB
:101660006F696365004C2E53776974636865730016
:101670004D697865720044696167416E6100446933
:101680006167537774636800417564696F4861707E
:101690007469630043616C6962726174696F6E00A2
:1016A000436F6E74726F6C7300416C61726D730086
:1016B00048617264776172650047656E6572616C3E
:1016C0000056657273696F6E00547261696E65725F
:1016D00000446973706C61790030313233343536CF
:1016E00037383971776572747975696F70617364B1
:1016F0006667686A6B6C207A786376626E6D5F2DC0
:101700002E20005B4D454E555D205748454E2044E8
:101710004F4E4500454449540053454C4543540001
:1017200053454C2F4544495400434F5059004D4FA9
:1017300056450044454C455445004241434B5550A5
:1017400000524553544F5245004544495400494EB8
:101750005345525400434F5059004D4F5645004495
:10176000454C45544500434C45415220414C4C00AA
:101770000473494478735448527352554473454C2A
:10178000457341494C734745417354524E0012080A
:101790001200081C0808081C080000082200490064
:1017A00022080000000000227F2200000008220022
:1017B0004900220800000822004900220800000019
:1017C000227F2200000000000822004900220800B9
:1017D00000081C0808081C08005343004756000175
:1017E00001010000000202020202020202020200E3
:1017F00002020202020202020000000000000002D7
:1018000002020202030303030005466565742056C5
:101810006F6C74734465675F434465675F466D41F1
:10182000682020416D7073204D6574726557617436
:10183000747300465643466D416D5718242F2F0090
:1018400033383B54656D706C6174657300015245AB
:1018500054410050726F746F636F6C00476C6F621D
:10186000616C5661727300536166657479205377B9
:101870007300437572766573004D6F646573004540
:1018800078706F2F44720048656C692053657475D9
:1018900070004C696D6974730054656C656D657496
:1018A0007279004D6F64656C2053656C65637400DC
:1018B0004D6F64656C205365747570004C61737472
:1018C000204D656E7500526164696F2053657475B3
:1018D0007000537461746973746963730042656561
:1018E0007020636F756E74646F776E004D696E75EE
:1018F0007465206265657000032D2D2D52746D4551
:10190000746D54746D41746D52454E527564456CDE
:101910006554687241696C50312050322050332038
:10192000000420204F4E204F4646424F544820414D
:101930004C4C4F4E434500072D2D2D2D2020207659
:101940003E76616C2020763C76616C20207C767C33
:101950003E76616C7C767C3C76616C414E44202006
:1019600020204F522020202020584F52202020207D
:1019700076313D3D7632207631213D76322076310A
:101980003E7632202076313C763220204C617463E2
:10199000682020462D466C6F702054696D654F6637
:1019A0006676603D76616C20312D53686F7420310E
:1019B0002D53686F7452004E616D65000657617259
:1019C0006E31205761726E32204368656570205217
:1019D000696E672020536369466920526F626F7495
:1019E00020436869727020546164612020437269E9
:1019F000636B74536972656E20416C6D436C6B52FE
:101A000061746174615469636B2020486170746310
:101A10003148617074633248617074633300546993
:101A20006D6572005452453031324147470052785B
:101A30003D000354783D53777200204142434445B2
:101A4000464748494A4B4C4D4E4F505152535455BE
:101A5000565758595A6162636465666768696A6B6C
:101A60006C6D6E6F707172737475767778797A3089
:101A70003132333435363738395F2D2E00000102CC
:101A800003FEFF0405060A0B0C0D0E0F23FD202498
:101A900025261D1E1F27F6F7F8F9FAFBFCF528117D
:101AA000292AF1F2F3F4F0042D2D2D2D41313D20A2
:101AB00041323D20525353495453534954696D3177
:101AC00054696D32416C742047616C744773706463
:101AD00054313D2054323D2052504D204655454C06
:101AE0004D6168314D61683243766C744261747443
:101AF000416D70734D61682043746F744661735615
:101B000041636358416363594163635A5673706418
:101B1000477672314776723247767233477672343F
:101B200047767235477672364776723746776174F4
:101B3000527856204864672041333D2041343D208F
:101B400053433120534332205343332053433420F3
:101B5000546D4F4B00032D2D2D783E30783C307C5A
:101B6000787C663E30663C307C667C633120633234
:101B700020633320633420633520633620633720AD
:101B8000633820633920633130633131633132632C
:101B900031336331346331356331360004503120E1
:101BA00020503220205033202048414C4646554C8E
:101BB0004C43594331435943324359433350504DB9
:101BC0003150504D3250504D3350504D3450504D97
:101BD0003550504D3650504D3750504D38434831A8
:101BE000204348322043483320434834204348357B
:101BF000204348362043483720434838204348395B
:101C00002043483130434831314348313243483131
:101C100033434831344348313543483136535743D1
:101C200048475631204756322047563320475634CE
:101C300020475635204756362047563720544849C6
:101C40005300537769746368205761726E696E67D9
:101C50000067656E7772697465206572726F7200D5
:101C6000454550524F4D20466F726D617474696ED8
:101C7000670042616420454570726F6D2044617455
:101C80006100434845434B204D4F44454C20544947
:101C90004D45525300434845434B204D49582F442E
:101CA0005220534F5552434553004D4F44454C200D
:101CB00020202020004D4520202020202020200012
:101CC000454550524F4D206F766572666C6F7700B8
:101CD000E2AEA6A4A22F2500000000000000000034
:101CE00000000000000000000000000000000B07E2
:101CF000000000C0C0C0C0C0C0C0000000000000A4
:101D000000000000000000000000000606000000C7
:101D10000080E0781E06181E0701000000F8FC8E07
:101D2000C66EFCF8070F1D181C0F07080CFEFE00FE
:101D3000000018181F1F1818000C0E86C6EE7C38FD
:101D40001E1F1B1918181806C6C6C6EEFC38181830
:101D500018181D0F07C0E0B0988CFEFE01010101AC
:101D6000011F1F7E7E6666E6C686060C18181C0FCD
:101D700007F8FCE666E6CC88070F1C181C0F070660
:101D80000606C6E67E1E001C1F0300000038FCEE9F
:101D9000C6EEFC38070F1D181D0F0778FCCE86CE47
:101DA000FCF8040C1D191D0F070000003030000066
:101DB00000000003030000E0F89C869CF8E01F1F71
:101DC0000101011F1FFEFEC6C6EEFC381F1F1818BA
:101DD0001D0F07F8FC0E060E0C08070F1C181C0C34
:101DE00004FEFE060E1CF8F01F1F181C0E0703FE53
:101DF000FEC6C6C606061F1F1818181818FEFEC60F
:101E0000C6C606061F1F0000000000F8FC0E06CE26
:101E1000CCC8070F1C18181F0FFEFEC0C0C0FEFE66
:101E20001F1F0000001F1F0606FEFE0606001818F2
:101E30001F1F18180000060606FEFE060E1E1818C4
:101E40001F0F00FEFEF0381C0E061F1F03070E1C9E
:101E500018FEFE00000000001F1F1818181818FEBA
:101E6000FC187018FCFE1F1F0000001F1FFEFC70F6
:101E7000C080FEFE1F1F0000030F1FF8FC0E060EA1
:101E8000FCF8070F1C181C0F07FEFEC6C6EE7C38B8
:101E90001F1F0000000000F8FC0E060EFCF8070FE4
:101EA0001C1B1E0F1BFEFE86C6EE7C381F1F030781
:101EB0000E1C18387CEEC6C68E0C0C1C18181D0F94
:101EC000070606FEFE06060000001F1F000000FEBB
:101ED000FE000000FEFE070F1C181C0F07FEFE0090
:101EE0000000FEFE01070E180E0701FEFE00800036
:101EF000FEFE1F0F0603060F1F1E3EF0E0F03E1E03
:101F00001E1F0301031F1E7EFEC0C0FE7E000000D8
:101F10001F1F0000000686C6E6F67E3E1F1F1B1927
:101F200018181800000000000000181818181818D9
:101F3000180060606060E0C0060F1F1B1B1F1FFEC3
:101F4000FEE060E0C0801F1F1C181C0F07C0E0E00F
:101F50006060E0C00F1F1C18181C0C80C0E060E01F
:101F6000FEFE070F1C181C1F1FC0E0606060E0C071
:101F70000F1F1B1B1B1B01C0F8FCCEC60E0C001F45
:101F80001F00000000C0E0703070E0C003C7CECC7E
:101F9000EE7F3FFEFEC0E0E0C0801F1F0100001F7B
:101FA0001F000060E6E600000000181F1F18000078
:101FB000000000E3E300307060607F3F00FEFEC081
:101FC000E07038181F1F03070E1C18000006FEFEE5
:101FD00000000000181F1F1800E0E060C060E0C0B3
:101FE0001F1F0001001F1FE0E0C0E0E0C0801F1FB6
:101FF0000100001F1F80C0E060E0C080070F1C18B8
:102000001C0F07E0F0703070F0E0FFFF0E0C0E0FB9
:1020100007E0F0703070F0E0070F0E0C0EFFFFE0ED
:10202000E0C06060E0E01F1F0000000000C0E06052
:1020300060606060191B1B1B1B1F0E6060FEFE6052
:10204000600000000F1F181C0CE0E0000000E0E042
:10205000070F1C1C0E1F1FE0E0000000E0E001075E
:102060000E180E0701E0E0000000E0E00F1F180E60
:10207000181F0F60E0800080E060181C0703071C39
:1020800018E0E0000000E0E007CFCECCEC7F3F603E
:1020900060606060E0E01C1E1E1B1B191900000040
:1020A00000000000006F000007000700147F147F8D
:1020B00014242A7F2A1223130864623649552250B9
:1020C0000005030000001C2241000041221C0014F6
:1020D000083E081408083E080800503000000808B0
:1020E00008080800606000002010080402003E4953
:1020F000453E0000427F4000625149460041494947
:1021000036001814127F0027454539003E494932F0
:1021100000017905030036494936000649291E00A9
:102120000036360000005636000008142241141410
:102130001414144122140800020151090600060972
:1021400009067E0909097E7F494949363E414141D8
:10215000227F4141221C7F494949417F09090901E8
:102160003E4149497A7F0808087F00417F410020AD
:1021700040413F017F081422417F404040407F02A0
:102180000C027F7F0408107F3E4141413E7F0909D8
:1021900009063E4151215E7F0919294626494949D0
:1021A0003201017F01013F4040403F1F2040201F7E
:1021B0003F4030403F63140814630708700807610C
:1021C00051494543007F414100020408102000416D
:1021D000417F0004020102044040404040080408DE
:1021E000100820545454787F4844443838444444B8
:1021F00020384444487F3854545418087E0901025A
:102200000C5252523E7F0804047800447D40002066
:1022100040443D007F1028440000417F40007C0482
:102220001804787C0804047838444444387C141436
:102230001408081414187C7C0804040848545454E6
:1022400020043F4440203C4040207C1C2040201C77
:102250003C4020403C44281028440C5050503C4402
:1022600064544C44000836410000007F00000041E7
:102270003608000808221C08081C22080804027FEF
:10228000020410207F20100102040810204080402A
:10229000800804201002019CCE003264E2F100327A
:1022A00064645A505A6450463C46649C141E465A14
:1022B000536572766F20546573742838290053650E
:1022C00072766F205465737428313629004779720D
:1022D0006F2053657475700048656C692053657490
:1022E000757000456C65766F6E5C44656C7461005A
:1022F000562D5461696C00537469636B7920542DB9
:1023000043757400542D4375740053696D706C658A
:1023100020342D4348000A230423F722F022E3222D
:10232000D822CD22BE22B0220000891112239B3276
:102330002446AD573665BF74488CC19D5AAFD3BE95
:102340006CCAE5DB7EE9F7F88110080193331A22A5
:10235000A5562C47B7753E64C99C408DDBBF52AE75
:10236000EDDA64CBFFF976E802218B301002991385
:102370002667AF763444BD554AADC3BC588ED19F55
:102380006EEBE7FA7CC8F5D983310A209112180365
:10239000A7772E66B5543C45CBBD42ACD99E508F35
:1023A000EFFB66EAFDD874C904428D5316619F7035
:1023B0002004A9153227BB364CCEC5DF5EEDD7FC15
:1023C0006888E1997AABF3BA85520C4397711E6025
:1023D000A1142805B3373A26CDDE44CFDFFD56ECF5
:1023E000E9986089FBBB72AA06638F7214409D5105
:1023F0002225AB343006B9174EEFC7FE5CCCD5DDD5
:102400006AA9E3B8788AF19B87730E6295501C41E4
:10241000A3352A24B1163807CFFF46EEDDDC54CDB4
:10242000EBB962A8F99A708B088481951AA793B6C4
:102430002CC2A5D33EE1B7F04008C919522BDB3AB4
:10244000644EED5F766DFF7C899400859BB712A684
:10245000ADD224C3BFF136E0C1184809D33B5A2A94
:10246000E55E6C4FF77D7E6C0AA583B41886919764
:102470002EE3A7F23CC0B5D14229CB38500AD91B74
:10248000666FEF7E744CFD5D8BB502A49996108744
:10249000AFF326E2BDD034C1C3394A28D11A580B54
:1024A000E77F6E6EF55C7C4D0CC685D71EE597F414
:1024B0002880A1913AA3B3B2444ACD5B5669DF7834
:1024C000600CE91D722FFB3E8DD604C79FF516E404
:1024D000A9902081BBB332A2C55A4C4BD7795E6814
:1024E000E11C680DF33F7A2E0EE787F61CC495D5E4
:1024F0002AA1A3B03882B193466BCF7A5448DD59F4
:10250000622DEB3C700EF91F8FF706E69DD414C5C3
:10251000ABB122A0B9923083C77B4E6AD5585C49D3
:10252000E33D6A2CF11E780F2B050A0C0D0B102BC6
:102530002B082B2B2B2B2B2B0406171A11131415DE
:102540001609181B122B2B2B2B07191C1D1E1F27BE
:10255000202122262B00708F11241FBECFEFD0E147
:10256000DEBFCDBF11E0A0E0B1E0E2EDF0E201E0BE
:102570000BBF02C007900D92A231B107D9F71FE03F
:10258000A2E1B1E001C01D92A335B107E1F715E268
:10259000C8E5D5E200E006C022970109FE010BBFA5
:1025A0000E943290C635D10780E00807A9F70E9443
:1025B000FF8D0C9467900C940000E0915E0694E00F
:1025C000E99FF0011124E80FF11DED58FC4F8491B3
:1025D0008F5F0895F8948091790D90917A0D789499
:1025E0000895E82FF0E0E65AFC4F849108952AE020
:1025F000829FC00111248E589D4F089590916006CE
:1026000091708091C90586FB882780F989270895F4
:102610000F93022F207104FF03C00F7E9DE201C0C3
:1026200094E2411104C024E04EE453E00EC0453072
:10263000A0F49091C90594FF0BC0006194E0499FFC
:10264000A00111244858594F24E00E94497716C030
:102650002FEF240F43E853E00FC0941728F02BEF1F
:10266000240F4CE95BE108C0222311F0475B491BB2
:102670002CED240F47EA5AE10E946D770F910895DF
:102680000F93CF93DF93C82FD62F022F411104C091
:1026900024E049E453E00DC04A3010F086E101C067
:1026A00081E18C0F202F6D2F0E94FD7922E046E4FE
:1026B00053E06D2F8C2F0E944977DF91CF910F91BE
:1026C0000895CF93DF93E6E8F1E080918C061082C5
:1026D00091E0918381FF09C092E2928393E2938318
:1026E000EF01259694E2948304C0EF01239692E0D3
:1026F000928382FF09C09FE1988390E29983FE0153
:10270000339691E29A8304C0FE01319693E0988358
:1027100094E0908395E0918396E0928384FF09C0D2
:1027200095E2938396E29483EF01269697E2958350
:1027300004C0EF01249697E0938385FF09C098E2D7
:10274000988399E29983DE0113969AE29A8304C0F2
:10275000DE01119698E0988399E09C93FD0186FD37
:1027600002C0319604C032969BE2ED01998387FF47
:1027700003C08CE280833196DF018AE08D938F5F06
:102780008C31E1F7828BCF018457914080935801BF
:102790002DE1238B40E099270196242F30E082170A
:1027A000930754F0F901EA57FE4FE081F0E0E75A51
:1027B000FE4F40834F5FF1CF9091900690FF0AC08B
:1027C000809164008B7F80936400809165008460B9
:1027D0008093650091FF02C0BF98C79ADF91CF91A7
:1027E000089587FF03C0819591E001C090E0E82F34
:1027F000FF27E7FDF095E75AFE4F80819111819503
:10280000089587FF03C0819591E001C090E0E82F13
:10281000FF27E7FDF095EA57FE4F808191118195E2
:1028200008950F931F93CF93DF93D62FC42F022FBA
:1028300016E0180F442339F04C3141F0443E81F446
:102840004CE953E005C042E453E002C048E953E0DC
:102850006D2F812FDF91CF911F910F910C947F7776
:1028600047FF04C041E20E949176C1952FEF2C0FE3
:102870002D3114F02CEF2C0F40EA53E06D2F812FF7
:102880000E946D77DF91CF911F910F9108950F9363
:102890001F93CF93DF93D82F162FC42F022F4D32C3
:1028A00034F04DE682E18D0F0E949176CC52202FBC
:1028B0004C2F612F8AEF8D0FDF91CF911F910F91D8
:1028C000B0CFDF92EF92FF920F931F93CF93DF93DE
:1028D000D82F162FF42E27FF03C0E2E1F2E002C04A
:1028E000EDE0F2E0C281D3802370E22E81E0821716
:1028F00018F1C4306CF483E0C802A00111244B5CD1
:102900005C4F0F2D23E0612F8D2F0E94497718C057
:10291000CD5F0F2D2C2F45E55BE1612F8D2F0E94A0
:102920006D77C0310CF4D6502F2D45E2612F82E136
:102930008D0F0E94917604C082E028130AC004C063
:10294000E11007C0C13029F42F2D4D2D612F8D2F9F
:102950009EDFDF91CF911F910F91FF90EF90DF905D
:1029600008951F93CF93DF93EA0194E0699FF001EC
:102970001124EB50FB4F408150E01381107C103844
:1029800011F4440F551F9A01A82FB0E00E947A8FCE
:10299000103C49F424E630E040E050E00E94EE8F25
:1029A00091E081E41EC04436510570F4103461F0AA
:1029B000660F771F881F991F23E330E040E050E047
:1029C0000E94EE8F92E009C02FEF30E040E050E02F
:1029D0000E94EE8F103419F091E086E702C090E07B
:1029E00080E2209709F0988380935701C901DF9115
:1029F000CF911F910895DF92EF92FF920F931F9353
:102A0000CF93DF931F92CDB7DEB7D82EF62E842F4B
:102A1000102FAE014F5F5F4F622FA3DFAC018981A2
:102A2000813011F4106203C0823009F41063809188
:102A30005701863781F49A0140E050E065E0E62EC8
:102A4000012F6F2D8D2D0E94C27817FD16C0212FEA
:102A5000409157010DC0212F6F2D8D2D0E94CD79F2
:102A600080915701813449F417FD07C0212F41E4BB
:102A70006F2D8091650D0E949176809157010F9086
:102A8000DF91CF911F910F91FF90EF90DF9008950C
:102A9000873038F4E82FF0E0EE0FFF1FE15CF74FCE
:102AA00024C08C3050F18431C0F4482F50E0DA015A
:102AB000AA0FBB1FA45FBE4F2D913C91803148F4FB
:102AC000FA01EE0FFF1FEC5CF94F80819181281B0A
:102AD000390BC901880F991F0895843248F4E82FF3
:102AE000F0E0EE0FFF1FE950F84F808191810895CB
:102AF0008E3418F484520C947D2B80E090E008957D
:102B00000E94FB8D882311F0A895FACF1092A90D91
:102B100008951F93CF93DF93EC01162F0E94457603
:102B2000BE0188E10E94A47712FF04C067E182E140
:102B30000E94928710FD11C011FF06C06FE173E083
:102B400080E30E94A47706C041E153E068E38CE192
:102B50000E94BA774CE653E002C049E053E024E01B
:102B600060E086E1DF91CF911F910C947F7761E067
:102B7000D0DF0C94F57A0F93262F00E040EA53E063
:102B800060E10E946D770F9108951F93CF93DF93BB
:102B9000C6E110E08C2F0E94EE7B110F182BC15064
:102BA000CE30C1F780918C0682FF12C08FE10E9467
:102BB0009C7C24E0829FE0011124137CC12B84E0E3
:102BC0000E949C7C20E1829FC00111241C2F182BA5
:102BD000812FDF91CF911F91089570E0882399F0A4
:102BE00090E0019725E0289FF001299FF00D112426
:102BF000E60FF71FEE0FFF1FE35EFA4F8081918112
:102C00008B509E4F0895FB01E65CFB4F8081992716
:102C100087FD909508951F93CF93DF93D82F162F9C
:102C2000C4E0DD2391F0612F8D2FD7DF9C01253F7C
:102C300081E0380764F08BE0820F8D1710F08CE094
:102C4000820FC15029F0D82FECCFC0E001C0CD2FAA
:102C50008C2FDF91CF911F910895CF93C62FDBDF8B
:102C60006C2FCF91BACF8E3791053CF483382FEF7C
:102C7000920734F483E89FEF03C08DE790E0089556
:102C80000895FF920F931F93CF93DF938A01C62F6E
:102C9000D0E08823D9F0BFDFF82E8823B9F0C8012F
:102CA000E2DF2F2D30E02150310945E0429FF00155
:102CB000439FF00D1124EC0FFD1FEE0FFF1FE35E8D
:102CC000FA4F855F91409183808305C0C801CBDFB7
:102CD000C65CDB4F888386E0DF91CF911F910F9117
:102CE000FF900C943B7090914A01911103C08111A7
:102CF00006C00895811103C08FEF890F01C080E0E5
:102D000080934A018EEB809349010895E0914A0136
:102D1000F0E0EE0FFF1FE55BFE4F918380838FEBAA
:102D2000809349010895809162062AEF829FC00135
:102D30001124880F991F20913A0130913B012817E7
:102D4000390720F490933B0180933A010895EEE413
:102D5000FEE037A1303180F420A541E0420F40A7CA
:102D6000DF01A20FB11DA20FB11D8D939C934031C5
:102D700008F010A63F5F37A3089590E08C5F9E4F48
:102D8000E6CF90E0E4CF8093230290E04097DFCF3E
:102D90000F931F93CF93DF93EC018091690681FF1E
:102DA00007C180917A0686FF89C012E001E00E9487
:102DB0009C7D8F3F2FEF920781F029A9211104C03C
:102DC0008F31A9F709ABF3CF213011F419ABEFCF55
:102DD000223069F78AAB19AAEACF8EA1813041F57A
:102DE0003FA1332309F452C029A5FE01E20FF11DD2
:102DF000E20FF11D808191812F5F203108F020E0EA
:102E000029A731503FA32091D30121FDE0C097FDB8
:102E100002C021E101C028E22BA32FE12AA722E072
:102E20002BA78CA79DA718AA84E08FA72EA32EC03E
:102E3000811106C08091780D8D3340F186E025C068
:102E4000823021F19AA99078833049F4992329F0AE
:102E50008BA181508BA3811119C084E016C08430EE
:102E600021F4992399F083E00EC0853039F48BA1C9
:102E700081508BA381110AC081E007C0863031F4F4
:102E8000992321F084E18BA385E08EA38EA182306B
:102E900009F49DC08BA98F5F8BAB8A3008F497C073
:102EA0001BAA8DE18AA781E08BA798A1911101C08F
:102EB00080E08CA718AA83E08FA789C098A189A178
:102EC000992311F0846001C08B7F89A38EA181308A
:102ED00081F5C79A2FA1222349F189A531E0380F46
:102EE00039A7FE01E80FF11DE80FF11D80819181E6
:102EF0009DA38CA3303108F019A621502FA3209157
:102F0000D30121FD64C097FD02C021E101C028E288
:102F10002BA329A12C7F97FD226029A389A18BBB1C
:102F2000C7988FE18AA382E08EA351C089A18BBB91
:102F30004DC081110CC0C79A89A1836089A38BBB46
:102F40008091780D8D3308F441C086E02FC0823027
:102F500009F43DC089A18BBBC79ABF9800C000008F
:102F600000C086B38078BF9A9EA1933049F488232D
:102F700029F08BA181508BA3811128C084E016C059
:102F8000943021F4882311F183E00EC0953039F498
:102F90008BA181508BA3811119C081E007C09630AD
:102FA000A9F4882399F084E18BA385E08EA30EC059
:102FB0008091900681FD0BC08091660686FB882774
:102FC00080F998A1981711F0C79A01C0C798DF91AE
:102FD000CF911F910F91089590915E0690FD02C0D0
:102FE00093E08927E82FF0E0E35BF74FE081E7FD0E
:102FF000E95FE595E595E5951E1624F0EE2321F0B1
:10300000E19502C080E801C080E0E83008F0E7E028
:10301000F0E0ED5AFC4FE491EE2319F099E0909323
:1030200055018E2B0895853030F46FEF680F809135
:10303000030713DE24C08D3080F4E82FF0E0EE0F9C
:10304000FF1FED5CF74F8081918197FD0796E3E0CC
:1030500095958795EA95E1F712C08D3170F4E82FC8
:10306000F0E0EE0FFF1FEB5FF74F808191816AE088
:1030700070E00E94DB8FCB0102C080E090E0F3CDD6
:10308000482F833021F0882321F0E82F03C0E0E0AF
:1030900001C0E3E0F0E0EE0FFF1FED5EFE4F808128
:1030A0009181443080F420917B0630E002C0359558
:1030B00027954A95E2F720FF06C020E038E0A901F5
:1030C000481B590BCA0108951F93CF93DF9310E05B
:1030D000C0E0D0E0812FD4DFC80FD91F1F5F1430AC
:1030E000C9F7C058DF4F8D2F90E0DF91CF911F912E
:1030F0000895CF9380915E068170C2E0C81B8C2F2B
:10310000BFDF6C2F0E945E4B2091C90525FF05C0D3
:103110000F964F9728F080E004C081319C4FDCF778
:1031200081E0CF910895E3E1F1E040E0842F8064F5
:1031300087B900C000C0369A3699FECF24B135B1A8
:10314000369A3699FECF84B195B1820F931F369A85
:103150003699FECF24B135B1280F391F369A3699EA
:10316000FECF84B195B1820F931F96958795819379
:1031700091934F5F4830D1F6089578941F920F9243
:103180000FB60F9211248F93809112018F5F80935D
:1031900012018F910F900FBE0F901F901895789489
:1031A0001F920F920FB60F9211240BB60F922F930E
:1031B0008F939F93CF93DF93EF93FF93F89487B709
:1031C0008F7B87BF78942091D7018091D90190910E
:1031D0006906882359F090FF07C08091520F820F33
:1031E0008093520F87FF02C01B9A01C01B9891FF6A
:1031F00050C080917A0686FF22C0EEE4FEE087A5EB
:10320000882309F446C080911702811142C0809141
:103210009B0085FF0DC080A991E0980F90ABEF0156
:10322000C80FD11D8AA580939C0087A5815087A7D0
:1032300087A581112EC086A1823059F526C08091C4
:103240006209811126C0EEE4FEE086A1823009F514
:1032500083A1882311F081501BC021A1C79A82A1AC
:1032600080FD09C02D7F84A195A196FD2260880F65
:10327000991F95A384A381E082278BBB81A3C79864
:1032800082A1815082A3811104C083E086A385E0DE
:1032900083A3F89487B7806487BF7894FF91EF91F8
:1032A000DF91CF919F918F912F910F900BBE0F9037
:1032B0000FBE0F901F90189578941F920F920FB623
:1032C0000F9211240BB60F922F933F934F935F935E
:1032D0006F937F938F939F93AF93BF93EF93FF93DE
:1032E00081B7845681BF85ED91E00E94D0850E9410
:1032F000CC7C0E94E88C8091B10D82608093B10DEE
:10330000E2E0F1E08081815011F0808304C084E626
:10331000808381E081838281815011F0828305C0A6
:103320008AE08283838181608383FF91EF91BF91E3
:10333000AF919F918F917F916F915F914F913F914D
:103340002F910F900BBE0F900FBE0F901F901895EE
:1033500078941F920F920FB60F9211240BB60F9212
:103360002F933F934F935F936F937F938F939F938D
:10337000AF93BF93EF93FF93209180003091810032
:10338000F89480917D008F7D80937D00789480916A
:10339000AB069091AC06A901481B590BCA01969542
:1033A00087953093AC062093AB06409123019C0196
:1033B000215A3F402F3D3E4230F12FEF240F28305D
:1033C00028F59C012152334027373540F0F424E69C
:1033D00020932202E42FF0E0EE0FFF1FEE5DFE4F80
:1033E0009C012C5D354050916406565F529FC00190
:1033F000539F900D11246AE070E00E94DB8F71836F
:1034000060834F5F03C041E001C040E0409323016F
:10341000F89480917D00806280937D007894FF9184
:10342000EF91BF91AF919F918F917F916F915F913C
:103430004F913F912F910F900BBE0F900FBE0F90A9
:103440001F90189590E0880F991F8455914FFC01AB
:10345000F894808191817894089584E0F3DF20913D
:10346000E5073091E607820F931F089592EC980FBD
:1034700081E0973008F080E00895FC018081882386
:1034800059F0843218F085520C94EA2B815000DBFD
:1034900040E060E00C949A8708959C0165E03595C2
:1034A00027956A95E1F7280F391FAC01440F452F86
:1034B000441F550B241B350B892F990F990B8595AC
:1034C000820F931F08959DE7980F9B3F88F08E57BA
:1034D000E82FF0E0EE0FFF1FE15FFA4F80818617C3
:1034E0001CF46083862F0895481714F44083842FBA
:1034F000089544E66CE9E7CF982F8091690284FF34
:1035000003C081E0923009F080E0089549E284022E
:1035100090011124359527953595279587FD815C78
:1035200086FB880F880B80F9A901481B510987FD8C
:103530005395CA0108955F926F927F928F929F92E6
:10354000AF92BF92CF92DF92EF92FF920F931F93B1
:10355000CF93DF93982E842E882309F4E7C12CE1C2
:10356000821721F034EE831303C0DCC181E0DFC198
:10357000992787FD909597FF03C0919581959109B3
:103580008D3191056CF00E94307C982F81E01914E8
:103590001CF49111CCC1C6C1992309F4C8C1C2C1A0
:1035A000892D87FD81958A3040F4825F0E94EE7BF1
:1035B00019140CF4BCC191E0B3C18A50082F10E07B
:1035C0008C3008F4EBC0E801CC0FDD1FCC0FDD1F01
:1035D000C75CDA4F8A81882309F4A4C194E0981566
:1035E00008F4EBC0A88079800E94F112811117C005
:1035F0008FEF8A0D4DDA6C01888185326CF05BEDBE
:10360000B52EB80E69818B2D0E940C2B7C018B2D61
:103610000E94DF2AB82E16C0898178DF09C0823067
:1036200059F48FEF8A0D34DA6C018981815030DAD8
:103630007C01BB24B39406C0BB24B394E12CF12CD1
:10364000C12CD12C4A8150E0FA013197E131F105CA
:1036500008F09EC0EA5BFF4F0C942C90D7FE4EC042
:10366000D194C194D1084AC0D7FE4DC0D194C19421
:10367000D10849C08881FADE882369F08AE0960182
:10368000829F6001839FD00C11249701829F70015B
:10369000839FF00C1124CE18DF083FE1C30ED11C2C
:1036A00091E08FE3C816D10408F44FC047C0EE2460
:1036B000E394E80C4E2D60E08A2D3DDFF82E4E2D70
:1036C00060E0872D38DF982F8A81853031F4FF2024
:1036D00009F45EC091115AC05BC0863019F4F11034
:1036E00055C033C09F2531C091E0CE14DF0431F5C1
:1036F0002CC091E0CE14DF0441F520C091E0EC1421
:10370000FD041CF11BC091E0CE14DF04F4F016C0E0
:10371000F801EE0FFF1FE155FE4F91819095991F23
:103720009927991F12C0F801EE0FFF1FE155FE4FB8
:1037300091E020813181121613063CF090E005C023
:10374000F801EF56F94F90819170BB2009F1992350
:1037500001F18B818823C1F097EF980F933108F422
:103760008F5F9BE1980F933110F4815002C08C3130
:1037700021F0843E19F487EF01C089E041E0480D53
:1037800060E0D9DE982F05C091E003C0B110E1CF11
:1037900090E08A818C3008F0C0C0BBC05801AA0CF0
:1037A000BB1CE501C00FD11FC255DB4F8A818F7052
:1037B00009F4B8C094E0981530F4F801EF56F94FC9
:1037C00090819170AAC0688059800E94F112811185
:1037D00017C08FEF860D5CD96C01888185326CF043
:1037E0009BED792E780E6981872D0E940C2B7C0130
:1037F000872D0E94DF2A782E16C0898187DE09C0B6
:10380000823059F48FEF860D43D96C018981815044
:103810003FD97C017724739406C077247394E12CFC
:10382000F12CC12CD12C8A818F7090E0FC01319752
:10383000EE30F10508F066C0E95AFF4F0C942C9069
:10384000D7FE32C0D194C194D1082EC0D7FE31C06A
:10385000D194C194D1082DC0EE24E394E80C4E2DF0
:1038600060E0862D68DEF82E4E2D60E0852D63DE4B
:10387000982F2A812F70253031F4FF2009F442C09F
:1038800081113EC03FC0263019F4F11039C025C067
:103890009F2523C091E0CE14DF0479F41EC091E08F
:1038A000CE14DF04D1F409C091E0EC14FD04ACF0B7
:1038B00004C091E0CE14DF0484F090E00EC0F50166
:1038C000E155FE4F91819095991F9927991F05C049
:1038D000F801EF56F94F90819170772099F0992374
:1038E00091F08A8182958F7049F089300CF08F5F5A
:1038F00041E0480D60E01FDE982F05C091E003C055
:103900007110EFCF90E02A812F7030E02C3031051C
:1039100024F4F801EF56F94F908319142CF081E04C
:10392000892705C080E003C0892F01C0862FDF9161
:10393000CF911F910F91FF90EF90DF90CF90BF90AC
:10394000AF909F908F907F906F905F90089540E030
:1039500060E0F1CD80914B06FADF811113C08091B8
:103960003A0190913B01892B69F410926E0E80917F
:10397000780D9091AF06981749F08093AF068EE4CA
:103980009EE006CA81E080936E0EF1CF0895CF933A
:10399000DF93C62F20915502222339F090935702CE
:1039A00080935602DF91CF91089564E0B2D80E94CF
:1039B000F57AC11103C08091480601C089E10E94D7
:1039C000C27A9ED8D1E00E94FB8D882319F0DF9146
:1039D000CF9196C88091B10D833019F4A8951092BB
:1039E000B10DCC2319F0D0936E0E02C010926E0E62
:1039F000B1DFE9CF60E0CBCFE0914A01E43018F0CD
:103A000086EB92E0F7CF2FEB20934901EF5FE09335
:103A10004A01F0E0EE0FFF1FE55BFE4F91838083CC
:103A2000089580915D0680FD16C07DDB62DB81110B
:103A300012C066E088EE92E06CD80E94F57A60D8F9
:103A400072DB88DFA89555DB811105C00E94FB8DD4
:103A50008823B1F355C80895DF92EF92FF920F9338
:103A60001F93CF93DF9380915D0681FD90C0C0913D
:103A70000705F090190680918C0682FD0CC08C2FF2
:103A80008873883041F0803131F0803221F0C77C7A
:103A9000C860C0930705E12CDD24D39476D8182F95
:103AA00085E20E949C7C082FD12FDC276E2D62605E
:103AB00083EC92E02ED8D0FF03C060E082E05BD8B8
:103AC000D1FF03C061E087E156D880918C0682FF68
:103AD0001AC08D2F8C7051F0612F70E0759567952D
:103AE000759567956370655E8CE245D88D2F807300
:103AF000F9F0612F70E0F4E075956795FA95E1F7BC
:103B000063706D5F13C0D2FF03C062E08CE233D8F4
:103B10008D2F887369F013FF02C063E007C014FFA4
:103B200002C064E003C015FF03C065E081E423D850
:103B300080918C0684FF0AC0802F8F25837061F0EE
:103B4000602F63706F5D86E516D806C0D6FF03C090
:103B500066E086E510D80F2DD7FF03C067E08BE63F
:103B60000AD80E94F57ADD2029F00E948015E4E051
:103B7000EE2E01C0E12C1C1302C00F1541F00E9473
:103B8000FB8D811104C0E6DEA895D12C87CFDF9193
:103B9000CF911F910F91FF90EF90DF9008958111C9
:103BA000C2D880913A0190913B01009709F00197AA
:103BB00020913901222361F020916A064AEF249F67
:103BC00090011124220F331F8217930708F4C901B3
:103BD00090933B0180933A01BDCE7F928F929F924A
:103BE000AF92BF92CF92DF92EF92FF920F931F930B
:103BF000CF93DF930E94EA122091AD063091AE067A
:103C0000AC01421B530B4B30510538F01092B306F8
:103C10001092B206FF24F39401C0F12C9093AE06EB
:103C20008093AD06D0908C06CEE0D0E098E0C92E0F
:103C300000E010ECB12C5D2D5470A52E8D2D8071FF
:103C4000982E8C2E2091B2063091B306202331237A
:103C50000C2E02C0369527950A94E2F7722EEC2CB2
:103C60008C2D75DE43E0C41651F057E0C5120FC02D
:103C7000992079F085E20E949C7C95E206C0AA20FA
:103C800051F08FE10E949C7C9FE1980F05C09C2D14
:103C900003C097E001C093E0781631F1282F30E09F
:103CA00002C0220F331F8A94E2F7A8014095509575
:103CB0006091B2067091B30646235723242B352B0F
:103CC0003093B3062093B206993010F0E92E0DC060
:103CD0009CEF9C0D933018F4811107C005C0811131
:103CE00004C0EC2CE19401C0EB2C169507951695B9
:103CF0000795CA942297CC2011F0BE2CA2CFCE2DCE
:103D0000E11012C089E023DE282F30E04091B10697
:103D1000C901842780FF08C0232B09F0C9E081E096
:103D200084278093B106EC2ED6FE16C0E11014C095
:103D30008BE20DDE282F30E0220F331F4091B106B9
:103D4000C901842781FF08C0232B11F0DBE2ED2E8F
:103D500082E084278093B106D7FE16C0E11014C01C
:103D60008CE2F5DD94E0899F900111249091B106D9
:103D7000A901492742FF08C0232B11F0CCE2EC2E09
:103D800084E089278093B106F110E12C8E2DDF911C
:103D9000CF911F910F91FF90EF90DF90CF90BF9048
:103DA000AF909F908F907F900895AF92BF92CF92E7
:103DB000DF92EF92FF920F931F93CF93DF938C01CB
:103DC0007B016A01A22EB09018029B2D9F7D943436
:103DD00039F080911D08882309F4A6C0933479F442
:103DE000B19906C080913E01E801C80FD11D02C003
:103DF000E801219683E10E94888785E010C0953410
:103E000019F0923409F093C0B1998BC080913E01B2
:103E1000E801C81BD10984E10E94888784E00E94E0
:103E2000EE7B811173C0E114F104F9F481E0C8164E
:103E3000D104D9F480E6B81619F08EE2B81211C098
:103E400010921D08C1E00115110509F0C0E0D0E095
:103E50008B2D0E94BD7C8EE2B81206C010925308D2
:103E600003C0C170DD2701C0B12CA3FE09C0B5DEBF
:103E7000882331F00E94F113C82FDD27C7FDD095AC
:103E80004091410150914201C41BD50B80915308D0
:103E9000813071F440912102B19905C084E148025A
:103EA000A001112403C0552747FD5095C40FD51F0D
:103EB000CC16DD0644F48B2D0E94BD7C83E10E946C
:103EC0008887E6010AC0CE15DF053CF48B2D0E94E1
:103ED000BD7C84E10E948887E701C017D10749F1C2
:103EE000B19903C08FEF8093B006209751F48B2DCA
:103EF0000E94AD7C17FF02C083E101C084E10E94F3
:103F000088878A2D83700E943B7013C0CC27DD27E1
:103F1000C01BD10B85E00E94BD7C84E00E94BD7C6B
:103F200082CFE801219777CF953409F46DCFE8016E
:103F30007ACFCE01DF91CF911F910F91FF90EF903B
:103F4000DF90CF90BF90AF900895552747FD5095D3
:103F5000772767FD7095992787FD909526CF20914B
:103F60001608F3CF462F2091160860E0EECF462FBB
:103F700050E02091160860E070E017CF1F93CF93B8
:103F8000DF93D62F142FC22F0E94F113412F5527F4
:103F900047FD50956D2F772767FD70952C2F99273A
:103FA00087FD909502DFDF91CF911F910C94011452
:103FB0001F93CF93DF93C5E2D5E090E0888111E0B5
:103FC000190F882329F0C3DC882311F0812F05C045
:103FD000912F2A96143091F780E0DF91CF911F91B5
:103FE00008958F929F92AF92BF92CF92DF92EF92FD
:103FF000FF920F931F93CF93DF93EC01A62EB12C6A
:104000006501CC0CDD1CF601EC5DFD4F00811181DA
:104010008981882309F457C08D809E8088818150D2
:104020000E9448157C018981853038F4833050F432
:10403000813079F0823091F039C08530A1F086303E
:1040400071F134C0F7FE03C0F194E194F1088330BC
:1040500029F481E08E149F043CF125C081E0E8142E
:10406000F90414F120C0888101DA882369F08AE01C
:104070009701829F7001839FF00C1124F4018E9FA1
:1040800040018F9F900C1124E818F908FFE1EF0E12
:10409000F11C81E02FE3E216F10430F004C081E06E
:1040A000E814F90409F080E0E82EF12C8A818111EE
:1040B00004C0EF2829F081E01BC049DC8111F9CF51
:1040C00000E010E014C08A81882331F040DC8111C7
:1040D0000BC00FEF1FEF0CC08B81833040F09C8131
:1040E000907681E029F403C080E091E002C080E096
:1040F00090E0892BF501EC5CFD4F5F01F080209191
:1041000005019B8121FD2EC0933059F48A810E94C4
:104110009C7CF81689F1FF24F394F80E00E010E07F
:104120002CC0813041F4F11003C0292F2D7FB1F054
:10413000913089F421C0F1E0FF120CC08FEF890F9C
:10414000823040F480E000E010E09230B1F432E0E0
:10415000F32E13C080E0913219F40CC000E010E09F
:10416000F82E0BC0FF24F394913209F0F12C0FEFDD
:104170001FEF03C00FEF1FEFF12CF50180838C813F
:1041800087FD03C0F1100BC07EC088818530D0F35D
:1041900085520E94DF2A882309F475C0F3CF17FFE8
:1041A00004C08B81833028F46EC00115110509F01D
:1041B00057C08C818076803211F4CE015ED98C811B
:1041C000877069F1813031F52F81822F98858C3F7E
:1041D000F1E09F0748F040E050E060E070E084E0EC
:1041E000820F0E945A2A0DC0853F21E0920748F0B5
:1041F000FC01EE0FFF1FEB5DFE4F8081992787FDCD
:1042000090952F2D30E021503109820F931F0E948D
:10421000A71605C060E070E08F810E948D878C81B9
:104220008076803411F4CE0128D98C81282F287112
:1042300081F0869586958695837090E0029724F0AC
:10424000283121F48FE003C08DE001C08EE00E9490
:1042500088878B8183508E31A0F00FEF1FEF13C042
:104260001016110684F40F5F1F4F8B813AE0839F75
:10427000C00111244397081719072CF000E010E043
:1042800002C001E010E0F601EC5DFD4F11830083F8
:10429000DF91CF911F910F91FF90EF90DF90CF9022
:1042A000BF90AF909F908F9008951F93CF93DF930F
:1042B000C1EDD5E010E0612FCE0193DE29961F5F9E
:1042C0001830C9F7DF91CF911F9108954F925F92F7
:1042D0006F927F928F929F92AF92BF92CF92DF9216
:1042E000EF92FF920F931F93CF93DF931092520898
:1042F0008091120102B7909112018913F9CF10E059
:10430000182B0E9493188EE587B91BBA8FE18ABBE0
:1043100000C099B38FEF8ABBE9E1F2E0878188237F
:1043200011F080E202C0892F807E8483292F207CB7
:104330008081281759F08074880F9078318189170F
:1043400011F0315001C03F5F31832083828193811E
:10435000891711F0838381838091790D9091A6064E
:10436000282F291B20933C018093A60680911702D9
:10437000811106C060E085EF97E00E94C55801C03A
:10438000A89580913C01882309F41BC3C4E3D1E0C4
:1043900080911B08882319F0815080931B080E948C
:1043A00064182B813C818217930741F09C838B8397
:1043B0001A82198281E0809339012DC060915F06D5
:1043C000665F49F180913D01823328F188818F5FDA
:1043D0008883803100F189819A8101969A8389834B
:1043E000188247E751E0649F9001659F300D1124CA
:1043F0002817390780F48F719927019761F480910C
:10440000D3018D7F8093D30186E00E94C3166DE2B5
:1044100080E10E9492870E944C3F0E94B63C8091AE
:104420002202882319F081508093220280E00E94AA
:104430008D700E9445760E94827BD82E8091170253
:10444000811102C23D2D3F70A32E4AEFA40EC091F0
:104450006A02C43021F0C33019F4C4E001C0C8E0DE
:1044600057E05A1508F495C08D2D807F803209F4ED
:1044700090C08A2D86950E94DD1290917A0690FD5B
:1044800004C0CC24CA94C80E03C094E0C92EC81A34
:104490006C2D809103070E940B16B82E6C2D0E9484
:1044A0002D167C01C1110CC0EC0197FF04C0CC2774
:1044B000DD27C81BD90BD595C795D595C795CF5F77
:1044C00082E0C8120FC08091690280FD02C0912C69
:1044D00003C099249394C2E00E94FE12882319F02D
:1044E000C19501C0912CDD27C7FDD095A0FE03C06A
:1044F000CE0DDF1D04C0F701EC1BFD0BEF01209773
:1045000021F08D2F8F2587FF11C091100FC0EF284C
:1045100069F040E050E06C2D8B2D0E9441168D2DEE
:104520000E94BD7C86E10E948887DFC59E012458D9
:104530003F4F293F310548F4AE016C2D8B2D0E9471
:1045400041166C2FC7FF18C016C01C161D061CF4A0
:104550004DE750E002C043E85FEF6C2D8B2D0E94C9
:104560004116CE0183589F4F8B3F910508F0BDC582
:104570006C2F1C160CF4619567FD6D5F6595659554
:10458000772767FD7095645C7F4F85E10E948D877A
:10459000ACC58D2D8F7B71F48091B006B19987C524
:1045A0008F3F31F08F5F883C19F48FEFCDEBDC2E1D
:1045B0008093B006EFE3F1E080914B0890914C08B6
:1045C00020813181281B390B37FF02C0215E3F4F0C
:1045D000B5E035952795BA95E1F72115310561F0DC
:1045E00024813581281B390B37FF02C02F5F3F4FD5
:1045F0003595279591838083958384838091600688
:1046000085FD04C080911908882311F020E030E076
:1046100033832283C9E1D2E02D818981821B8F3FC0
:1046200009F480E087FD8F5F85958887982F990F23
:10463000920F9D838D29B3DAC0907606F7E0CF0EF6
:10464000E0914A01F0E0EE0FFF1FE55BFE4F808135
:104650009181805B934509F07BC080917608811140
:1046600077C02885222309F448C08E81332727FD8F
:104670003095A901480F511D87FD5A95CA010E9426
:1046800033168E8340E1E42E45E0F42E5FE0A52E44
:1046900055E0B52E6AEC862E65E0962EF7018081F6
:1046A0008530E1F440E061E0F40180810E949B1AD2
:1046B0008823A1F0F50170802885822F992787FD36
:1046C0009095870D911D77FC9A950E943316F50100
:1046D0008083781619F086EF0E943B70F2E0EF0EAF
:1046E000F11C22E0A20EB11C3FEF831A930A4EE1A7
:1046F000E41645E0F40691F61886E091D4048E2F76
:10470000807E31F1E295E695E770F0E0E430F10566
:1047100054F4EE0FFF1FEB5BF74F208131813C5FBC
:1047200060E078E00CC0EE0FFF1FE95FFA4F2081D8
:10473000332727FD309523583F4F6AEF70E047E05D
:10474000429FC001439F900D11240E94C78FC62E27
:1047500080912302C81619F08C2D0E94C3168091F7
:10476000660687FF3CC0809156018823C1F1809185
:1047700055018823B1F18091A50687FD03C08F5FA5
:104780008093A50682E00E94EC17982F9F7789F00E
:104790002091A506921728F51092A506D11021C0E8
:1047A000D82ED094DD1CDD24DD1C83E68D19D82E97
:1047B00018C083E00E94EC17982F9F7791F020910A
:1047C000A506921770F41092A506D1100AC0D82E33
:1047D000D094DD1CDD24DD1C54E6D50E02C0109201
:1047E000550181E080935601C0E1D5E08FE0E82ECD
:1047F00085E0F82E9AECA92E95E0B92EC880CC2041
:10480000C1F0F5018081811106C0F5E0CF1207C02B
:10481000F701808107C09BD88111F7CF0AC08C2D8A
:104820000E941318992787FD90950E943316F7016F
:1048300080832296F2E0EF0EF11C2FEFA21AB20A4B
:1048400035E0CE31D307D1F68091560290915702D0
:104850000097B1F060E00E9489150E94FB8D909155
:10486000A406992339F0811128C0109257021092A2
:10487000560223C0882309F181E08093A4061DC05D
:104880001092A406C0914901CC2331F01092490145
:1048900087E10E948887DC2E84E180933E01D092DC
:1048A0001802E0914A01F0E0EE0FFF1FE55BFE4FBA
:1048B0000190F081E02D8D2D09950E94F57AC0912F
:1048C000650085ED91E00E94BC85882311F084E1AC
:1048D00005C08091510F882321F081508093510FA2
:1048E00006C080916300869581708093500F8091FF
:1048F000500F80935402882309F4DBC3809166062D
:1049000085FDD7C3CF7EC09365008091780D8F71F0
:10491000823009F054C08091210190912201AC01B4
:10492000A4E0440F551FAA95E1F797FD0796BC0137
:10493000F3E075956795FA95E1F720914A063327DC
:1049400027FD30952A5F3F4F629FC001639F900D06
:10495000729F900D1124840F951F2091600626FDF3
:1049600005C0609100017091010102C060EF70E02C
:104970000E94C78F80913D01680F711D6F5F7F4F4F
:104980007595679560933D018091A306805F809344
:10499000A306811114C080914906681780F4623320
:1049A00070F06EE281E10E9492878091600683FF41
:1049B00006C082E390E090933B0180933A0110920D
:1049C00039018EE587B9369A3699FECF84B195B113
:1049D00090930101809300018091B10D833019F40F
:1049E000A8951092B10D2091120182B790911201F9
:1049F0002913F9CF90E0922B801B910B2091080195
:104A0000309109012817390720F490930901809308
:104A1000080180910501882309F4A1C20091A9062B
:104A20001091AA060F5F1F4F1093AA060093A906C4
:104A30008091D4048F7150E1B52EB81AF7E1FB15BF
:104A400008F478C0EB2CF12CE701CC0FDD1FCB5222
:104A5000DB4F4FE04B1528F4E701CC0FDD1FC75C9F
:104A6000DA4F8881C82EC294C69427E0C222D9802A
:104A700055E05C1550F09AEF9D1538F4ED2DF0E0FF
:104A8000EE0FFF1FE15EFC4FD0808F7109F450C024
:104A90000E94A71CA82E80910501F701E45CFD4F40
:104AA0007F0181FD43C08C2D857049F48081811187
:104AB00006C0AA2021F08D2D90E00E94A7168FEF4E
:104AC0008C0D823058F4F7018081813079F5A11086
:104AD0002DC0F2E0CF1226C0D39424C025E02C15BF
:104AE00048F4F7018081811121C0AA20F9F0898161
:104AF00071D61CC0F2E0FC15C8F4AA20B9F024E07D
:104B0000C21631F035E0C31631F066E970E005C039
:104B10006CE271E002C068E572E0C8010E94C78FD4
:104B2000892B21F48D2D90E00E94A716F701A08219
:104B3000B39484CF0EEA14E0B1E9AB2EB6E0BB2EFD
:104B4000CFEACC2EC1E0DC2EE12CF12CF8019280D2
:104B5000892D8F700E94F1128330E1F5F601C0813A
:104B6000D181209771F4F801C081C7FD06C0C095BE
:104B7000FAE0CF02E00111241BC0DD27C7FDD0956C
:104B800017C0D7FF14C0219699F4F701E155FB4FE8
:104B9000C081C7FD06C0CF5F2AE0C202E001112438
:104BA00006C0DD27C7FDD095C095D09501C02197DF
:104BB000892D807F61F0892D82958F7089300CF06E
:104BC0008F5F0E94A71C811102C0CFEFDFEFF601BB
:104BD000D183C083F501C081F80182818F708C3050
:104BE00081F480810E94A71C81110AC0F701E15560
:104BF000FB4F80810E94A71C882319F0C0E001C0F0
:104C0000C1E0F80182818F708D30A1F480810E9413
:104C1000A71C882361F0C1FD0DC0F701E155FB4FD2
:104C200080810E94A71C882321F0C3E003C0CD7FB0
:104C300001C0C2E0F501C1935F010D5F1F4FF3E0BA
:104C4000EF0EF11C22E0C20ED11C34E2E316F10497
:104C500009F07CCF77ECE72E71E0F72ECDE9D6E0B6
:104C6000A12CB12C66246394E2E05E2EF3E07F2E4B
:104C7000AAE04A2E8501085A1D4F68014DEEC41A5C
:104C80004CEFD40AF60180810E94F112833009F0C2
:104C90005AC0F701808091808114910489F4F80151
:104CA000EF5EFC4F808087FC07C0882D8095FAE07E
:104CB0008F024001112425C0992487FC909421C0C3
:104CC00097FE1CC02FEF821A920A81149104C9F436
:104CD000F801EE5EFC4F808087FC0AC081E0880D01
:104CE0003AE083024001112441E0841A910809C08E
:104CF000992487FC90948094909403C051E0851A85
:104D00009108F801EC5EFC4F80818823C9F097EF91
:104D1000980F933108F48F5F9BE1980F933110F453
:104D2000815002C08C3121F0843E19F487EF01C01C
:104D300089E00E94A71C811103C088248A94982CC2
:104D4000F70191828082F60180818C3091F4F80124
:104D5000EF5EFC4F80810E94A71C882311F06882BF
:104D600008C0F801EE5EFC4F80810E94A71C8111F3
:104D70001882F60180818D30D1F4F801EF5EFC4F8E
:104D800080810E94A71C882379F0888181FD0FC053
:104D9000F801EE5EFC4F80810E94A71C882311F071
:104DA000788205C0588203C088818D7F8883F60190
:104DB000908180EF890F823008F054C08091050106
:104DC00081FF03C088818D7F88839131E9F4F801E8
:104DD000EC5EFC4F808197EF980F933108F48F5F62
:104DE0009BE1980F933110F4815002C08C3129F06F
:104DF000843E29F0882341F003C089E001C087EF99
:104E00000E94A71C982E02C099249394F801EF5E8B
:104E1000FC4F80810E94A71C882359F0888181FD66
:104E20000BC0F6018081813109F045C1992021F044
:104E300042C188818D7F8883F701808191810097AD
:104E400089F0F6012081213121F4911002C081E026
:104E500090E00197009719F428812E7F2883F701AD
:104E600091838083F4E0AF0EB11C22E0E20EF11CCE
:104E7000219638E1A316B10409F0FCCE16DA10929F
:104E8000050180914505882309F469C08091460594
:104E90000E94A71C882309F462C08091A806882379
:104EA00019F081508093A8068091A806811157C0FF
:104EB00080914505813081F487E20E94221AEC013D
:104EC000609147056695669570E062307105D4F093
:104ED0000E94DB8FEB0116C081E00E94221A8058ED
:104EE00091099C012E5F3F4F2530310510F480E081
:104EF00090E02091470526952695289FE001299F5F
:104F0000D00D11242097C9F0D7FF09C0D195C195C4
:104F1000D1098091470580FD05C082E201C081E290
:104F20000E948887CB34D1058CF0CD37D10584F031
:104F3000CF3AD1057CF484E010C08091470580FD14
:104F40000BC081E20E94888784E107C088E005C029
:104F500086E003C082E001C080E08093A8068091D3
:104F60000301882309F4C3C08091260F882319F117
:104F70006091890E2AE83EE0F9014CED80E090E076
:104F80005E2F521B561738F45191850F911D5417FF
:104F9000B8F7452FF5CF65E070E00E94C78F70939A
:104FA000F70E6093F60E4C3D31F0842F90E0909315
:104FB000F30E8093F20E2091A7062F5E822F8F7042
:104FC00090E00C970CF0207F2093A7068091D404EA
:104FD0008F7150E1F52EF81AC8E5D2E0E12C422F8E
:104FE0004073D42E522F5F70C52E822F807FB82E33
:104FF0002077A22EEF1409F450C08E0103581D4FE4
:10500000F8018081982F907C9034B1F4D11014C0B5
:10501000880F880F859585950E94A71C882361F0CD
:105020008091690680FF05C0FE01E258FD4F808136
:1050300001C081E00E948887F8018081982F907CD0
:10504000903841F5880F880F859585958D31A4F0AE
:105050008D51813029F0823031F0A1101BC006C083
:10506000C11018C003C0F0E2BF1214C0FE01E25824
:10507000FD4F8081AFD30EC0D1100CC00E94A71C81
:10508000882341F0FE01E258FD4F8081805890E076
:105090000E94A716E3942296ADCF1092030180914F
:1050A0005501882321F181508093550120C080E073
:1050B0007FCAC06128CC7882F801EE5EFC4F208167
:1050C000332727FD309537FF05C088279927821B96
:1050D000930B07C02F5F3F4F429EC001439E900D30
:1050E0001124F70191838083A7CED12C55CADF917B
:1050F000CF911F910F91FF90EF90DF90CF90BF90D5
:10510000AF909F908F907F906F905F904F90089599
:10511000282F30E0883058F02850310949E0429F6C
:10512000C001439F900D11248A599B4F089545E07B
:10513000429FC001439F900D1124825C9B4F0895B4
:10514000813649F40E94BD7C81E00E94731685E699
:105150009FE50E94FC1C64E973E180E10C94A47754
:10516000CF93DF93D82F9091AF0DC92FC17090FFCF
:1051700003C06FEF72E102C06DEE72E188E10E9440
:10518000A477D13629F41092AF0D80E00E947316F7
:10519000C11109C04091B00E5091B10E24E060E3FE
:1051A00088E40E94CD798091F50881508093F508BC
:1051B000811103C081E00E948887DF91CF9108951B
:1051C000CF93DF93EB01E2E7F8E08F3B29F4909176
:1051D00072089150988316C08E3BA9F4908191502B
:1051E00098839381992371F09F719883238130E094
:1051F00095E0359527959A95E1F723702093F4076C
:10520000138201C010829281992321F091819F77AE
:105210009083128290819923A9F0813219F08E38FF
:1052200009F047C020911D08211108C091509883B2
:1052300010820E94BD7C87E10E94888710921D0821
:1052400080E037C09881843681F4292F30E04830DF
:1052500031F050E024173507FCF427E004C0273074
:105260003105D4F428E0920F17C0853629F4292F90
:1052700030E0483099F417C0803611F08E3261F476
:105280009F5F9083906891830E94BD7C109218026A
:105290001092F40790E080E098830BC0273031052E
:1052A000DCF327E004C028303105B4F328E0921B7A
:1052B000F3CFDF91CF9108951F93CF93DF93182FF2
:1052C000D62FC42F662329F06FE0842F0E94B21FCF
:1052D000C82F809169024C2F83FF02C0440FD06217
:1052E00050E02D2F612F80E60E94CD798C2FDF9129
:1052F000CF911F910895FF920F931F93CF93DF9348
:10530000182FF62E0AE08AE0189FE0011124CE58EB
:10531000DD4F2FE130E0211B3109029FA001039FE7
:10532000500D1124BE01CE010A960E943F90FF202D
:1053300049F0BE016A5071094AE050E0CE010E9476
:105340003F900DC0FE0111920A95E9F78091030983
:105350008883898384E68A838F8188608F83109312
:10536000050982E0DF91CF911F910F91FF900C947E
:105370003B70AF92BF92CF92DF92EF92FF920F936A
:105380001F93CF93DF93EC01C62ED42E88E06813D1
:105390000AC0FE013E964591549160E085E40E946A
:1053A000BA7708E001C007E010E07801EE0CFF1CBE
:1053B00038E0A32EB12CFE01659174918A2D0E94D4
:1053C000A477BC1448F4FE01EE0DFF1D45915491E5
:1053D0006A2D85E40E94BA77B394229688E0A80EDD
:1053E00087E0B812E8CF4FE360E083E40E94807862
:1053F000DD20F1F087E06D2D8D1540F4601B660F08
:10540000660F660F20E04BE385E406C0660F660F6B
:10541000660F20E042E480E0DF91CF911F910F9171
:10542000FF90EF90DF90CF90BF90AF900C94E0771B
:10543000DF91CF911F910F91FF90EF90DF90CF9070
:10544000BF90AF9008950F93443051F4909167024C
:105450009F70913029F442E456E10F910C947F77CC
:10546000022F242F47EA5AE10E946D770F91089589
:105470009C01220F331F280F391F9595879595950D
:105480008795280F391F95958795959587959595BB
:105490008795820F931F0895429643E7489F900196
:1054A000499F300D1124C901E6E095958795EA954D
:1054B000E1F70895CF92DF92EF92FF920F931F933F
:1054C000CF93DF937B018A01D090520895E09D1520
:1054D00008F46AC091E09D0D90935208EBE08E9F16
:1054E000E0011124C556DA4F88818823A1F081504C
:1054F0000E9448159C01442737FD4095542F688130
:105500006552623058F440E050E00E94B1149C01B2
:1055100040E050E003C020E030E0A901D092520802
:10552000DE80FD2DF870CF2ED3FC0AC089819A81D0
:10553000AA2797FDA095BA2F280F391F4A1F5B1F76
:10554000AB81B0E011960E94998F2C8130E02F5FE3
:105550003F4F442737FD4095542F0E941090CC2098
:1055600051F089819A81AA2797FDA095BA2F280F1B
:10557000391F4A1F5B1FD0FE07C0509540953095DC
:1055800021953F4F4F4F5F4FE114F10419F08D818A
:10559000F70180830115110529F08E8186958370AE
:1055A000F8018083C90102C080E090E0DF91CF91D3
:1055B0001F910F91FF90EF90DF90CF90089590E0B2
:1055C000FC01E152F84EE491E330A9F485972BE019
:1055D000289FF001299FF00D1124E556FA4FE08134
:1055E0008FEF8E0F8432B0F0E550F0E0E152F84ECC
:1055F000E491E33079F0EE2369F0E13021F4809119
:10560000270F811107C081E09091260F911103C0EF
:1056100080E0089581E00895E82FF0E0E358F54E2A
:10562000E491262F332727FD3095C90183589F4FDA
:10563000EC3009F446C084F4E6305CF4E430FCF469
:10564000E53F09F44FC00CF457C0EE5FE230A8F01C
:105650000895EA30F4F50895E43209F43EC044F4C4
:10566000EE300CF449C0E031C4F1E332C1F10895E9
:10567000E732ACF1E732E1F108952AE023C080344B
:1056800091059CF0880F991F80549109813C9105E8
:1056900064F0880F991F805C9109813C51E0950767
:1056A00024F0880F991F885E91402AE0AC01249F66
:1056B000C001259F900D11242091640225FF1CC07C
:1056C000D7CE24E6AC01249FC001259F900D112464
:1056D0000895C901815A9F4F089522E3F3CF880F9F
:1056E000991F0895F3E0880F991FFA95E1F708953F
:1056F0005AE06502C00111240895CF93DF93E82F8B
:10570000F0E0E358F54E8491803F19F480914D0FFD
:1057100054C0853FC9F486E20E94221AEC0180E25F
:105720000E94221AD595C7959C0135952795C29F51
:10573000C001C39F900DD29F900D112469E170E0CC
:105740000E94DB8FCB0143C0853F44F440E050E032
:1057500060E070E0815FDF91CF91ACCE8D3F54F47B
:10576000E82FEE0FFF0BED5DFA4F8081992787FD43
:1057700090952DC08F3F09F03CF48E3F7CF48D3F17
:1057800011F580913D0119C08430C9F08332D9F4FC
:1057900083E20E94221A880F991F19C0992787FD5A
:1057A000909502962FE0289FF001299FF00D11247B
:1057B000EC5AF74F838594850AC090E008C0DF91CA
:1057C000CF910C942D1ADF91CF910C94221ADF9176
:1057D000CF910895CF92DF92EF92FF921F93CF93D4
:1057E000DF9300D0CDB7DEB7D82E1A82198285DFBD
:1057F0007C018D2DE4DE811105C08AE30E94C11673
:1058000011E001C010E0ED2DF0E0E358F54E849179
:10581000482F552747FD5095652F752FFA013F9664
:10582000E733F10508F078C0EB59FF4F0C942C904A
:10583000AE014F5F5F4FBE016E5F7F4F815F3ADE0B
:105840007C01EA81F0E0E55CF74EE491EA8364C014
:1058500084E28A8346C084E28A8382E089835CC0D2
:105860006CE370E0C7010E94DB8F6B017C0146E2B4
:1058700060E0C6010E949A8785E344C0E82FEE0FDE
:10588000FF0BED5DFA4FE080FF24E7FCF09444C08D
:10589000AE014F5F5F4F682F8E2D0E94B1147C01C7
:1058A00084E28A83809157018134F9F08130A1F537
:1058B0001A8232C088E38A8390916402892F8072B1
:1058C00093FF03C0882341F005C0882329F0C70156
:1058D000CFDD7C0188E18A8388EEE81683E0F80654
:1058E000ACF481E0BBCF81E0898383E30BC08FE21E
:1058F0008A838091640285FF0FC0C701CDDD7C01E2
:105900000BC08BE38A8308C081E08983C7016AE00A
:1059100070E00E94DB8F7B01111105C04A81698113
:10592000C7010E949A870F900F90DF91CF911F912E
:10593000FF90EF90DF90CF9008950F939FE0499FE5
:10594000F0011124EC5AF74F43855485022F0E9431
:105950000B7A0F9108957F928F929F92AF92BF9290
:10596000CF92DF92EF92FF920F931F93CF93DF932B
:1059700000D0CDB7DEB7F82EB62E6901102F80E229
:105980008A83E42FFF27E7FDF095E358F54EA490B6
:105990008E2D8170982EE0FE22C0AFE0AA0DA430BB
:1059A00008F001C18BE0A89FD0011124FD01EE5544
:1059B000FA4F8081882309F4F6C0AF0100E124E0AA
:1059C0008F2D0E94497712FD03C008E10F0D08C01A
:1059D0000CE10F0D88EFB80EECE08E2E03C00F2DFA
:1059E00076E0872E8E2D8870782EE3FC1F7B85E075
:1059F0008A15FCF084E0A8160CF08BC08DEFA81679
:105A000009F49DC08A1564F081EFA8160CF4A1C0BA
:105A100084EF8A157CF585EFA8129BC087E791C0BB
:105A20008FEF8A150CF041C081E08A150CF053C04D
:105A300090C083E2A81609F480C08A1574F08AE049
:105A4000A8160CF486C08BE08A150CF055C080E2D5
:105A5000A8127FC0106281E474C085E2A8160CF41D
:105A600078C086E28A150CF06AC087E2A81271C07D
:105A7000106269C0AE014F5F5F4FBE016E5F7F4F26
:105A80008FE08A0D17DD2981213011F4106203C0E7
:105A9000223009F41063EA81F0E0ED5CF74EE49106
:105AA000EA83E7FCC6016C0154C012FD02C08CEF12
:105AB00001C082E0800F9110865F1770012F212FA7
:105AC000A6016B2D83500E940B7AE3E3EA0DEA8373
:105AD0008AEFF80E47C0912F90684C2D772019F06F
:105AE0008DE38F0D02C0802F8819092F2A2D6B2D71
:105AF0000E94FB148A8336C083E48A838091640207
:105B000085FF27C0C601C8DC6C0186E48A830819BA
:105B100020C08DE68A838091640285FF07C083FDE3
:105B200003C0C601A5DC6C0186E68A8388EEC81630
:105B300083E0D80644F410620CC0106301C0106208
:105B400086E78A8306C0C6016AE070E00E94DB8FA8
:105B50006B01772071F18DE38F0D212FA6016B2D45
:105B60000E94CD798E2D867069F0E2FE04C08AE035
:105B70008F0D1B7F02C08091650D212F4A816B2DF7
:105B80000E9491768A810F900F90DF91CF911F91A3
:105B90000F91FF90EF90DF90CF90BF90AF909F90CC
:105BA0008F907F9008954F5F20E06B2D8F2D4BDC01
:105BB0000ACF802FD2CF0F931F93CF93DF93C82F9D
:105BC000D62F042F122F4CED57E10E947F7740E330
:105BD000400F212F6D2F8CE08C0FDF91CF911F9103
:105BE0000F910C949176EF920F931F93CF93DF93C5
:105BF000C42F122F2E2DDE2DD3709DE7940F9B3FC7
:105C000080F043E84C0F8251D6DFDD2359F122E0CA
:105C100042E850E06EE770E08C2F90E00E94D51EC5
:105C20000CC0552747FD50950E94CD79DD23D1F05A
:105C3000402F612F8C2F0E94AF1FC82F8091180218
:105C40008D3B81F48DE78C0F8B3F40F0EC2FF0E023
:105C5000EE0FFF1FED5EFB4FC08101C0CEE782E07B
:105C60000E943B708C2FDF91CF911F910F91EF908D
:105C70000895EF920F93E22E0DE723E8B4DF0F9122
:105C8000EF900895CF93DF939EE0899FE001112468
:105C9000CE5FDB4F8C850E94A71C882339F08D8551
:105CA0000E94A71C811104C081E003C080E001C0F4
:105CB00082E0DF91CF910895942F9695691B242F50
:105CC000891B0C94717A9091210281E0191624F0BD
:105CD000911101C080E08195109221020895BF9238
:105CE000CF92DF92EF92FF920F931F93CF93DF93A8
:105CF000B82EC62EEA01D22E102F07FD05C067EB85
:105D000079E18C2D0E94A47700E12D2DAE016C2D40
:105D10008B2D0E944977012F10E00F77012B79F12D
:105D20004D2D440F4D0D440F4E5F6FEF6C0D29E06C
:105D30008FEF8B0D0E94717A80911802803211F0E2
:105D40008E32E9F4D0927C08D0937E08C0937D080F
:105D5000F0928008E0927F0810921D080E94BD7C9E
:105D60001092180284EC9DE3DF91CF911F910F9167
:105D7000FF90EF90DF90CF90BF900C94FC1CDF91D0
:105D8000CF911F910F91FF90EF90DF90CF90BF9038
:105D9000089521E0AC0160E080E00C947F770F93E0
:105DA0001F93CF93C62F0E94CD79B8018C2FCF912E
:105DB0001F910F910C94A477EF92FF920F931F9372
:105DC000CF93DF93E82E142FFB01F490EB01229682
:105DD00031964491222381F080911508882321F087
:105DE00080911D08882351F02091160860E0812FD2
:105DF0000E94A51F182F02C000E002C000911708E2
:105E0000212FAE016E2D8F2D0E946D77812FDF9196
:105E1000CF911F910F91FF90EF900895982F862FAB
:105E2000242F492F62E275E1C7CF1F93CF93DF93F1
:105E3000D82FC62F122FBA018C2F0E94A477412F82
:105E40006C2F8D2FDF91CF911F91E8CFCF93C1E0C1
:105E50009C2F981B892FE9DFC81B8C2FCF910895A9
:105E6000982F862F242F492F68E376E1A5CF0F9333
:105E7000909167029F7021E0913009F020E000E0EE
:105E800042E35AE10E946D770F910895442321F077
:105E900050E08E5E0C94CD794CE953E00C947F7702
:105EA000EF92FF920F931F93CF93DF93EC01062F96
:105EB000F42E1091F407A0914708B0914808209162
:105EC000490830914A08EFE3F1E0868197818A1B07
:105ED0009B0B97FDCF9666E0959587956A95E1F7C0
:105EE000482F80931A0880859185821B930B97FD1C
:105EF000CF9656E0959587955A95E1F7982F809320
:105F00001808442311F0B783A683992311F0318731
:105F1000208780911908811104C08091600685FF57
:105F200006C010921A081092180810921908809151
:105F30001A08811108C080911808811104C082815B
:105F40009381892B11F00E949316E09008098FEF3E
:105F5000F81609F44DC08091530881112DC080912D
:105F6000FF08882319F01092FF081E2DACDE1816CA
:105F70006CF41E1510F41F5FC9F488818F1518F496
:105F80008F5F888301C0188210E010C0882371F0F1
:105F900011110BC08881882319F08150888301C0BA
:105FA000F88281E08093FF0801C011500E3271F435
:105FB00081E0809353080AC0813041F40E3221F011
:105FC00080911D08811102C0109253088091F3073F
:105FD000B1990BC08F3F19F08F5F8D3338F091E08E
:105FE00090931D089093530801C080E08093F307BD
:105FF000E092150880911D0881112CC0809118082D
:106000008823A1F04881481B47FD40E08F2D90E098
:10601000242F332727FD3095281739070CF04F2DF3
:106020004883E11608F41E2D1092180888818823F1
:1060300089F080911A08882369F0181B17FD10E079
:106040008E2D90E0212F332727FD30952817390713
:106050000CF01E2D003679F190F4023409F46BC077
:1060600028F40132E9F10E3231F184C0043409F42C
:1060700042C008F46EC0053409F44DC07BC005363B
:1060800009F44BC040F4033609F466C0B0F502369B
:1060900009F454C06FC00E3801F10F3B39F00138DC
:1060A00009F068C010921D0881E022C01882109289
:1060B0001D0810E05FC08FEFF81609F45BC081E0A7
:1060C00090911D08911180E080931D08882309F4A8
:1060D00051C081E0809353084DC08EE80E94BD7C82
:1060E00080911D08882319F010921D0843C080E09C
:1060F0000E9473163FC01E15E9F1EE20D9F1809180
:106100001D08811137C01E1510F41F5F01C010E07B
:10611000109218022FC0112369F1EE2059F18091DD
:106120001D08811127C0112319F0EE24EA94E10E15
:10613000109218021EC088818F15E1F080911D0811
:10614000811118C088818F1510F48F5F0DC01882DF
:106150000EC08881882371F080911D0881110AC0CA
:106160008881882319F08150888301C0F882E11664
:1061700008F41E2D20911D0821110AC031E08091E4
:10618000410190914201892B09F430E0832F01C035
:1061900081E080931C081093F407222311F082E021
:1061A00001C081E08093170810920809DF91CF9118
:1061B0001F910F91FF90EF9008954F925F926F9211
:1061C0007F928F929F92AF92BF92CF92DF92EF9287
:1061D000FF920F931F93CF93DF93C82F8CE598E125
:1061E000D8DD4AE06C2F89EF98E05ADE9090F908EC
:1061F0006090F407CE3211F0C03679F486E089154C
:1062000080F489EF890D809309098C2F0E94BD7C51
:1062100084E29CE50E94FC1C9FC0E6E0E91508F4BE
:106220009BC082E080930809AFE0CA2EA5E0DA2E79
:10623000CAECD5E018E05C2EB1E38B2E8C1A6CED25
:1062400077E1812F0E94A4777C2E4C2F480D612F7F
:106250008CE00E944777F6017F01A12C75189710FA
:106260000BC06A1009C0B0901708BB2031F08091B4
:106270001D08811104C001C0B12C00E001C001E083
:10628000A11013C02B2D4881612F8EE10E941114A3
:10629000002309F454C040915801642F61952AE00D
:1062A00088810E94BE1F88834AC0F1E0AF1233C0CC
:1062B000002339F06EE2F70181810E94B21FF701DD
:1062C0008183F70121812D3020F40B2D48EF58E117
:1062D00006C02D3148F42D5F0B2D4CE95BE1612F99
:1062E0008CE30E946D772BC0F3EE4F2E420E242DCF
:1062F00026950B2D43EA54E1612F82E40E946D77CD
:1063000040FE02C04DE201C04BE22B2D612F8CE319
:106310000E94917614C0002341F04DE763E8F70135
:1063200080810E94AF1FF7018083F70140815527CC
:1063300047FD50952B2D612F8CE60E94CD79A394BB
:10634000F3E0AF128CCF185F82E0C80ED11C21960B
:10635000103409F074CF41C0E9EF9E0E0BE915E04F
:1063600071E3E72EE8E0FE2E6AE974E18F2D0E94CA
:10637000A4774E2D6F2D8CE00E944777E80120E036
:1063800048816F2D88E10E94081349815A816F2D41
:106390008BE40E94FB794B8150E04F5F5F4F6F2D84
:1063A00080E60E94FB794C8150E04F5F5F4F6F2D7C
:1063B0008EE70E94FB79F8E0FF0EE394055F1F4F24
:1063C00088E2F812D1CF692D660F660F660F685FFD
:1063D00020E04EE780E00E94E077DF91CF911F91AF
:1063E0000F91FF90EF90DF90CF90BF90AF909F9074
:1063F0008F907F906F905F904F9008951F93CF93F1
:10640000DF93C82FD62F142F47E16BE255DC43E012
:106410006AE28C2F0E94807843E06BE28FEF8C0F52
:106420000E947E78812F69EF0E94BA8F382F375DE6
:106430008D2F67E00E94BA8F8C0F25E045E0632F17
:106440008250DF91CF911F910C94517ACF92DF92BD
:10645000EF92FF920F931F93CF93DF93CDE4D8E099
:10646000498168818AE2CADF4A816B8186E5C6DF9D
:10647000CFE3D8E028961AE3F12E0DE510E087E38C
:10648000C82E899199919C5FB8010E94DB8FDD2411
:10649000D394D60EEC2CE61A4D2D6E2D8F2D0E9426
:1064A00080784D2D6E2D81E08F0D0E9480784D2DCE
:1064B0006E2D82E08F0D0E94807885E0F80E89E4D1
:1064C000F812DFCFDF91CF911F910F91FF90EF90E6
:1064D000DF90CF90089543E256E168E388E60C949C
:1064E000BA770F931F93CF93DF93D82F162FC42F14
:1064F000022F47FF08C041E28AEF8D0F0E9491767C
:1065000086E08C1BC82F2C2F45E55BE1612F8D2F7A
:106510000E946D77DF91CF911F910F9108950F9396
:106520001F93CF93DF93162F042FC62FD0E0AE0119
:106530004F5F5F4F202F682F86E60E94CD790023A2
:1065400029F06FEFCE010E94B71F182F812FDF9126
:10655000CF911F910F9108950F93CF93DF93C42F85
:10656000D02FD27001FF03C00E94471402C00E94C6
:10657000111400FF42C0DD23B9F1CD3274F084ED77
:106580008C0F0E94F1132091580130E0280F311D2B
:1065900087FD3A952150310907C08C2F0E94F113D5
:1065A000282F332727FD309580915801482F440F1D
:1065B0004250C1E06C2F681B822F0E94AF1F909148
:1065C0005801482F552747FD5095292F30E0421795
:1065D00053073CF0C91B8C0F0E940114CCE2C80F7A
:1065E0000CC00E94011408C040915801642F6195AD
:1065F0002AE08C2F0E94BE1FC82F8C2FDF91CF91D5
:106600000F9108956F927F928F929F92AF92BF9257
:10661000CF92DF92EF92FF920F931F93CF93DF936E
:10662000C82F89E998E1B5DB43E16C2F8BEF98E047
:1066300037DCF090FB089090F407C23288F0C63245
:1066400030F0CF3B69F48091830E806407C0809165
:106650001D08882329F08091830E80638093830E28
:10666000109117088DE08F1508F48FC034DFE3E038
:10667000EF1508F416C164E176E188E00E94A47782
:1066800021E0F11020E04091640243FB442740F9EF
:1066900066E076E188E090DB9091640280FB93F9FC
:1066A0009093640221E0F21220E04091640245FBE5
:1066B000442740F96CEF75E180E17EDB9091640244
:1066C00080FB95F99093640281E080930809FEE0D5
:1066D000CF2EFFE0DF2EC5EFD4E0A2E0AA2EB8E176
:1066E000BB2E106863EF75E18B2D0E94A477EEEF4F
:1066F0008E2E8A0C4FE24A0D6B2D86E00E94477762
:1067000000E8282DF60140816B2D8EE70E94FB14D6
:10671000FA1004C0911002C0012F01C000E8282D1A
:106720004FEF6B2D88E40E94FB14FA100CC080918F
:106730001C08882351F0911008C088816FEF90E009
:106740000E94B71F888320E004C081E09812FBCF2D
:1067500022E04B8142954695469543706BEE75E17C
:106760008B2D2ADB8295880F880F807C9B819F73FD
:10677000982B9B83A394F8E0BF0E86E0C80ED11C33
:106780002496E8E2BE12AECF2CC16AE675E188E03D
:106790000E94A477FEE0FF1212C0C12FC062809158
:1067A000FD046FE082958F700E94B21F8295807FFA
:1067B0009091FD049F70982B9093FD0401C0C0E25E
:1067C0004091FD0442954F7050E02C2F68E086E622
:1067D0000E94CD79D0E1C0E05FE0C52EFC1411F03D
:1067E000D12C01C0D12EC1110CC021E0FC1020E041
:1067F000409145056AE575E18D2FDEDA8093450508
:1068000049C0C13069F401E0D11001C000E02D2D74
:10681000409146056D2F8AE59FDE809346053AC07C
:10682000C230E1F4DD2079F08091470562E386957E
:1068300086950E94B21F880F880F9091470593702C
:10684000982B90934705409147054695469550E013
:106850002D2D6D2F86E60E94CD791CC0C33079F4B2
:10686000809147052D2D4FE455E16D2F8170EEDAB3
:106870009091470580FB90F9909347050BC021E06C
:10688000FC1020E0409181056CE275E18D2F94DAD7
:1068900080938105C394CF5FD85FC53009F09ECF48
:1068A000A0C0E8E0EF1500F568EA75E188E00E9415
:1068B000A477C9E0D5E000E169E0D62EDC1A8C2F80
:1068C0008D0DF81207C06AE288810E94B21F88838A
:1068D000212F01C020E04991602F80E00E94232AEF
:1068E000085F003461F77DC09CE0A92E9FE0B92EBF
:1068F0002AE0C22E2FE0D22EE50134E0732E48E0CC
:10690000842E662463946092080960EE75E1882DF8
:106910000E94A4778C2F8A19813029F46DED75E1DE
:10692000882D0E94A477F71002C0992011F020E072
:1069300001C022E0F60140816DEC75E1882D3CDA62
:10694000F60181936F01F71003C0F1E09F1611F07B
:1069500000E001C0012F288130E040E050E073E00A
:10696000E72E682D86E60E94C278F7100CC0809151
:106970001C08882341F081E0981205C068E78881EF
:106980000E94B21F88837394E8E08E0E2196F6E091
:106990007F12B9CFFF120AC04FE761E08091000576
:1069A0000E94AF1F8093000521E001C020E04091CC
:1069B000000550E002EC15E168E186E6F0D921E03F
:1069C00087E0F81220E08091640247EB55E160E235
:1069D000829581702ADA9091640280FB94F99093F9
:1069E0006402DF91CF911F910F91FF90EF90DF90A4
:1069F000CF90BF90AF909F908F907F906F900895B1
:106A0000FF920F931F93CF93DF93182FF62EEA0177
:106A1000022F4981453249F4298522952695277010
:106A200040E757E10E946D7711C020610E94081372
:106A300089818551803150F48F8186FF07C0202FD6
:106A40004DE854E16F2D812F0E947F77DF91CF9128
:106A50001F910F91FF9008958091A803882329F03A
:106A600080EA98E20E94FC1C81E00895CF93DF93B6
:106A7000C82F88E00E94A4776DE773E188E20E9446
:106A8000A477C13671F028F4CE3269F0C03659F0DF
:106A900012C0CE3831F0CF3B71F480E00E9488877D
:106AA0000AC0D2E001C0D1E08C2F0E94BD7C81E001
:106AB0000E94731601C0D0E08D2FDF91CF91089511
:106AC000CF939091F1079F3F19F46CE673E102C0F8
:106AD00060E673E1CBDF813019F0823019F127C015
:106AE000C091F107CF3F19F40E94297E1BC08C2F63
:106AF0000E94F7122FE130E02C1B3109CAE0C29F3F
:106B0000A001C39F500D1124BC01665F7F4F0E94FE
:106B10003F90E8EAF3E0DF011D92CA95E9F782E0D1
:106B20000E943B7085E69FE5CF910C94FC1CCF91B1
:106B300008950F93CF93C82F4FE06AE778E08091D4
:106B4000EE070E94806F00E12AE04AE758E060E12A
:106B500081E00E9449774FE360E182E40E94477739
:106B60008091EF07882319F067E273E102C06AE1C0
:106B700073E18C2F7BDF813019F08230F9F024C073
:106B80008091EF078823A9F088E093E10E94B71570
:106B90008091EE070E94C86F882339F087E10E9438
:106BA000888782E08093EF0709C080E00E94888791
:106BB00005C08091EE078F5F0E94EC738CE796E32F
:106BC000CF910F910C94FC1CCF910F910895DF92FF
:106BD000EF92FF920F931F93CF93DF93EC01062F59
:106BE000D42EF62E18E0E12CFF20B9F0F0FE0EC0F6
:106BF0002D2D41E553E1612F82E10E947A77AE01AC
:106C0000612F88E10E94BA77E394185FF694FE0141
:106C1000849121968111FBCFE7CFCD2DCC0FCD0DE7
:106C2000CC0F2AEF210F4C2F67E082E10E94717A8E
:106C300044EF4C0F60917708660F660F660F685F30
:106C400020E088E10E94E0773ED8282FC6E7D8E010
:106C500099818B81882351F03091780D36FF08C0DF
:106C600081508B83811104C018821CC08FEF8B83ED
:106C700080911802813681F028F4803249F08E32FA
:106C800039F012C08336C9F088F08E3829F00CC074
:106C900018821B8281E01AC00E94BD7C10921802EB
:106CA00018821B8282E012C012162CF4EA949E1500
:106CB00030F49F5F04C0222339F0911191508B81F1
:106CC000882311F08FEF8B83998380E09091770870
:106CD0009F5F20E000FF02C0915021F006952F5FDA
:106CE0002830C1F720937808DF91CF911F910F9141
:106CF000FF90EF90DF900895DF92EF92FF920F9355
:106D00001F93CF93DF93C82F8CE692E142D8F09087
:106D1000EF0880917608811105C04FE06C2F8FEE4F
:106D200098E0BED866E672E180E00E94A4770E94F7
:106D3000E572AC0160E086E60E94FB791091EF08F5
:106D40008091EF07823021F41092EE081092EF0745
:106D500080911E0891E0980F191728F4123068F0FE
:106D60008FEF810F0BC094E0980F911738F48CEFE0
:106D7000810F8B3018F08AE001C080E080931E08FC
:106D8000082FD0E1EE24E3941013E12CDD24D394FA
:106D9000D00E2E2D4D2D6D2F82E10E94FD79809118
:106DA0004706081305C04AE26D2F81E00E9447772D
:106DB0004FE06AE778E0802F0E94806FEE2031F08C
:106DC0008091EE08882311F001E101C000E12FE07D
:106DD0004AE758E06D2F88E10E944977D85FD034A8
:106DE00011F00D2DCFCF80917608882309F477C05C
:106DF0008091EF0890914706981302C0D9E501C031
:106E0000DEE70E94B16F811101C0D6E98091690669
:106E100082FFDF734AE06D2F84E197E1D8DE813095
:106E200009F09CC0D0917808D11105C083E492E6A6
:106E30000E94861693C09FEF9D0F923060F50091DF
:106E4000EF08009347068093AE0D8C2F0E94BD7C07
:106E50000E94377100934706802F0E9446718091EF
:106E6000050182608093050181E00E943B700E94D1
:106E700037710E94111D0E942C1D809162020E9498
:106E8000BD160E94068580917608823079F2D23054
:106E900009F055C0CBCFD53031F48C2F0E94BD7C8A
:106EA0001092EF0704C0D33049F48093EF0710939A
:106EB000EE0789E995E30E94FC1C50C0D63019F416
:106EC00080937E0804C0D73039F410927E08109366
:106ED00082088EED9AE3EFCF8093EE083FC0C6366E
:106EE00038F4C43688F4C036C1F0C13641F036C03B
:106EF000C13829F1CF3B39F1CE3681F50EC08091F2
:106F0000EE08882359F10FC0909147068091EF0851
:106F1000981709F48BCF82E00AC010921D08809167
:106F2000EE08882319F01092EE0818C081E08093D3
:106F300076088C2F0E94BD7C109277080FC081E0EC
:106F40000E9473160BC01092EE0810927608809182
:106F500047068093EF0881E00E948D708091EE08D3
:106F60008823F9F0CF2DDD27C7FDD095812F90E044
:106F7000C817D907B1F061E0610F81E08F0D0E9461
:106F8000CB7380914706181303C0F092470606C0E2
:106F900090E0C817D90729F41093470681E00E94B2
:106FA0003B70DF91CF911F910F91FF90EF90DF9099
:106FB0000895CF92DF92EF92FF92CF93DF93FC017F
:106FC000EB019C01DC010E947A8F9B01AC01DE0188
:106FD0000E948F8F272F382F492F5527DF010E94BE
:106FE0008F8F6B017C013CE0F694E794D794C794B3
:106FF0003A95D1F724E630E02C1B3D0B0E947A8FA6
:107000006E5C7F4F8F4F9F4F6C0D7D1D8E1D9F1DA2
:1070100024E630E040E050E00E94EE8FC901DF91AD
:10702000CF91FF90EF90DF90CF9008951F93CF9373
:10703000DF936115710519F1192F111F1127111F08
:1070400019F091958195910977FF0FC07195619520
:107050007109C0E0D4E09E01281B390BC901A9DFEA
:107060009E01281B390BC90101C0A3DF112329F0A0
:1070700022273327281B390B01C09C01C901DF914E
:10708000CF911F910895EF920F93CF93DF93382FF5
:10709000862F642F922F332319F02091170801C0F7
:1070A00020E0C09106094EE0C49FE0011124CE5FAC
:1070B000DB4F933629F4032F4C854EDA8C8726C09C
:1070C000923629F4032F4D8547DA8D871FC0E02FB4
:1070D000F0E0E90FF11DE90FF11DEE0FFF1FEE0DBE
:1070E000F11DEC0FFD1FEF01011107C0E22E04E6B8
:1070F0002CE948810E94F32D08C048814C59E22EAA
:1071000004E620E00E94F32D84568883DF91CF911E
:107110000F91EF90089590E0E92FF0E0E65CF54ED6
:10712000E491E81721F0EE2321F09F5FF5CF892F3E
:10713000089580E00895823430F4E82FF0E0E65CB2
:10714000F54E8491089580E20895DF92EF92FF92C8
:107150000F931F93CF93DF93F82E162FEA01E22EA1
:10716000D02E67EB79E1812F0E94A47700E12E2DCC
:10717000AE01612F82E40E944977DD2099F18F2DC5
:10718000880F8F0D880F20911D0846E0612F8E5BC0
:107190000E94E0774E2D440F4E0D440F4C5F6FEF71
:1071A000610F29E080E40E94717A80911D08882394
:1071B000C9F0CF0DD11D88818111ADDF2D2D41E4A6
:1071C00060E00E94A51FB7DF488150E0282F3327D9
:1071D00027FD30954217530729F0888380911608C0
:1071E0000E943B70DF91CF911F910F91FF90EF9024
:1071F000DF900895FF920F931F93CF93DF93C82FD3
:10720000D62FF42E122F622F842F0E94ED15FC0131
:10721000E53F81E0F80774F09BE09E0F9F1510F0AA
:107220009CE09E0F40E3490F202F6D2F8C2F0E9472
:10723000917607C0212F4DE458E16D2F8C2F0E94CD
:107240006D77DF91CF911F910F91FF9008957F92FD
:107250008F929F92AF92BF92CF92DF92EF92FF9266
:107260000F931F93CF93DF93182FC09109092AE042
:10727000C29FE0011124C35EDA4F85EE92E10E94C5
:10728000C92E43E0612F84EF98E00E94502F409177
:1072900009094F5C60E080E30E944777B090F408F2
:1072A00078E0C72ED12CE3E0AE2EBD1003C0909045
:1072B000170801C0912C82E0D81609F467C0E3E0FA
:1072C000DE1609F478C0F1E0DF1681F067EC72E1B8
:1072D0008C2D0E94A47701E0911001C000E0292DBF
:1072E00048856C2D80E338D9888780C09110A092A2
:1072F00008096CE3762E812C8091F407881511F033
:1073000000E001C0092D409109094F5F282D6C2D27
:10731000872D70DF992099F18091F40788112FC093
:1073200080911C08882359F18E01080D111D080D4C
:10733000111DF801E080F180FBE0EF1AFEEFFF0A7B
:1073400024EFE21621E0F20624F454EFE52EFF24A8
:10735000F39422E048EF51E064EF71E0C7010E942E
:10736000D51E8E159F0559F0843FE1E09E0711F46C
:1073700080E090E0855F9140F80191838083839461
:10738000F6E07F0E24E08212B7CF30C0992051F092
:1073900089856FE08F700E94B21F8F709985907FF2
:1073A000982B998749854F70292D206285E0489F49
:1073B000A001112417C0992061F089856FE08295A2
:1073C0008F700E94B21F8295807F99859F70982B45
:1073D0009987498542954F70292D2062E5E04E9F9F
:1073E000A00111246C2D86E60E94CD79D394F8E09B
:1073F000CF0E24E0D21259CFDF91CF911F910F9180
:10740000FF90EF90DF90CF90BF90AF909F908F90C4
:107410007F9008951F93CF93DF93C82FD62F142FFB
:1074200044EC52E10E94BA7740E3410F6D2F8CE0AB
:107430008C0FDF91CF911F910C944777BF92CF9221
:10744000DF92EF92FF920F931F93CF93DF93C82F9A
:1074500089E798E10E94C92E43E06C2F80EF98E005
:107460000E94502FB090F008C03611F0CE3649F48B
:10747000B09209098C2F0E94BD7C87E299E30E949B
:10748000FC1C65E772E180E10E94A477FDE1EF2E2C
:10749000F5E0FF2EA8E1DA2E10E0CC24C3941B11F6
:1074A000C12CE7018985882331F02C2D4AE26D2D0E
:1074B00089E70E9491761F5F412F6D2D86E0AADF3C
:1074C0002C2D48856D2D88E10E941114DCE3C0E06D
:1074D0000C2D2C2F412F6D2D8D2F8CDECF5FDA5F81
:1074E000C430B1F78AE0E80EF11C88E0D80E143001
:1074F000A1F60E94D81F682F660F660F660F615FA6
:1075000029E04AE180E0DF91CF911F910F91FF9038
:10751000EF90DF90CF90BF900C94717A1F93CF9330
:10752000DF93162FEC01112329F089910E94957D9C
:107530001150F9CFDF91CF911F910895CF93C82FAC
:107540000E949C7D8F3F21F08C13FACF81E001C017
:1075500080E0CF910895CF93C82F81E00E94957D60
:1075600080E00E94957D8C2FCF910C94957DEAE769
:10757000F8E01382128282E08093020984E40C9482
:10758000957D0F93209180083091810842E3429FBE
:10759000C001439F900D112461EE71E00E94C78FDE
:1075A000062F28E044E660E38EE00E947C7A0F918B
:1075B0000895AC0168E184E20C94BA779F92AF928F
:1075C000BF92CF92DF92EF92FF920F931F93CF93D0
:1075D000DF93B82ECAE7D8E08C81882319F08CEBB2
:1075E00092E102C084EB92E10E94C92EA89521E6A7
:1075F000B21659F08FEBB81217C00E94837D10921B
:10760000020919821092F3080FC08AE50E94957D45
:10761000809147060E94467189E08093020910928A
:107620001D0881E60E94BD7CC090F30840910209CC
:1076300050E04A30510508F084C1FA01E456FF4F8A
:107640000C942C908BE10E94957D8BE10E94957D9E
:1076500018821B8281E09FC08B81853030F48EE3DD
:107660006DDF8B818F5F8B836CC18C81882341F0B0
:107670001D8287E08093020982E40E94957D61C1AA
:1076800076DF5FC127E08C2D622F0E94AE8F829F34
:10769000202D112429838CEA92E18BDF1CE00AE083
:1076A0000E949C7D8F3F09F44CC12091F1083091DC
:1076B000F2082F5F3F4F3093F2082093F108833098
:1076C00009F469C08D3009F480E02A819881FE01B7
:1076D000129FE00DF11D1124E90FF11D8187811129
:1076E00016C09B818981981750F081E0820F8A83B0
:1076F000883028F088E50E94957D83E04CC08EE4B8
:107700000E94957D8B818F5F8B831882C9CF81E02A
:10771000890F8B3010F48883C3CF0883C1CF8A814F
:10772000982E883010F017E0912E4981480F415073
:107730006B2D83EF98E00E94502F8981C81A8C2D01
:10774000873008F09DCF7E0199E0E90EF11C00E042
:1077500010E0B8E0AB2EDD24C7FCD094091598F4F6
:1077600021E0C016D10609F020E02061A7016A2DB2
:107770008CE00E947F7728E0A20E0F5F1F4F8CE005
:10778000E80EF11CEBCF90E6B912DBC082E50E9457
:10779000957D1D8284E080930209D3C082EA92E144
:1077A00008DF8D81811120C01F821E8282E7C6DE24
:1077B000882309F44FC08DE0CEDE8C2D90E0298126
:1077C000821B91092CE0289FF001299FF00D1124C4
:1077D0003996EC0FFD1F82EC838783E084876DE090
:1077E000CF019CDE188264C08130A1F50E949C7D8F
:1077F0008F3F2FEF920771F1988121E0290F2883A5
:10780000FE01E90FF11D818788818F3078F38E8129
:107810009F8102EC13E0081B190B0D30110510F0CD
:107820000CE010E0A80166E878E0885A9D4F0E94BD
:1078300036908E819F81800F911F9F838E83823C23
:10784000934008F48AC085E08093020985E60E948F
:10785000957D188296DE75C08BE992E1AADE888557
:107860000E943F6F882309F46CC086E094CF82E9C0
:1078700092E15CC08BE892E19CDE8D8181111AC09F
:107880001F821E8282E65ADE882321F388850E94A9
:10789000B36F8DE060DE6AE088E592E03FDE8BE06A
:1078A0000E94957D82EC0E94957D83E00E94957DEB
:1078B00081E02FC0813049F483E640DE882351F215
:1078C00082E08D831F821E82C5CF8230D1F48E81EB
:1078D0009F81823C934028F083E00E94957D84E064
:1078E00018C08CE038DE8E819F816CE0885A9D4FF5
:1078F00015DE83E08D838E819F810C969F838E831E
:10790000A9CF833041F484E619DE882309F4A2CF9D
:1079100082E08D839FCF86E011DE882309F49ACF21
:1079200088E08093020996CF8FE792E142DE09C09A
:107930008AE704DE882329F00E948D7D80E00E9482
:107940007316DF91CF911F910F91FF90EF90DF9011
:10795000CF90BF90AF909F9008958EE678CF21E0B2
:10796000411101C020E0405D0C9491760E94EA1222
:107970002091EC083091ED08AC01421B530B9A01A9
:10798000283E334088F09093ED088093EC08809176
:1079900067028F70823041F48BE10E94A71C88231C
:1079A00019F087E00C94888708950F9300E020E099
:1079B0000E940B7A0F9108951F93CF93DF93182F96
:1079C00081E692E10E94C92E163628F4143630F46E
:1079D000113659F00FC01E3841F00CC08091EB08F1
:1079E00091E089278093EB0805C01092EB0880E0B6
:1079F0000E9473168091EB08882309F43FC0C6E00B
:107A0000D1E0103641F48FEF888319821B821A82ED
:107A100087E10E9488876BE272E188E00E94A47788
:107A20004981469550E068E086E60E94FB794881EE
:107A3000469550E060E186E60E94FB7949818881A5
:107A4000481B469550E068E186E60E94FB798A81F2
:107A50009B8129E1289FA001299F500D1124569553
:107A600047955695479520E360E286E60E94CD79DA
:107A700068E172E188E30E94A47729C0C4E5D8E0F8
:107A800061E072E180E00E94A4774091E9075091A3
:107A9000EA0768E08AE289DF4C815D8168E08EE474
:107AA00084DF4F81588560E18AE27FDF49855A850E
:107AB00084E0569547958A95E1F760E18EE475DF9D
:107AC0004091E7075091E80760E08EE46EDFDF91B8
:107AD000CF911F910895CF93DF93282F30E095E049
:107AE000899FE0011124C35FDD4F4C818FE0829FAD
:107AF000F001839FF00D1124EC5AF74F9881898192
:107B000095878687442311F090E080E093878487EF
:107B100010861782158214821286118611821082B5
:107B2000DF91CF910895EF92FF920F931F93CF9320
:107B3000DF93F62E022F11E0180FEA01EE24EA94EB
:107B4000E60E0023D1F0FE014491809101098823C3
:107B500029F08FE9840F8A3108F440526F2D812F6C
:107B60000E9447772AE04BE06E2D8DEF810F0E9437
:107B7000717A0150165F2196E4CFDF91CF911F916A
:107B80000F91FF90EF900895CF92DF92EF92FF92C6
:107B90000F931F93CF93DF93082FCAE7D8E06D812F
:107BA0007E816115710511F467EB79E180E00E9437
:107BB000A47745E0602F8AEE98E00E94502F2AE0DB
:107BC00049ED56E164E182E0AEDF2AE043EE56E1A2
:107BD0006DE185E0A8DF2AE04DEE56E166E288E03F
:107BE000A2DF2AE047EF56E16FE28BE09CDF6FEE09
:107BF00071E188E30E94A4771091EA080F3B11F429
:107C000018821983E12EFF24E7FCF094898190E02B
:107C10008E159F0531F0111103C088818093F40700
:107C200019831230B9F034F4112379F0113021F5B1
:107C300089E00DC01430D1F09CF01530E9F483E0F8
:107C40008093080927E2D22E18C08A818150809340
:107C5000080912C089E0809308095AE0D52E0DC0AA
:107C600089E08093080944E1D42E07C089E080931D
:107C700008093EE1D32E01C0D12CC090F407003298
:107C800019F00E3209F08AC0153009F059C0C11040
:107C900008C081E090910109911180E08093010971
:107CA00025C082E0C81222C068816623F9F06150C5
:107CB00068838A81262F30E090E0AC014150510961
:107CC000AB81BC81241735073CF4FD01E20FF31FA3
:107CD000818180836F5FEDCFA80FB91F119780E27C
:107CE0008C938091160883700E943B708091F407FA
:107CF000833041F54A81888190E0242F30E0215083
:107D00003109821793076CF08881AB81BC81A80F81
:107D1000B11D80E28C938091160883700E943B70A5
:107D200011C08FEF840F9881981770F7AB81BC81D9
:107D3000A80FB11DFD01319790819C938150F3CF25
:107D4000111664F5DC0CED2DF0E0E752F94EE491EC
:107D500080910109882329F08FE98E0F8A3108F478
:107D6000E052153021F48091F4078130B9F4888114
:107D7000AB81BC81A80FB11DEC934881842F90E0AA
:107D80002A8130E0215031098217930714F44F5FA4
:107D900048838091160883700E943B70003851F42C
:107DA00081E090910109911180E08093010980E8C0
:107DB0000E94BD7C111103C08091F40788834B8120
:107DC0005C8100E12A8168E081E00E94497711111D
:107DD00004C08091780D86FF28C09881892F880F74
:107DE000890F29E047E067E0880F0E94717A111639
:107DF000E4F48091F4078A3018F089E08093F40766
:107E00009091F407292F220F822F880F880F820F5D
:107E10001230B1F48C5F49E0612F98E0E99E600D6B
:107E20001124655F20E00E94E07710921D08DF9129
:107E3000CF911F910F91FF90EF90DF90CF90089519
:107E4000133011F4895FE7CF143011F4865FE3CF6C
:107E5000153011F08F5FDFCF943018F083E08093FE
:107E6000F4078091F407882349F0813051F098E1BC
:107E7000899F802D1124845F42E1CECF42E180E0D2
:107E8000CBCF4EE188E1C8CF1092EA071092E90704
:107E900080E021CE81E01FCE5F926F927F928F9221
:107EA0009F92AF92BF92CF92DF92EF92FF920F9389
:107EB0001F93CF93DF9307EE17E0F8018F018681C0
:107EC0008F5F868394E5A92E98E0B92E21E1E22EFA
:107ED00022E0F22E812C55245394E501811003C039
:107EE0008091C70502C08091C805882309F48FC11D
:107EF0008D324CF08C520E94A71C9E81891709F488
:107F000086C18E8302C00E94A71C882309F47FC10A
:107F1000811002C0B9DF01C0BDDF66246394F701A0
:107F200032979080F701319770808EEF890D823003
:107F300028F4C0904308D090440802C0C12CD12C32
:107F400080915108882319F0C12C8CEFD82EF3E0D2
:107F5000F91548F4E92DF0E0EE0FFF1FE351F84F5B
:107F6000C080D18002C0992059F12CE2271504F578
:107F7000F8018481958128813981822B932B2B8173
:107F8000822B2681822B2A81822B892B09F41A824B
:107F900084ED870D0E94A71C882341F09A819111DE
:107FA00005C091E02B81211190E09B838A8308C05A
:107FB000772029F0872D0E94A71C8B8301C05B824C
:107FC0008B81882379F061100DC0FCEFDF1AD7FE9A
:107FD00003C02FE3C20ED11CA6E0D594C794AA9586
:107FE000E1F701C0C12C888199818C0D911D998385
:107FF00088830E94EA12F801C480D5808C199D09FB
:108000008436910508F46AC0668170E088819981A0
:108010000E94DB8F462F99838883F80181100DC061
:10802000208131812F5F3F4F318320832281338133
:108030002F5F3F4F3383228307C01682F4E6CF0EB3
:10804000D11CF801D582C482442331F02F813885B8
:108050002F5F3F4F38872F83611009C02B81222368
:1080600031F02C813D812F5F3F4F3D832C8377275B
:108070007595679589859A85680F791F7A876987CD
:10808000F7013497808191819C878B879920E1F05B
:10809000F1E09F1209C0711004C0F8016281738180
:1080A0000EC06C817D810BC0F2E09F1203C06F8116
:1080B000788505C0E4E076956795EA95E1F79C013F
:1080C000261B370B3C872B87F7012081222331F0B9
:1080D0002B853C85821B930B9C878B878394FFE0C9
:1080E000AF0EB11C25E0E20EF11C32E08312F5CE9A
:1080F00004E518E0F8018F01F090110280910D0263
:1081000090910E02C385D485258536852C173D07B1
:1081100009F47FC0D687C5872381222309F479C05B
:10812000FF2021F09C012C1B3D0BE90120916006F2
:1081300022FF2DC0892B59F1CE31D10519F469E206
:1081400089E10BC0C431D10519F46AE28AE105C0A6
:10815000CA30D10529F46BE28BE10E9492870AC0F4
:10816000C630D1052CF4D7FD05C06C2F8CE1F5CFBE
:1081700080E001C081E09091600693FF08C08823F1
:1081800031F082E390E090933B0180933A01D7FF76
:1081900005C0FF2019F0F801C385D4856CE370E0B9
:1081A000CE010E94DB8FDC01CB014091600641FFD4
:1081B0001AC0AB2BC1F44091690641FF07C000977C
:1081C00041F046E260E00E949A8703C080E00E948E
:1081D00088878091600683FF06C082E390E09093D9
:1081E0003B0180933A01F801838594850A960A97AA
:1081F00080F48CE10E9488878091600683FF09C02B
:1082000082E390E090933B0180933A0102C0612C9D
:1082100086CEDF91CF911F910F91FF90EF90DF906D
:10822000CF90BF90AF909F908F907F906F905F9016
:1082300008950F9304E12AE048E552E0682F88E1B1
:108240000E9449770F9108950F931F93CF93DF9367
:10825000D82F162FC42F423049F480918C0682FF0C
:1082600012C08FE10E949C7C2BE10AC0463059F479
:1082700080918C0684FF07C085E20E949C7C21E2ED
:10828000280F00E006C081E08C0F0E94A71C082F79
:108290002C2F40EA53E0612F8D2F0E946D77DF91E4
:1082A000CF911F910F9108956F927F928F929F921D
:1082B000AF92BF92CF92DF92EF92FF920F931F93F4
:1082C000CF93DF9391E0909316089091D30190FFA4
:1082D00002C044E001C043E066EE78E00E94E0287E
:1082E000F82E40910A094150682F86EE98E00E94CE
:1082F000502FD090E608B09017080091720810E057
:108300000C30110508F02CC7F801EA55FF4F0C940A
:108310002C9086EC98E10E94C92E8091D30180FFB9
:1083200002C06BE001C06AE060930A0941E04D0DB4
:10833000675089E391E10E94B92912C781ED96E166
:108340000E94C92E86E080930A09DD2011F0C0E06A
:1083500001C0CB2D4091480650E000E311E12C2FE5
:1083600068E086E60E94CF2ECC2351F04DE26AE011
:10837000809148060E94AF1F809348060E94CF7AE2
:1083800064EE70E180E10E94A47781E0D8120DC014
:1083900040915801642F619529E080914B060E941D
:1083A000BE1F80934B062B2D01C020E040914B0651
:1083B00060E180E60E94111441E092E0D91240E0B1
:1083C0008091660668E186FB882780F90E940E2F5F
:1083D0009091660680FB96F990936606C0916206BE
:1083E000E3E0DE1207C068E78C2F0E94B21FC82F9F
:1083F0002B2D01C020E04C2F440F440F4C0F60E2A6
:1084000086E60E94462FCC2329F043E760E288E706
:108410000E944777C0936206C0916A06F4E0DF12BB
:1084200006C068E78C2F0E94B21FC82F01C0B12C74
:108430004C2F440F440F4C0F2B2D68E286E60E9410
:10844000462FCC2329F043E768E288E70E9447776C
:10845000C0936A0641E085E0D81240E08091600652
:1084600060E383FB882780F90E940E2F90916006BD
:1084700080FB93F98BC088E896E10E94C92E86E0C4
:1084800080930A096CEB70E188E00E94A477C091A8
:108490007606C95FD11008C0DB2DD06467E08C2F51
:1084A0000E94B21FC82F01C0D0E44C2F50E02D2FE6
:1084B00068E086E60E94CD79C750C093760621E039
:1084C000D21220E040915D0646954695469547704C
:1084D0006EE870E180E10E94DC2E8770880F880FC3
:1084E000880F90915D06977C982B90935D06409144
:1084F0006906443008F044E021E092E0D91220E01F
:1085000068E570E188E10E94DC2E843008F087E0A5
:1085100080936906E3E0DE120AC044E661E08091E0
:1085200067060E94AF1F8093670621E401C020E424
:108530004091670650E060E286E60E94CD79F4E063
:10854000DF1209C065E0809168060E94B21F809327
:10855000680621E401C020E44091680650E007E489
:1085600010E168E286E60E94CF2E21E085E0D81275
:1085700020E0809160064CEE58E160E386958170C2
:108580000E94152F9091600680FB91F990936006F0
:10859000E7C580EA96E10E94C92E8AE080930A0925
:1085A00095E09D1508F4C3C00E946B326BE070E14A
:1085B00088E00E94A47741E0D11040E080917A06E3
:1085C00068E081700E940E2F90917A0680FB90F9EE
:1085D00090937A06C0916006C17041E0D41240E0E9
:1085E00060E18C2F0E940E2F81709091600680FBBD
:1085F00090F9909360068C130E94111D41E0E2E017
:10860000DE1240E08091660668E185FB882780F9EC
:108610000E940E2F9091660680FB95F99093660656
:10862000F3E0DF12B12CE0916306F0E0E35EFB4F74
:10863000D491CCE6ED2FE370F0E0E25BF74E44918D
:108640002B2D60E28C2F0E949176D695D695C65040
:10865000C43581F7BB2039F067E1809163060E9441
:10866000B21F8093630614E2C0E0D0E02C2F4EE8E6
:1086700057E168E2812F0E94507620917B0630E01E
:108680000C2E02C0359527950A94E2F720FF06C00C
:1086900020E042E168E2812F0E94E0772196185E97
:1086A000143821F794E0D9120FC08091D30180FFD4
:1086B00066C56FE080917B060E94B21F80937B06A7
:1086C0008091780D86FF5BC580915E06E5E0DE1245
:1086D00013C090911D08992389F063E00E94B21F96
:1086E00090915E06891761F0909166069F7790934E
:1086F000660680935E0604C020E003C021E001C04E
:1087000022E041E3480F60E382E10E949176D4E2E7
:10871000C0E08C2F0E94DD1220E0482F60E38D2FF7
:108720000E940813CF5FD85EC43099F719C5F9E0ED
:10873000FD1528F489E08093E608F9E0DF2E77EF55
:10874000A72E7FE0B72EC0E0D0E016E0E0E89E2E36
:108750009D0CCC2E84E0C80ECC0C00E02AEF210F3B
:1087600043E853E06C2D8EE10E946D77D11202C078
:108770009092750801E0D11200E0AE014458594FC3
:10878000750124E06C2D82E40E946F2E1F5F2496F9
:1087900095E0A90EB11C1A30E1F6E2C489EA96E12F
:1087A0000E94C92E86E080930A0964ED7FE088E08C
:1087B0000E94A477D1100BC0CB2DC06448E768E2BB
:1087C000809149060E94AF1F8093490601C0C0E412
:1087D0002C2F4091490668E086E60E94DB79E1E0B3
:1087E000DE1209C04EE666EF80915F060E94AF1F61
:1087F00080935F0601C0B12C80915F06482F5527FA
:1088000047FD5095465F5F4F2B2D60E180E70E944A
:10881000CD7921E0F2E0DF1220E080915D0643ECAB
:108820005FE068E181700E94262F90915D0680FBD9
:1088300090F990935D0621E083E0D81220E08091CA
:108840005D0642E45CE160E2869581700E94262F1D
:1088500090915D0680FB91F990935D0621E094E094
:10886000D91220E080915D0644EB5FE068E282FB74
:10887000882780F90E94262F90915D0680FB92F94F
:1088800090935D0621E0E5E0DE1220E080915D0638
:1088900087FB882780F946EA5FE060E30E94262F85
:1088A00090915D0680FB97F990935D0659C489EB22
:1088B00096E10E94C92E86E080930A0980E88093A1
:1088C000750801E0D11000E06BE9E62E6FE0F62EAE
:1088D0002AE04BE656E068E080E40E946F2E21E03B
:1088E000D21220E0809160064DED58E160E182FBFC
:1088F000882780F90E94152F9091600680FB92F9DD
:108900009093600621E0F2E0DF1220E080916006A3
:108910004DE85FE068E1829581700E94262F90917A
:10892000600680FB94F99093600621E083E0D81202
:1089300020E08091660641E85FE060E28295817008
:108940000E94262F9091660680FB94F9909366060C
:1089500021E094E0D91220E08091600647E75FE0D3
:1089600068E285FB882780F90E94262F9091600697
:1089700080FB95F99093600621E0E5E0DE1220E0AF
:108980008091660687FB882780F94BE65FE060E30D
:108990000E94152F9091660680FB97F990936606CA
:1089A000DFC381EC96E10E94C92E6FE378E080E19D
:1089B0000BC186E69FE00E94C92E10E0C0E0C430E3
:1089C00018F0D8EFD10F01C0D12F80918C0601E0B3
:1089D0000C0F82FF04C0C23011F442E005C084FFD6
:1089E00007C0C63029F446E06D2F80E32DDC0FC0B0
:1089F00020E0402F6D2F8AE20E9411148FE08C0F2F
:108A00000E94EE7B482F6D2F84E40E94AF3CC02F64
:108A1000185F0930A1F664E47FE080E10E94A4774A
:108A2000D8E3C0E08C2F0E94EE7B482F6D2F80E2B0
:108A30000E94AF3CCF5FD850C630A1F74CE35FE057
:108A400068E184E50E94BA7716E0C0E2D0E02D2FFD
:108A50004EE857E16C2F84E50E945076812F0E94EA
:108A6000EE7B482F6C2F8CE60E94AF3C81E0810F9B
:108A70000E94EE7B482F6C2F88E70E94AF3CDF5F9F
:108A8000C85F1E5FD43019F780918C0686FF0DC039
:108A900067E37FE088E00E94A4778BE20E94A71C36
:108AA000482F68E088E70E94AF3C80918C0687FFE2
:108AB00057C362E37FE080E10E94A4778CE20E94CA
:108AC000A71C482F60E188E70E94AF3C49C38EE2B3
:108AD0009FE00E94C92E81E080930A0910925601FE
:108AE000D0E0C0E019E10B2D006241E46D2F88E178
:108AF0000E94477741E34C0F6D2F8EE10E9447772C
:108B00008C2F0E944018AC016D2F8AE20E94BC7726
:108B1000C43028F48C2F0E94DD12815003C0C7306E
:108B2000D9F08C2FE82FF0E0EE0FFF1FE15CF74F3C
:108B300020813181129FF001139FF00D1124F7FF66
:108B400002C0E150FF4F5F2F550F550B4F2F6D2F78
:108B50008AE50E94FB7905C0402F6D2F8AE50E94AF
:108B6000EF79CF5FD85FC83009F0BFCF6AE27FE00E
:108B700088E20E94A477409100015091010160E3D6
:108B800088E70E94FB7981E08093190880911D0895
:108B9000882309F4E5C24FE761E880914A060E9404
:108BA000AF1F80934A06DCC289EC96E10E94C92E71
:108BB00086E080930A098090F4078091630081FF2A
:108BC00006C063E27FE088E10E94A477C9C263E146
:108BD0007FE088E00E94A477C4E5D6E0C12C30E1B4
:108BE000A32E43E0742E992493949C0C20E0492DED
:108BF0006A2D80E00E940813E12CDC1004C0709202
:108C000008098E1419F020E010E002C01B2D22E0AC
:108C1000F2E0EF16D1F183E0E81609F44DC091E0DF
:108C2000E91689F04981429546954695437066E07C
:108C30007FE08A2D0E94DC2E8295880F880F807C31
:108C400099819F731FC00981000F000F059505953D
:108C50008DE00802F0011124F7FD3396AF01559520
:108C6000479555954795212F6A2D82E40E94CD792D
:108C700011FF3AC04FE161EE802F0E94AF1F8F734A
:108C80009981907C982B99832FC06880962D97703E
:108C9000692E20E1290F012F4CE95BE16A2D88E460
:108CA0000E946D7711FF20C063E0862D0E94B21FE5
:108CB00087709881987F16C0088105950595059560
:108CC000212F402F6A2D8AE50E94111411FF0CC03C
:108CD0004FE061EF802F0E94AF1F880F880F880F31
:108CE00098819770982B9883E394E4E0EE1285CFF7
:108CF000F8E0AF0E22969E1611F0C92C74CF84E0D6
:108D0000D8120BC0CB2DC06248E266EF809164069A
:108D10000E94AF1F8093640601C0C0E240916406C8
:108D2000552747FD5095465F5F4F0BEF1EE02C2FF8
:108D300060E38EE40E94CF2E04E211E0CCE4D6E0A2
:108D400090E3E92EF801419151918F0129913991D8
:108D5000421B530B440F551F20E268E38E2D0E94E7
:108D6000CD79F8E1EF0E80E9E812ECCF95E0D91269
:108D700015C0E0E6FE1214C010921D0888E0E4E27F
:108D8000F1E0ACE4B6E001900D928A95E1F781E064
:108D90000E943B7087E10E94888702C020E001C0EA
:108DA00021E047EF5EE068E380E00E947F77D8C172
:108DB00080EB96E10E94C92E8BE080930A09F3E0D4
:108DC000FD1508F46DC00E946B3221E0D11020E047
:108DD000809160064FEE5EE068E086FB882780F9B0
:108DE0000E94262F9091600680FB96F99093600672
:108DF000C0917A06C5FBCC27C0F921E0D21220E051
:108E00004FED5EE060E18C2F0E94152F90917A0665
:108E100080FB95F990937A06C81721F08091860E11
:108E20000E94BB8CC0917A06C695C17021E082E099
:108E3000D81220E040ED5EE068E18C2F0E94152FF3
:108E400090917A0680FB91F990937A06C81741F0C9
:108E5000882321F080E00E94BB8C02C00E94E4893C
:108E6000C0917A06C6FBCC27C0F921E093E0D91265
:108E700020E041EC5EE060E28C2F0E94152F909183
:108E80007A0680FB96F990937A06C81709F468C1B0
:108E9000882319F00E946A7D63C110929A0060C114
:108EA00066E77EE088E00E94A477C0E008E0F090EA
:108EB0008C06C23051F0C33069F040918D06C1304C
:108EC00079F442954F7010E10DC040918F064F70BC
:108ED00010E408C040918F0642954F7010E802C020
:108EE0004F7014E021E084E08C0FD81220E062E59E
:108EF0007EE0802F0E94DC2ED82F812F80958F213D
:108F0000D11103C080938C0603C0182B10938C06DC
:108F100080918C06F8120E946113C23051F0C33068
:108F200069F0C130A1F4D295D07F90918D069F70E9
:108F300012C0DF7090918F06907F05C0D295D07FD0
:108F400090918F069F709D2B90938F0607C0DF70C6
:108F500090918D06907F9D2B90938D06085FCF5F3B
:108F6000083209F0A4CFE8E0DE1611F040E001C0BD
:108F70004B2D8091900668E281700E940E2F909197
:108F8000900680FB90F990939006F9E0DF1611F0BF
:108F900040E001C04B2D8091900660E38695817082
:108FA0000E940E2F9091900680FB91F9909390066D
:108FB0008AE0D812B12C809190064B2D68E382FB99
:108FC000882780F90E940E2F9091900680FB92F9DD
:108FD00090939006C5C084E996E10E94C92E81E075
:108FE00080930A091092E608CAE7D8E010E0812FC2
:108FF0000E9440182E853F85821793070CF49C0130
:109000003F872E874C8D5D8D481759070CF4AC01B6
:109010005D8F4C8F143060F02E853F85240F351FF7
:1090200037FF02C02F5F3F4F35952795398328833F
:109030001F5F22961730D9F68091A40880931908F3
:1090400090E2F91621F0EFEBFE120EC00BC08F5F1D
:109050008093A408833041F487E10E94888781E0EF
:109060000E943B701092A4088091A408813089F07E
:1090700050F0823009F072C010925601E8E8F8E032
:10908000CBE1D6E01FC061E47EE088E10E94A477D6
:1090900065C0CAE7D8E0F12CB8E9AB2EBAE3BB2E25
:1090A00008E615ECBF86AE861D8F0C8F8F2D0E94B3
:1090B000401889939993F394F7E0FF12F3CF63E399
:1090C0007EE043C061917191848595859B01281B49
:1090D000390B37FF03C03195219531092333310511
:1090E0003CF1DF0150974D915C91598348839A017F
:1090F000261B370BB90137FF02C0615C7F4FA6E02A
:1091000075956795AA95E1F7261B370B3F872E8744
:10911000841B950B9C0197FF02C0215C3F4F46E0EA
:10912000359527954A95E1F7821B930B9D8F8C8F80
:10913000229688E0E639F80729F60E94016F90939D
:1091400046068093450661E27EE080E10E94A477B6
:1091500043E057E168E182E10E94BA770E9426323B
:10916000DF91CF911F910F91FF90EF90DF90CF9003
:10917000BF90AF909F908F907F906F90089529E05F
:109180004CE567E283E20E94717A9ECACF93DF9337
:10919000C82FD62F462F60E257D841E04D0F68E226
:1091A0008C2F52D842E04D0F60E38C2FDF91CF918E
:1091B0004BC80F93CF93C82F8091F504882371F08B
:1091C0006BEE71E18C2F0E94A47704E420E04091C3
:1091D0000E0F68EF6C0F82E10E94FB148091F9047E
:1091E000882379F047EE51E16C2F80E40E94BA7732
:1091F00068EF6C0F04E421E04091140F84E50E94B5
:10920000FB14CF910F9108951F93CF93DF93EC013F
:10921000862F11E0683008F410E00E948828FC01D5
:109220009E013C5F37FD0DC0211588E0380784F0B2
:10923000112319F048E050E002C044E050E0E40F90
:10924000F51F8081992787FD9095982F882723C047
:10925000832F112321F03327220F331F02C086955D
:109260003170482F50E0E40FF51F608140E052E07C
:10927000421B530B559547956403C001659F900DA4
:1092800011246181359527956203A001639F500DDC
:109290001124840F951F69E170E00E94DB8FCB01E0
:1092A000DF91CF911F910895BF92CF92DF92EF92FD
:1092B000FF920F931F93CF93DF93182F7B010E9490
:1092C000422EC82E812F0E947C1A811104C001E019
:1092D0001E141F040CF400E08EE0189FE00111241E
:1092E000CE5FDB4F84E0C89E60011124F601E00FE1
:1092F000F11DEC0FFD1FB080812F0E947C1A882386
:10930000A1F08B2D0E94791A682F772767FD709541
:10931000C7019C5F97FD0196959587950E94163829
:109320007C01EE0CFF1C00E00BC08B2D0E94791A13
:10933000682F772767FD7095C7010E9416387C015A
:10934000CC0DDD1DC00FD11D8A8144E660E08C5933
:109350000E94631A9701A82FBB27A7FDB0950E9412
:10936000748F24E630E040E050E00E941090E90164
:10937000812F0E947C1A8111D450CE01DF91CF91B0
:109380001F910F91FF90EF90DF90CF90BF900895C5
:10939000DF92EF92FF920F931F93CF93DF93D62E1E
:1093A00020EEF22EF80EC0E0DCEF0FE730E2E32E05
:1093B000D11005C060910709CE0126DF04C0BE01AF
:1093C0008091060971DF97FD4F969C0195E03595D8
:1093D00027959A95E1F7122F0F3709F4022F412FA5
:1093E000552747FD5095401B510907FD539557FFE1
:1093F00003C0519541955109423030F46E2D611BE7
:109400008F2D0E9432780CC001171CF09FEF940F33
:1094100001C090E06E2D611B691B8F2D0E9480782A
:10942000112321F060E28F2D0E943278F394A096F0
:10943000C03284E0D80711F0012FBACFDF91CF916D
:109440001F910F91FF90EF90DF900895DF92EF92C0
:10945000FF920F931F93CF93DF93D82E809107092C
:10946000EE24E394883008F4E12C0E948828EC0173
:1094700040E460E08CE50E948078F12C0CE91FEF5D
:109480002F2D30E0EE2019F049E050E002C045E019
:1094900050E0241735075CF5C90145E0880F991F96
:1094A0004A95E1F7EE2019F064E070E002C062E056
:1094B00070E00E94DB8FE62FDE01A20FB31F2C911C
:1094C00030E22302C0011124B8010E94DB8FDF10BB
:1094D00005C0625E25E045E08AE304C0615E23E0EA
:1094E00043E08BE38E0F0E94717AF394C9CF60E062
:1094F0008CE5DF91CF911F910F91FF90EF90DF905E
:1095000047CF5F926F927F928F929F92AF92BF925E
:10951000CF92DF92EF92FF920F931F93CF93DF933F
:10952000882EAA24A39480910709883008F4A12CDE
:1095300082E396E10E94C92EAA2011F049E001C001
:1095400045E0682D8EEF98E00E94502F8FEB881237
:1095500002C01092FD084091070950E04F5F5F4F35
:1095600021E060E08AE20E94CD79809107090E94A3
:109570008828EC01B090FE0860901708AA2019F026
:10958000F9E07F2E02C0E5E07E2E5C2E0C2F1D2F11
:1095900065E0E62EF12C70E1972ECB2CD12C802F9C
:1095A0008519B81611F020E001C0262DF80141916F
:1095B0008F01552747FD5095692D88E10E94CD798F
:1095C000AA20A1F0F9E0EF1689F0CE14DF0411F023
:1095D00020E001C0262DFE01EE0DFF1D4081552724
:1095E00047FD5095692D80E30E94CD7988E0980E63
:1095F000EFEFEE1AFE0AF8E39F12D1CFB71411F085
:1096000020E001C0262D4BE256E168E38CE00E9489
:109610007F77B7103AC080911D088823F1F18092BE
:1096200018021091FD0820E044E06CEF812F0E94A9
:10963000A51F082F8093FD08811779F1AA2011F04A
:1096400024E001C022E0122F119530E059E1F52EFF
:10965000E12FFF27E7FDF0952E173F0794F0EC0F61
:10966000FD1FE20FF31F1002A0011124F49EC001A0
:10967000F59E900D1124B9010E94DB8F60831F5F5E
:10968000E7CF82E00E943B7008C0CB0DD11D44E6BD
:109690006CE988810E94AF1F88838B2DDF91CF9169
:1096A0001F910F91FF90EF90DF90CF90BF90AF9000
:1096B0009F908F907F906F905F90C8CEEF92FF92B7
:1096C0000F931F93CF93DF93C62FD0E0FE01EE0FD1
:1096D000FF1FE65EF94F21813281821B930B9C01B3
:1096E000BC01882777FD8095982F0AE0660F771FC9
:1096F000881F991F0A95D1F7121613061CF4258DA1
:10970000368D02C0278530892436310514F424E6CD
:1097100030E0442737FD4095542F0E941090790186
:1097200021308CEF380744F0211584E038073CF0F5
:10973000E12CA4E0FA2E03C0E12CBCEFFB2E0E942A
:10974000FE12882379F080915E06082F017010E0E8
:1097500082E090E0801B910BC817D90719F4F194AF
:10976000E194F108C701DF91CF911F910F91FF9014
:10977000EF9008952F923F924F925F926F927F9257
:109780008F929F92AF92BF92CF92DF92EF92FF9211
:109790000F931F93CF93DF93CDB7DEB7A1970FB68B
:1097A000F894DEBF0FBECDBF8F879B876D8B8091F6
:1097B0005E06880F880F9E012F5F3F4F4901E12C05
:1097C000F12C1D8E1C8E1B8E212C682E712CA3015A
:1097D0004D585C4F3A0160726E8B5D8951705D87A8
:1097E0006D896270562E3E2C8E2D0E9440186E2D73
:1097F00065DF8C0173E07E1570F054E095958795D8
:109800005A95E1F7F701E35BF74F8083F301EE0D23
:10981000FF1D449001C04E2CC42CD12CC601880FD2
:10982000991F9A878987FC01E15CF74F11830083B8
:10983000C80117FD0F9634E0959587953A95E1F7A5
:10984000282F87FD219522307CF481E090E00C2CBC
:1098500001C0880F0A94EAF7211102C0982F03C0B3
:109860009091E4079823292A93E0931508F473C094
:10987000AD85A11158C08091640281FF54C056018A
:10988000AA0CBB1CF501EC5AF94F5F018181807C69
:1098900009F449C080818595859585950E94A71C0E
:1098A000882309F440C0809122028823E1F1D50188
:1098B000EC91E770F0E0DF01AA0FBB1FAC5DBE4F7B
:1098C000EE0FFF1FE45BF94F8D919C912081318158
:1098D000821B930B97FD0196AC0155954795F501B9
:1098E0002181322F330F330F359535953403C00165
:1098F000359F900D11246FE170E00E94DB8F660FA1
:10990000771F660F771F22952695269523702130A5
:1099100009F09DC6060F171FF2E04F1204C07C8F9E
:109920006B8F21E02D8F3E89332339F0F601EE0F46
:10993000FF1FE452F84F11830083B801842DB4DC7B
:109940008C01632D809103070E942D16880F991FAB
:10995000D4018D939C93BE89BB2339F0F601EE0FA1
:10996000FF1FEC53F84F118300835520E1F0E3E033
:10997000E315C8F0F2E04F16B1F0065F1F4F053156
:10998000110538F0F601EE0FFF1FEC53F84F11826E
:109990001082E1E0F0E0EC0FFD1F29853A85E20F2F
:1099A000F31F118210823FEFE31AF30A42E0840EA4
:1099B000911C57E0E516F10409F015CF809169027A
:1099C00080FF27C062E0809103070E942D16182FA8
:1099D0000E94FE12012F81110195202F332727FDB0
:1099E0003095432F532F23583F4F4F4F5F4FA0E0E9
:1099F000B4E08091C8079091C907A81BB90B0E94D9
:109A0000998F20E034E040E050E00E9410903E83C7
:109A10002D836E89662309F435C110916D021221E0
:109A20008091E4078095812319F088E10E9488875E
:109A30001093E40704EC17E0D8018D0180E094E076
:109A4000FD0197878687918B808B4091700244231C
:109A500009F458C0A281B381E680F7809D010E947D
:109A6000748F4B015C019701D7010E94748F860EA1
:109A7000971EA81EB91E842F0E94861A7C019C0185
:109A8000DC010E94748F681579058A059B05D0F565
:109A900080E1C82ED12C40E050E8E0E0F0E89A01E7
:109AA000DA010E947A8F86169706A806B90610F486
:109AB0004E275F27F695E79521E0C21AD108C11419
:109AC000D104E9F4F801228133814A01A12CB12C9F
:109AD000D7010E94748FA50194010E941090F80193
:109AE0003383228326813781D7010E94748FA50199
:109AF00094010E941090F8013783268303C04E2BF7
:109B00005F2BCDCF60916E02862F807E09F4BAC0A4
:109B100051100EC0F801228133818B819C81280F66
:109B2000391F868197814F815885840F951F04C006
:109B300080E090E020E030E040916F02442379F033
:109B40004150E42FF0E0EE0FFF1F443118F4E00F16
:109B5000F11F02C0E950F84F4081518102C040E03E
:109B600050E062FF03C031952195310963FF03C0C6
:109B700091958195910964FF03C0519541955109D3
:109B8000629566956770633009F463C0643009F4C8
:109B900069C0623059F1BC0197FF02C0695F7F4F15
:109BA000F3E075956795FA95E1F7DC01A61BB70B15
:109BB000BC0197FF02C061587F4F660F672F661F79
:109BC000770BA61BB70B97FF02C081509C4F892FC4
:109BD000990F990B85958595A81BB90B7A01E21A07
:109BE000F30A37FF2CC02F5F3F4F29C0B90137FF61
:109BF00002C0695F7F4FF3E075956795FA95E1F7CD
:109C0000D901A61BB70BB90137FF02C061587F4FBE
:109C1000660F672F661F770BA61BB70B37FF02C0B7
:109C200021503C4F232F330F330B25952595A21B35
:109C3000B30B7A01E81AF90A97FD01969C01359554
:109C40002795240F351FB9016A0F7B1F2A1B3B0B79
:109C500012C07A01E21AF30A240F351FB901680F06
:109C6000791F07C07A01E21AF30ABA01680F791F57
:109C70009A01281B390BF801F38AE28A758B648BF1
:109C8000378B268BFF85FB8B2B852C8B42EB53E090
:109C90005A8F498F1E861D86B2E72B2EB2E03B2ECF
:109CA0001F8A198A5D8559A3B101665F7F4F788B42
:109CB0006F87C12CD12C7601D1018C9190E0019756
:109CC000ED85FE858E179F0709F059C3EF85F8894A
:109CD000389780810E94791A8A8B7F89672F70E07C
:109CE0007A8769876C5F784F5B01FB01E056FF4F15
:109CF000908040E061E00F85188907501109D80174
:109D00008C910E949B1AF8019081992359F0EF855C
:109D1000F889399790819C50983020F490912202D4
:109D2000992399F0882391F0F10181858F7190E05A
:109D30000090030702C0959587950A94E2F7817019
:109D40009927F1E08F27817001C080E02F85388945
:109D50002950310938A32F8FD9011C91811131C0AD
:109D6000F501E056FF4F10821D32C9F4E985FA85EE
:109D7000EE0FFF1F29853A85E20FF31FEC5BF84FCA
:109D8000AFE8B2E0A70196010E948F8FBB2797FD35
:109D9000BA95A92F982F872F80839183A28388EF6C
:109DA000810F823008F0DEC2F10187818670843035
:109DB00009F4D8C280E0193009F0BCC000E01CEF03
:109DC000BDC081E0911080E0982E2FEF210F2C3044
:109DD000B0F4822F90E0DC01AA0FBB1FAC53B84F48
:109DE0000D911C91243008F091C0F101278126FFCC
:109DF0008DC0FC01EE0FFF1FE452F84F26C0243146
:109E0000C0F483EF810FE82FF0E0DF01AA0FBB1F42
:109E1000AC5DBE4F0D911C91843040F4EE0FFF1FDE
:109E2000E45BF94F80819181081B190B000F111F12
:109E30006DC0243280F4F1018781E22FF0E0EE0F53
:109E4000FF1F86FF05C0E353F84F008111815EC0FC
:109E5000E950F84FFACF243281F5F10191859295BE
:109E600096959770B1F08EE0890F823128F081E1EC
:109E7000890F853149F01CC08131D1F490918C0655
:109E800092FF16C01FE106C090918C0694FDE4C3BA
:109E90000FC014E0812F0E94307C811135C081E019
:109EA000810F0E94307C882361F100E010E02EC019
:109EB0000E94EE7B882341F124C02C3260F4E22F13
:109EC000F0E0EE0FFF1FEB53FB4F0081F8E00F02B5
:109ED000800111241BC02C3251F4C701B60124E6C5
:109EE00030E040E050E00E94109089010FC040E057
:109EF00050E060E070E082ED810F0E945A2A8C01F0
:109F000005C000E014E002C000E01CEFF101878111
:109F1000982F907391F082958370815021E030E00A
:109F200002C0220F331F8A95E2F7C9013989382B05
:109F3000398B03C000E010E001C081E0E985FA85BB
:109F4000EC55F84F8083F101878183FD0EC0EF85CA
:109F5000F88932978081882341F04DE763E80E94B9
:109F6000631A0E94861A080F191FF101F681FE8FED
:109F7000F11105C0F1018581882309F421C1809187
:109F8000690283FF03C0F4E1F88F02C024E6288F42
:109F900049855A85440F551FDA01AC5FB84F3C9193
:109FA000FD012181E985FA85E40FF51FEC5BF84F8F
:109FB00080819181A281AC016A2F772767FD70951E
:109FC0002A013B01BB2777FDBA95A72F962F852F36
:109FD000B801681B790BCB01AB01465F5F4F453180
:109FE000510550F0A32EB22EA114B10439F4F101A1
:109FF0002581211108C002C0A12CB12C911003C0F1
:10A000009C878B8737C0F101878186708430D9F4B3
:10A01000E081F0E0EE0FFF1FE35EF74FA081B1811A
:10A0200020E034E60E94898F2B013C01FA89FF234E
:10A0300051F02F2F332727FD3095432F532F0E94A8
:10A04000109029013A01BB2777FCBA95A72D962DD0
:10A05000852D9801281B390B3C872B87211531054D
:10A0600049F0F101858137FF82958F70F88DF89F57
:10A07000500111241A141B04B4F480913C0188236C
:10A0800031F021E0A21AB108A114B10449F033273C
:10A0900077FC3A95272D162D052D1C861B8603C0AF
:10A0A000AA24AA94BA2CE985FA85EE0FFF1FEC5F6B
:10A0B000F84FB182A0824B855C85452B09F473C0B3
:10A0C0004801AA2497FCA094BA2C5E8D552309F46C
:10A0D00066C080913C01882309F440C06A896623E8
:10A0E00079F0262F27FD219530E040E050E060E038
:10A0F00070E080E293E00E941090CA01B90104C0B0
:10A1000060E070E080E293E0F10126814B855C85A0
:10A110001416150644F090958095709561957F4FC3
:10A120008F4F9F4F22952F7030E02115310591F010
:10A13000A88DA29FA001A39F500D11249A0144272E
:10A1400037FD4095542F0E941090420E531E641EFE
:10A15000751E04C04424582C692C7A2CBB2777FC2C
:10A16000BA95A72D962D852DEB85FC851E161F060D
:10A1700034F488169906AA06BB0634F009C088157F
:10A180009905AA05BB0524F44424582C692C7A2C83
:10A19000332777FC3A95272D162D052D04C044242E
:10A1A000582C692C7A2CE985FA85EE0FFF1F29853A
:10A1B0003A85E20FF31FEC5BF84F408251826282D6
:10A1C000F1018781EF85F889369787FF26C0808166
:10A1D0000E94791AA82FBB27A7FDB0951A161B0657
:10A1E00044F417FF62C024E630E02A1B3B0BD90180
:10A1F00009C0109709F459C0101611060CF055C08B
:10A20000AC59BF4F98010E94748F24E630E040E0C3
:10A2100050E00E941090890148C060818BE1860F58
:10A22000873340F06058772767FD7095C8010E941A
:10A23000163834C0862F992787FD9095A92FB92FFE
:10A2400087309105F8F4FC01EE54FF4F0C942C90EC
:10A2500017FF2BC010C0101611066CF026C017FF98
:10A2600024C011950195110920C010161106C4F0E3
:10A2700002C017FD18C000E010E017C0101611064C
:10A280007CF011C067FF06C011950195110936E0F9
:10A29000361B632F6750C8010E9404498C0105C01A
:10A2A00000E014E002C000E01CEFF101478140FD36
:10A2B00012C0AF8DB8A18C919FEF980F943058F4D5
:10A2C000FE013196E80FF11DE80FF11D32978081F4
:10A2D0009181080F191F9801EA89AE2FBB27A7FDAE
:10A2E000B0950E94748F4B015C0143FF15C0EF8550
:10A2F000F88932978081882379F04DE763E80E94DE
:10A30000631A0E94861A24E630E0DC010E94898FDD
:10A31000860E971EA81EB91EF1018781869583704F
:10A32000813039F08230E1F0C80CD91CEA1CFB1CEA
:10A3300019C0C501B40124E630E040E050E00E94BD
:10A340001090CA01B901A70196010E949F8F20E0D9
:10A3500034E040E050E00E94109069017A0102C0B0
:10A3600075016401FAE02F0E311C2F892F5F2F8BAE
:10A370004F855889465F5F4F588B4F879DCC109211
:10A3800051088091B406882309F441C08F01000F61
:10A39000111F000F111FF801EC54F94F87849088AA
:10A3A000A188B288FE89FF2319F0812C912C5401D9
:10A3B000C701B60124E630E040E050E00E94109072
:10A3C000E0910307F0E0EE0FFF1FEC54F94FA58179
:10A3D000B6810E948F8F680D791D8A1D9B1DF80123
:10A3E000EC54F94F6787708B818B928B2D8926FFF8
:10A3F000F9C02091B7063091B80640E050E00E94C5
:10A400001090A4E6B0E00E948F8F6B017C010D8557
:10A410001E85000F111F015E174FC701B60124E60C
:10A4200030E040E050E00E941090D8012D933C9322
:10A43000698C7A8CF3013F018381948180900805B7
:10A44000912C881699063CF0919481949108881675
:10A4500099060CF44C01F30121818401FAE02F02EA
:10A46000000D111D1124D3012C91F4014AE02402A6
:10A47000E00DF11D11249F01285E334008511C4F4F
:10A48000033E54E0150714F002EE14E049012E31AA
:10A490006BEF360724F42EE1822E2BEF922E302F15
:10A4A000212F8017910714F4382F292FA32EB22EB5
:10A4B000A814B9040CF45401C114D104E104F1044A
:10A4C000A9F0F7FE04C0D501A819B90903C0D80145
:10A4D000AA19BB09A70196010E94998F20EA36E8C4
:10A4E00041E050E00E94109069017A01C5010E948C
:10A4F0004D1A5C01AC0CBD1CC8010E944D1A8A1596
:10A500009B050CF45C01C4010E944D1AA816B90603
:10A510000CF45C01F3018281882319F0B194A194B9
:10A52000B1089091D4049F7180E1891BF9A1F817BB
:10A5300008F052C00D851E85000F111F0B521B4FD6
:10A54000D8018D018C91982F9F7309F445C0982FE5
:10A55000907C903409F440C09038F1F1880F880F56
:10A56000859585950E94A71CF8019081907C903C70
:10A5700039F5882319F01092E7081BC09091C9059E
:10A58000209143083091440895FF06C02D5E3F4F4F
:10A590002732310520F00DC024313C4F54F4AD8DED
:10A5A000AA2309F45BC02B8D3C8D24313C4F0CF465
:10A5B00055C09091E708911101C081E08093510846
:10A5C000882351F0ED85FE85EE0FFF1FEA52FB4F09
:10A5D00080810E94861A5C01F894AB89BC89AD9297
:10A5E000BC927894ED85FE853196FE87ED872B89A8
:10A5F0003C892E5F3F4F3C8B2B8B498D5A8D4B5F97
:10A600005F4F5A8F498F709709F04CCB1091780D9E
:10A61000798970FF05C0111103C08EE10E948887FF
:10A62000898981FF07C0812F877F803419F48FE1EA
:10A630000E948887998992FF15C0812F877F803873
:10A6400011F0103979F480E20E9488870BC0223023
:10A6500009F062C98B0160C915E21CCC91E09093AE
:10A66000E708A7CFA1960FB6F894DEBF0FBECDBF07
:10A67000DF91CF911F910F91FF90EF90DF90CF90DE
:10A68000BF90AF909F908F907F906F905F904F9012
:10A690003F902F900895FF920F931F93CF93DF93D6
:10A6A0000E94D81F182F8093030763E68AE798E07B
:10A6B00061D861E68AE998E05DD8CAE7D8E0E4EBC2
:10A6C000F3E021813281499159918E8D9F8D481BF4
:10A6D000590B8081811103C0519541955109240F77
:10A6E000351F293E83E038073CF428318CEF3807CA
:10A6F0002CF428E13CEF02C028EE33E032832183C2
:10A70000359628E0CA39D207E1F600E0023071F44C
:10A710000F5F0430D9F786E00E943B7081E0DF9143
:10A72000CF911F910F91FF900C948887602F812FFC
:10A730000E942D16EC01F12C602F8F2D0E94ED153B
:10A74000853F21E092073CF4AC014C1B5D0B602F70
:10A750008F2D0E944116F39484E0F812EDCFD8CFEC
:10A76000AF92BF92CF92DF92EF92FF920F931F931F
:10A77000CF93DF93C0915C061C2F1F70C07710929F
:10A780005601909176089111D0C08038D1F1A8F48B
:10A79000843209F449C040F4823209F48AC008F0D6
:10A7A0007BC0803249F1C1C08E3231F1813609F46B
:10A7B000A1C0853209F0B9C053C0843861F158F4A2
:10A7C000823809F484C008F49DC08CED9CE30E949B
:10A7D000FC1C83E883C08E38A1F08F3B09F497C03E
:10A7E000853809F0A2C081E08093190884E591E4DE
:10A7F0000E94FC1C85E84DC0143009F096C091E021
:10A8000001C092E090937608109277080E94BD7C78
:10A81000109218028AC081E0809319088CE796E3B1
:10A820000E94FC1C84E835C01330A8F44091000954
:10A830004F5F242F332727FD3095123019F483E022
:10A8400090E002C081E090E0821793070CF440E0B2
:10A85000409300096AC0143009F067C080E113C05A
:10A86000133068F480910009815087FF05C01230D1
:10A8700011F483E001C081E08093000956C01430D8
:10A8800009F053C080EF8C0F8073846080935C0666
:10A8900035C00E94BD7C49C01F5F153008F010E034
:10A8A000812F8C2B80935C0681EA0E943B7083E1B0
:10A8B00026C0112311F0115001C014E0812F8C2B00
:10A8C00080935C0681EA0E943B7084E118C0C460FA
:10A8D000C0935C0687E10E94888782E8DF91CF9170
:10A8E0001F910F91FF90EF90DF90CF90BF90AF90AE
:10A8F0000C94BD7C1430C9F40E949F8C87E10E94A7
:10A90000888713C00E94443F0E944A3FF5CF81E0F0
:10A910000E94BD7C83E00E94BD7C82E00E94BD7CE1
:10A9200081E08093E9081092000980916C020E94F6
:10A93000A71CD82F882329F08091E908811101C034
:10A94000AADED093E908143009F4B2C090913D0119
:10A9500080914906981710F4C6E001C0C4E080E079
:10A960000E9419414C2F406860E185E20E94EF7916
:10A9700046E568E186E20E94477724E040E060E136
:10A980008FE50E949D2C20E040E068E183E30E9477
:10A9900061140E94D81F882379F0482F60E186E275
:10A9A0000E940A3A29E046E26FE085E20E94717A4D
:10A9B000D0E08FE1E82E3EC000E020916A0246ED33
:10A9C00051E160E186E20E946D778091690280FF2B
:10A9D000EFCF42ED51E160E188E30E94BA77E8CF22
:10A9E00055954795559547954423B9F1443E0CF448
:10A9F00044EE042F4D310CF00CE18FEF8D0F46E348
:10AA0000823008F040C064E08C2F0E948078D13002
:10AA100069F18091690280FF29C06E2D601B63502F
:10AA200027E047E08DEF8C0F0E94517ADF5FD43032
:10AA300009F46BC08D2F0E94DD12E82FF0E0E35384
:10AA4000FE4EC4916D2F809103070E942D16AC011C
:10AA500097FFC6CF4D5F5F4FC3CF1816190614F48A
:10AA600041E0C4CF492F440F440BC0CF43E06EE117
:10AA70008FEF8C0F0E94807843E06EE181E08C0FB5
:10AA80000E948078CACF6BE385EE8C0F0E947E789F
:10AA9000FF24FA94FC0E43E06AE38F2D0E947E7837
:10AAA00043E06CE38F2D0E947E78C00F6BE3B7CF3D
:10AAB00001E12AE048E552E060E080E00E94497749
:10AAC00090913D0180914906981710F442E001C031
:10AAD00040E060E084E50E94EF7920E040E060E043
:10AAE0008FE60E949D2CC03109F04CC188E10E9484
:10AAF000D94895EFC92E94E0D92E20E9E22E2EE018
:10AB0000F22EC0E0D0E012E1E8C0123008F099C2A5
:10AB100080910009823014F01092000925E544E28A
:10AB200061E28EE20E94437825E544E262E28EE231
:10AB30000E94437880910009C2E18C9F802D1124EE
:10AB40002AEA42E161E2825D0E9443788091000935
:10AB50008C9F802D11242AEA42E162E2825D0E94EC
:10AB6000437800E0B9E1FB2ECBE1EC2E80910009A7
:10AB7000E02F28E0829FE00D1124F0E0EE0FFF1F90
:10AB8000EB50F84FC081D181802F8370113031F1AB
:10AB90008E9D802D1124043010F468E201C060E322
:10ABA0009E01D7FF02C0215E3F4FE5E03595279516
:10ABB000EA95E1F7AE01421B530B9A01D7FF02C0A1
:10ABC000C158DF4FAE01440F452F441F550B420FB4
:10ABD000531F20E28F5D0E94CD794CC0043018F4E1
:10ABE00062E2B62E02C05EE5B52ED82EDD0CDD0C7D
:10ABF000D80E46E2A42EAD0C80916E0281FF03C0F8
:10AC000060E075E002C060E074E0AE01D7FF04C010
:10AC1000442755274C1B5D0BF49EF001F59EF00D6B
:10AC20001124CF019E5F0E94DB8FC62E59E156177B
:10AC300014F439E1C32E25E543E36A2D87EE8B0D2D
:10AC40000E94437845E064E26D0D8B2D0E94807870
:10AC50001C161D0614F4B39401C0BC1867E26D0DF8
:10AC60004C2D8B2D0E947E786D2D6B5D4C2D8B2D88
:10AC70000E947E780F5F083009F078CFFCC1FE019A
:10AC8000EE0FFF1FEE0FFF1FE850FB4F90819295D4
:10AC900096959695937086E0B82EB10E933011F587
:10ACA0008C2F825F0E94221AAC0160E28B2D0E94E1
:10ACB000FB7900E42C2FF701468560E282E1810FE9
:10ACC0000E94FB142196F4E0CF0ED11C22E0E20E8C
:10ACD000F11CC230D10579F012E5F601808188239C
:10ACE00089F3CDCF00E02C2FF701408160E28B2D5E
:10ACF0000E94FB14DECF8091260F882379F069EC47
:10AD000071E188E00E94A4778DE00E94221A082F4A
:10AD100026E046E669E089E10E947C7A6EE27AE10B
:10AD200080E30E94A47760E380E40E94372F409183
:10AD30001A0F50E024E468E280E10E94CD7940914E
:10AD4000200F50E024E468E280E50E94CD79C0E95C
:10AD5000DEE04C815D8168E388E10E94FB794A89ED
:10AD60005B8920E468E384E20E94CD794E815F81B3
:10AD700068E388E50E94FB794C895D8920E468E3FB
:10AD800084E651C0C03209F051C08091260F88235B
:10AD900089F18AE00E94221AA5E0EA2E04E49C01CF
:10ADA00049E060E180E00E94AB2C8BE00E94221A17
:10ADB000B3E0EB2E00E49C014AE068E384E50E94E6
:10ADC000AB2C64EC71E180E10E94A4778CE00E94DE
:10ADD000221A24E4AC0168E08EE40E94CD790E943E
:10ADE0002D1AC5E0EC2E04E49C0146E060E280E010
:10ADF0000E94AB2C80E30E94D9484091B00E509144
:10AE0000B10E0EE21AE120E468E382E10E94CF2E47
:10AE100068E380E30E94372F4091B20E5091B30E49
:10AE200020E468E382E40E94CD7925C1C03309F0B3
:10AE3000C9C08091260F811102C0C2E101C0C0E1EA
:10AE400062E871E180E10E94A4778AE10E94221AFF
:10AE50009C0140E050E06BEFE62E0C2F60E180E3B8
:10AE60000E94C2784EE260E180E30E9447778BE166
:10AE70000E94221A9C0140E050E07CEFE72E60E146
:10AE800088E40E94C27887E10E94221A9C0140E077
:10AE900050E0EBEFEE2E68E180E30E94C2784EE2D4
:10AEA00068E180E30E94477788E10E94221A9C01B2
:10AEB00040E050E0FCEFEF2E68E188E40E94C278A9
:10AEC0004091A80E5091A90E60E288E70E94FB799C
:10AED0004091CE0E5091CF0E68E188E70E94FB7939
:10AEE0000091AA0E1091AB0E8091640285FF12C0F2
:10AEF0006DE771E188E20E94A4778DE492E0A801F9
:10AF0000489F8001499F100D589F100D1124012F5B
:10AF1000112706952C2F2F7EA80168E288E70E9452
:10AF2000CD798091260F882309F4A5C085E00E9481
:10AF3000221AAC0160E280E30E94FB7986E00E9465
:10AF4000221A2091640225FF0DC02DE432E0FC019D
:10AF5000E29FC001E39F900DF29F900D1124892F75
:10AF600099278695AC0168E280E30E94FB79D09036
:10AF7000890EF6E0FD1510F496E0D92ECAE8DEE061
:10AF800010E000E3C02E84E2F82E1D1509F473C012
:10AF9000133021F4A8E3CA2EB4E2FB2E299130E04D
:10AFA000220F331F40E050E0F4E0EF2E00E36C2D61
:10AFB0008F2D0E94C2782AE2F20E153009F45BC090
:10AFC0001F5FE3CF40E368E08FE30E948078C9E031
:10AFD000D5E010E088818823B1F081500E947D2B5C
:10AFE0009C0148814150612F6E70660F660F660F9D
:10AFF000605F10FF02C080E401C080E07FE0E72EC8
:10B0000004E00E94AB2C1F5F2196163019F76EE208
:10B010007AE188E30E94A4770091B00E26E04BE22B
:10B0200069E384E10E947C7A68E38EE60E94372F10
:10B030000091B20E26E04BE269E381E40E947C7A43
:10B040001AC0123009F094C00E94263260910009A3
:10B05000C1E0C60F662329F0862F880F680F660FA0
:10B060006D5F8AE00E94C6486C2F660F6C0F660FFA
:10B0700084E60E94C64880917608882309F46DC052
:10B080004EE0813039F46FE08FE491E10E94E735C2
:10B0900025E006C06FE183EA98E10E94E73520E0F1
:10B0A00010927408813009F058C090917808920F7E
:10B0B00019F48CE796E308C0913049F4809319089D
:10B0C0001092530883E492E60E94FC1C46C0923022
:10B0D00061F480937408E0914A01F0E0EE0FFF1FE5
:10B0E000E35BFE4F80819181EFCF933019F484E5CB
:10B0F00091E4EACF943019F48CED9CE3E5CF9530E0
:10B1000061F48091B40E9091B50E9195819591095D
:10B110009093E6078093E50720C0963041F4809134
:10B12000F804807C803CC9F48EE09FE009C0973031
:10B1300051F48091FC04807C803C79F484E19FE0B0
:10B140000E94E6890AC0983041F41092AB0E10922A
:10B15000AA0E1092A90E1092A80EDF91CF911F9106
:10B160000F91FF90EF90DF90CF90BF90AF90089538
:10B1700024E041E068E289E30E949D2C20E840E061
:10B1800060E38FE00E94611476CFAF92BF92CF92BE
:10B19000DF92EF92FF920F931F93CF93DF936C0197
:10B1A000162FC4EBD6E00E94D81FF82E4091E80875
:10B1B0008417E1F1442361F0EFEFE40F8AE0E89FA8
:10B1C000F0011124EA5DFA4F808182958F7001C0F1
:10B1D00080E0FF2061F0EFEFEF0D9AE0E99FF001D2
:10B1E0001124EA5DFA4F90819F70891718F0882327
:10B1F000D9F001C0892F682F70E080E092E00E94B2
:10B20000DB8F7A83698381E090E09C01042E01C08A
:10B21000220F0A94EAF73881322B0F2C01C0880FD5
:10B220000A94EAF7382B3883F092E8081062E12E8E
:10B230008881882329F11C821B828E01B12CAA24CB
:10B24000A39488818A21A1F0BF1491F0B0920307E2
:10B250008B819C81F80125813681820F931F9C830D
:10B260008B836E2DC6010E94BA4BFE2DFF7DEF2E03
:10B27000AA0CB3940E5F1F4F85E0B812E2CF09C04D
:10B28000FE01EF0DF11DEF0DF11D80E094E69683B8
:10B290008583FE01EF0DF11DEF0DF11D8B819C816A
:10B2A00025813681820F931F9C838B83F092030745
:10B2B0006E2D6064C6010E94BA4B8881882309F410
:10B2C0003EC080913C018823D1F1FE01B0E0A1E0B5
:10B2D00080E094E62581368118814A2F412331F19F
:10B2E00000913C0169817A81069FA001079F500D62
:10B2F0001124BF1559F04217530718F4241B350BBE
:10B3000017C02A2F20952123288310C0BC01621B5F
:10B31000730B4617570718F4240F351F09C02A2F3F
:10B3200020952123288320E034E602C020E030E08D
:10B3300036832583AA0FBF5F3296B53059F6DF9169
:10B34000CF911F910F91FF90EF90DF90CF90BF9022
:10B35000AF9008950F939CEF940F9D3138F450E017
:10B36000425051098E5E0F910C94CD79413208F014
:10B370004D51022F242F41E259E10E946D770F9128
:10B380000895CF92DF92EF92FF920F931F93CF9386
:10B39000DF93C82E85E19EE00E94C92E40910909E5
:10B3A00050E04F5F5F4F60E08EE40E94FB79C091F8
:10B3B000090989E0C89FE0011124CF52DA4F8C813E
:10B3C000877011F04AE001C049E06C2D85EE98E0ED
:10B3D0000E94502F1091E50816301CF46CEE7DE0B1
:10B3E00002C067EC7DE088E00E94A477F090170827
:10B3F00016300CF0ADC00E946B32111107C06EE424
:10B4000088810E94B21F88832F2D01C020E04881CF
:10B4100068E080E60E94081388818823D9F0815073
:10B420000E9448156C0162EC7DE088E00E94A477E0
:10B430004881453250F0455252E0E52E00E0960139
:10B4400068E088E40E94AB2C05C0A60168E088E4AF
:10B450000E94FB79113039F466E089810E94B21FA5
:10B4600089830F2D01C000E02981253018F447E3BE
:10B4700059E103C0255042EB5DE060E18EE40E949B
:10B480006D77123081F484E680933E0122E040E043
:10B490005DE760E073E88D819E810E94D51E9E83EA
:10B4A0008D832F2D01C020E048818D819E81453202
:10B4B00050F0455232E8E32E022F9C0168E188E704
:10B4C0000E94AB2C05C0AC0168E188E70E94CD79F1
:10B4D000133059F440915801642F61952AE08A8114
:10B4E0000E94BE1F8A832F2D01C020E04A8160E2A6
:10B4F00080E60E941114143031F461E28B810E94C5
:10B50000B21F8B8301C0F12C2F2D4B8168E280E6A6
:10B5100021DF21E0153009F020E04C814695469569
:10B520004695437062E97DE080E30E94DC2E8370E3
:10B53000880F880F880F9C81977E982B9C83DF91C2
:10B54000CF911F910F91FF90EF90DF90CF900895D2
:10B5500021E0163009F020E04C8142954695437079
:10B560006CE77DE088E00E94DC2E83708295880F76
:10B57000807E9C819F79982B9C8321E0173009F075
:10B5800020E04C8147FB442740F960E77DE080E103
:10B590000E94DC2E4C8180FB47F94C83042F0770FE
:10B5A00021E0183009F020E0402F6AE57DE088E1D5
:10B5B0000E94DC2E87709C81987F982B9C8380173B
:10B5C00011F018861F828C81877009F466C06FE4C1
:10B5D0007DE080E20E94A4778C818770813009F041
:10B5E00041C0193069F422E04FEF51E060E070E0B3
:10B5F0008F8198850E94D51E98878F830F2D01C05B
:10B6000000E04F8158854C3FE1E05E077CF0202F41
:10B6100049ED57E160E28CE60E947F774F814B5CF9
:10B62000202F60E288E70E94917633C0453FF1E029
:10B630005F073CF0445F202F60E28CE60E94DB2D28
:10B6400028C0202F60E288E70E94CD79002309F10D
:10B6500080E8C81204C08F8198850E94A7161092B6
:10B660001D0817C08230A9F4193059F44FE060E08A
:10B670008F810E94AF1F482F50E058874F830F2DB6
:10B6800001C000E02F814CEB59E160E28AE50E94A5
:10B690006D772AE0D22E08E203C099E0D92E00E2AD
:10B6A00068E47DE0802F0E94A4774D2D50E0E12FCB
:10B6B000FF27E7FDF095E417F50781F4E0E8CE12E7
:10B6C0000EC089E0FE0111928A95E9F710921D08DB
:10B6D0001A3029F488E08093E50801C0F12C2F2D61
:10B6E0004EE35DE0602F88E4DF91CF911F910F91D1
:10B6F000FF90EF90DF90CF900C947F77CF93C62F81
:10B7000020E04EE1682F80E00E94E07780911802EF
:10B71000803831F4C093AF0D80EB98E20E94FC1C9E
:10B7200010921D08CF9108951F93CF93DF93D82FC8
:10B73000162F237021F0223021F4C1E803C0C0E8A5
:10B7400001C0CDE2612F8D2F0E9447774C2F612FD2
:10B7500086E08D0FDF91CF911F910C9447779091E8
:10B760001E08282F291B181644F4273014F0865081
:10B7700005C027FD03C0892F01C080E080931E080B
:10B780000895CF92DF92EF92FF920F931F93CF9382
:10B79000DF93C82F82E798E10E94C92E4FE06C2FFB
:10B7A0008CEF98E00E94502FF090FC088F2DD7DF8F
:10B7B000D82EC03621F0C43611F0CE3269F4F7FC31
:10B7C0000BC0F09207098C2F0E94BD7C10921802CA
:10B7D00081E89AE40E94FC1C68E0E62E0F2D1127F8
:10B7E00007FD1095CD2DD0E0CC24C3940C171D0778
:10B7F00009F0C12C2C2D48E256E16E2D80E00E940C
:10B800007F77AE014F5F5F4F88E08D1510F486E1C2
:10B8100001C081E12C2D6E2D0E94CD7988E0E80ECB
:10B82000D39480E4E812DECFF7FC05C0F09207095C
:10B8300084E60E94264ADF91CF911F910F91FF90DD
:10B84000EF90DF90CF9008959F92AF92BF92CF92EA
:10B85000DF92EF92FF920F931F93CF93DF9348E015
:10B86000682F8AEF98E00E94502F69ED77E180E021
:10B870000E94A477C091090941E34C0F60E08CE07D
:10B880000E944777C090FA088C2D69DF982E45E218
:10B890004C0FE2E0EE2E00E020E030E060E080E3DC
:10B8A0000E94AB2C40911E0863EE74E188E00E9478
:10B8B000A97718E0DD24C7FCD0948BE0C89FE00195
:10B8C0001124C556DA4F5E01E7E0AE0EB11C492DDA
:10B8D00050E0C416D50619F40091170801C000E025
:10B8E000892D90E08930910508F093C087549F4FCF
:10B8F000FC010C942C90202F4881612F82E40E943F
:10B900000813002309F485C06EE488810E94B21FE9
:10B9100088837FC077EDE72E74E1F72E24E0A50140
:10B92000612F80E40E946F2E74C049815A81202FBC
:10B93000612F8EE40E94CD79002309F46AC022E0D1
:10B9400040E05DE760E073E889819A810E94D51E3E
:10B950009A8389835EC0402F6B81812F0E948F3232
:10B960008B8357C0402F6C81812F0E948F328C8334
:10B9700050C0002329F067E08D810E94B21F8D83A3
:10B980002D8149E058E1612F88E40E946D7741C024
:10B99000002349F08E8161E081700E94B21F9E8178
:10B9A00080FB90F99E838E8180FF02C04DE201C032
:10B9B0004BE2202F612F88E40E9491762AC0002359
:10B9C00061F08E81869562E083700E94B21F837061
:10B9D000880F9E81997F982B9E834E814695437058
:10B9E00050E0202F612F84E50E94CD7912C021E024
:10B9F000C416D50609F020E04E8143FB442740F9E8
:10BA000069EC74E1812F0E94DC2E9E8180FB93F90A
:10BA10009E839394185F103409F059CFDF91CF9132
:10BA20001F910F91FF90EF90DF90CF90BF90AF905C
:10BA30009F900895DF92EF92FF920F931F93CF9301
:10BA4000DF93C82F80E994E10E94C92E48E06C2F53
:10BA500088EF98E00E94502F0091F808802F7FDE39
:10BA6000D82FC03861F480E80E94BD7C89E18093C2
:10BA70001B08802F0E94587E81E00E9488874D2FEE
:10BA8000B8E0FB2E112707FD1095493051F1C42F66
:10BA9000D0E0EE24E3940C171D0709F0E12CDD241F
:10BAA000D394D40E2E2D4D2D6F2D82E10E94FD7961
:10BAB00080911B08882311F020E001C02E2DFE018B
:10BAC000EE0FFF1FEA5EFC4D459154916F2D88E10A
:10BAD0000E947F7788E0F80E80E4F81611F04D2D73
:10BAE000D4CFDF91CF911F910F91FF90EF90DF9016
:10BAF00008956F927F928F929F92AF92BF92CF9252
:10BB0000DF92EF92FF920F931F93CF93DF93C82E94
:10BB1000809105090E94F712EC014FE06C2D87EF30
:10BB200098E00E94502F83E894E10E94C92E20E003
:10BB3000488160E08A5F0E944013A090F7088A2D38
:10BB40000EDED82E40911E086DEF73E188E00E9452
:10BB5000A97718E0F12EBB24B39404E0902E80E87E
:10BB6000882EAD1003C0E090170801C0E12C0D2D08
:10BB700010E00031110508F093C1F801EE53FF4FBA
:10BB80000C942C9019812E2DAE016F2D84E50E940E
:10BB90000035153231F419851295169517701B5D15
:10BBA00003C0163208F01A5FEE2009F479C147E3AA
:10BBB00061E0812F0E94AF1F853268F08C3210F057
:10BBC000865009C085528295880F807E99859F7125
:10BBD000982B998785E2898363C12E2D4A816F2D29
:10BBE00080E60E94392E8A835BC12E2D48856F2DF9
:10BBF00080E60E94392E888753C18F814E2D6F2D8C
:10BC000083FB882780F90E940E2F9F8180FB93F988
:10BC100005C199818F81953080F486FB882780F952
:10BC20004E2D6F2D9B2D981B892F0E940E2F9B2D23
:10BC3000981B8F8190FB86F91BC02E2D4EEE53E191
:10BC40006F2D86FB882780F90E94152F9F8180FB2E
:10BC500096F9E4C08F8181704E2D6F2D9B2D981B1E
:10BC6000892F0E940E2F9B2D981B8F8190FB80F9AE
:10BC70008F8316C18F8187FD08C08C81855E8633D6
:10BC800040F410E04CED53E107C011E042EE53E107
:10BC900003C012E048EE53E12E2D6F2D86E00E9486
:10BCA0007F77EE2009F4FCC062E0812F0E94B21F72
:10BCB000181709F4F5C0823011F48C8201C01C827F
:10BCC0009F8180FB97F9AAC08F8187FF09C004E696
:10BCD0002CE94C816F2D88E40E94F32D8C83E0C009
:10BCE0004C818BE1840F8733B8F010E8140F2E2DB0
:10BCF0002064412F552747FD50956F2D86E60E9401
:10BD0000CD79EE2031F044E66CE9812F0E94AF1F1F
:10BD1000182F10581C83C4C02E2D6F2D8CE00E944C
:10BD20007132EE2009F4BCC046E160EF8C810E94C4
:10BD3000AF1F8C8390E6C912B3C087303CF08750A8
:10BD40008093070981E89AE40E94FC1C8C8187FF9C
:10BD5000A7C080958093070981E89AE40E94FC1CA3
:10BD60009FC001E0E11001C000E02E2D4B816F2D3E
:10BD70008EE40E94AC328B8393C0E110909208094C
:10BD80000FE310E07724739466246A946F0C99850E
:10BD90009F71972121E009F020E040E3410F6F2DD2
:10BDA000802F0E949176EE20E9F08091F4078113B4
:10BDB00019C029E048E0662D8FEF800F0E94717A4C
:10BDC00080E2C81619F09EE2C9120CC08985972D31
:10BDD00098279F71807E892B898782E00E943B7023
:10BDE00010921D08770C1F5F095F153081F658C04F
:10BDF0001F81129513702E2D412F6F2D8EE40E94FE
:10BE0000462FEE2009F44CC063E0812F0E94B21F40
:10BE100083708295807F9F819F7C982B9F8340C0F9
:10BE200021E08BE0A81220E04F814695437060EC42
:10BE300073E18F2D0E94DC2E8370880F9F81997F84
:10BE4000ECCF4D8142954F706E2D8F2D0E945C2955
:10BE50008295807F9D819F7009C04D814F706E2DAE
:10BE60008F2D0E945C298F709D81907F982B9D83E0
:10BE700017C04E8142954F706E2D8F2D0E945C2908
:10BE80008295807F9E819F7009C04E814F706E2D7C
:10BE90008F2D0E945C298F709E81907F982B9E83AE
:10BEA000D39498E0F90E80E4F8125BCEDF91CF9145
:10BEB0001F910F91FF90EF90DF90CF90BF90AF90C8
:10BEC0009F908F907F906F9008952F923F924F9206
:10BED0005F926F927F928F929F92AF92BF92CF921A
:10BEE000DF92EF92FF920F931F93CF93DF93A82ED1
:10BEF0008BE493E10E94C92E8091F007882301F121
:10BF00000E94632E882331F01CF022E6A22E02C08C
:10BF100093E6A92E2091F608211103C083E6A81606
:10BF200061F030E08091F207992787FD90952817FE
:10BF3000390721F4E2E6AE1201C0A12CA09218024A
:10BF400080917608811107C04091F2076A2D86EF33
:10BF500098E00E94502F9090F60880911802803649
:10BF600041F08F3B19F08E32D1F403C01092F007EC
:10BF700016C09091F007992339F01092F0071092B3
:10BF80001D08109253080BC090917608911107C0BC
:10BF90000E94BD7C109218027724739401C0712C0A
:10BFA000892DDDDB582E80917608811110921802C0
:10BFB0008091F0078823E1F0809118029EE9980FA4
:10BFC0009230B0F401E0823609F000E010910509EA
:10BFD000812F0E94F712EC0111119CC10111A4C123
:10BFE0008881823010F08150888382E00E943B700B
:10BFF00066246394B12C812CC52CD12C882D0E94F1
:10C00000F712EC01B51488F06B2D70E06C197D0906
:10C010006730710554F46F5F7F4F660F660F660FD0
:10C0200020E0462D81E00E944013FFE1F81508F45E
:10C03000B8C028802610B5C02A96482C7E018AE018
:10C04000E81AF108B51408F49FC08B2D90E08C1904
:10C050009D09873091050CF088C00196382E330C6D
:10C06000330C330C8091F007811112C09B1010C06B
:10C070004092050920920309772031F01092770849
:10C08000E1E0E0937608A12C11E08091760881111F
:10C0900010E0841459F0F70127812695237000E001
:10C0A00046E453E1632D83E10E946D7720E0A70110
:10C0B000632D80E30E940035212F8E010850110965
:10C0C000F8014081632D8DE20E94392EF8018083B2
:10C0D000FE0137974081442329F020E0632D88E456
:10C0E0000E941114FE01369740814423B1F0F701FC
:10C0F000878187FF03C020E044E60BC08BE1840FFB
:10C1000020E0873328F4632D80E60E94713205C059
:10C1100045E4632D80E60E949176F70186818111C6
:10C1200002C040E201C043E5F7018581882329F080
:10C13000433511F44AE201C044E4632D89E70E94CB
:10C1400047778091F0078823F9F0809104098411E2
:10C150001BC020E046E6632D88E10E94E077409214
:10C160000509B092F6089B2C0FC0079769F48091DF
:10C17000F007882349F080910409841105C080915B
:10C18000F6088F5F8093F608B3944394F0E24F165D
:10C1900071F12A96FE013A978081821509F44ECFFB
:10C1A00026C09B1022C06092030980920509692D68
:10C1B0006C19660F660F660F695F29E049E180E040
:10C1C0000E94717A772089F00E942C3581110DC070
:10C1D00060E0809105090E947B291092F00789E7B1
:10C1E0009DE50E94FC1CB92C08C0B394482C6394B4
:10C1F00081E1681611F0842C01CFB51428F18B2D44
:10C2000090E0851991090797FCF467E373E188E3EF
:10C210000E94A477292D30E08091F207992787FDAD
:10C2200090952817390781F420E04EE768E380E015
:10C230000E94E077E0E6AE1619F0FEE2AF1204C00D
:10C240008AE19DE50E94FC1C80917608882309F410
:10C250004CC0A09218024BE06FE389E497E10E9482
:10C26000E735909178088130D1F5913079F40E94CA
:10C270002C3581110DC0809105098F5F80930509D0
:10C2800060E00E947B291092F00702C0923018F4FF
:10C2900089E79DE50EC0943079F48091050980937B
:10C2A000F107809118020E94BD7C1092180280E66E
:10C2B00095E30E94FC1C11C0953011F48FEFEFCF75
:10C2C000923041F4809105098F5F8093050961E008
:10C2D0000E947B2981E08093F0071092760880917C
:10C2E00005098093040910921D08B092F207DF91AE
:10C2F000CF911F910F91FF90EF90DF90CF90BF9063
:10C30000AF909F908F907F906F905F904F903F90F5
:10C310002F900895113208F06BCE103219F40023DB
:10C3200029F066CE002311F01F5F01C01150812F4C
:10C330000E94F712FC0198818FEF890F803108F07D
:10C3400057CE2081213108F053CE291302C08BE053
:10C3500009C0002309F448CE903108F046CE9F5F13
:10C36000988343CE815029F090812881219399931D
:10C37000F9CF1093040939CE9F92AF92BF92CF921A
:10C38000DF92EF92FF920F931F93CF93DF93D82FFB
:10C3900088E39DE00E94C92E47E06D2F84EE98E06F
:10C3A0000E94502FC091E4088C2FD9D9A82EDE32DC
:10C3B00011F0D03659F4C8304CF4C09309098D2FD0
:10C3C0000E94BD7C81EC99E50E94FC1C38E0B32EF4
:10C3D000CC2EDD24C7FCD09449E0942EEA2CF12C1D
:10C3E0009E9CE0019F9CD00D1124CF52DA4FA701F3
:10C3F0004F5F5F4F05E31DE020E06B2D81E10E9460
:10C40000CF2E20E048816B2D8EE10E94081320E0A2
:10C410004A816B2D86E30E94111420E04B816B2D25
:10C420008EE40E94AA599C819770913021F092303D
:10C4300039F441E401C043E26B2D82E70E94477763
:10C440008C81887129F048E46B2D88E70E9447773A
:10C45000CE14DF0431F420E048E76B2D80E00E9429
:10C46000E07788E0B80EA39480E4B812B7CFDF91EC
:10C47000CF911F910F91FF90EF90DF90CF90BF90E1
:10C48000AF909F9008953F924F925F926F927F92EC
:10C490008F929F92AF92BF92CF92DF92EF92FF92D4
:10C4A0000F931F93CF93DF9392E09093160848E089
:10C4B00063EE78E00E94E028C82E40910A094150BE
:10C4C000682F83EE98E00E94502F4091720850E050
:10C4D000FA013197EC30F105D0F4EE52FF4F0C9495
:10C4E0002C9085E69FE511C08EE19AE30EC08AE1AB
:10C4F0009DE50BC081EC9BE508C082E093E305C09D
:10C500008DED90E302C08CEB91E60E94FC1CD09074
:10C51000E308C09117080091720810E0003111057E
:10C5200010F00C94CD6EF801E252FF4F0C942C9059
:10C5300080EB98E10E94C92E8FE080930A0941E0C8
:10C540004D0D68E087E19DE00E94B9290C94CD6E05
:10C5500089EB96E10E94C92E2AE02D1510F00E9469
:10C560006B3280E180930A0985E08D1508F4E7C0FD
:10C5700080E88093750801E0D11000E05CE0E52ED2
:10C580005DE0F52E2AE048E552E068E080E40E9494
:10C590006F2E91E0D91210C0E0E6CE1204C0809157
:10C5A00062020E94BD1661E3809162020E94B21F86
:10C5B000809362022C2F01C020E04091620250E083
:10C5C0004C5F5E4F0BEF1CE060E188E50E94CF2ED0
:10C5D00066EC7CE088E10E94A47711E0D0E08091D5
:10C5E0008C0682FF20C08EEF8D0F8430E0F48091A6
:10C5F0000705D23051F4282F30E035952795359531
:10C60000279545E468E18EE40CC0D43071F4282FFE
:10C6100030E094E0359527959A95E1F749E468E193
:10C620008AE582D802C081E001C080E090918C064A
:10C6300094FF0CC0D63039F42091190641E468E12A
:10C6400086E672D818C0D73009F4D8E0882399F06C
:10C6500080910705812301E009F400E04D2F50E0AF
:10C660004C5D554E8D2F880F8D0F880F21E068E1AE
:10C670008E5B0E944977110FDF5FD83008F4AFCF8F
:10C68000F2E0DF121DC029E048E367E181E40E9487
:10C69000717A20E6C21619F08EE2C81211C08C2DF4
:10C6A0000E94BD7C0E94C5158093070585E20E940B
:10C6B0009C7C8093190610921D0882E00E943B70BA
:10C6C00041E093E0D91240E08091C90560E2829593
:10C6D00081700E940E2F9091C90580FB94F9909370
:10C6E000C905E4E0DE1209C0C06264E68091080575
:10C6F0000E94B21F8093080501C0C0E24091080566
:10C7000050E02C2F68E288E70E94CD7921E0F5E027
:10C71000DF1220E04091D4044295469547706AEAC2
:10C720007CE080E30E94DC2E8295880F807E9091D1
:10C73000D4049F71982B9093D4040C94CD6E2AE06E
:10C740002D1508F487C063E67CE088E00E94A4779A
:10C7500041E086E0D81240E080916E0268E0869564
:10C7600081700E940E2F90916E0280FB91F9909340
:10C770006E0291FF1BC0C091C905C5FBCC27C0F953
:10C7800021E097E0D91220E04C2F63E57CE080E1C6
:10C790000E94DC2E81709091C90580FB95F99093E1
:10C7A000C9058C1791F00E94111D0FC0E2EBF3E058
:10C7B000808187FD1082818118160CF411823596D4
:10C7C00024E0E230F207A0F3D6CFC091C905C6FB42
:10C7D000CC27C0F941E088E0D81240E068E18C2F16
:10C7E0000E940E2F81709091C90580FB96F990935D
:10C7F000C9058C130E94111D0E94FE12882311F09E
:10C8000041E801C040E860E280E60E94477741E0ED
:10C8100099E0D91240E08091690268E281700E943B
:10C820000E2F9091690280FB90F99093690241E08C
:10C83000EAE0DE1240E08091690260E38295817057
:10C840000E940E2F9091690280FB94F990936902E7
:10C850000C94CD6E6FE17CE088E00E94A47721E02B
:10C86000FBE0DF1220E040916A026DEF7BE088E0A0
:10C870000E94DC2E80936A022CE0D21204C001E0F8
:10C88000C11103C001C0C0E000E02C2F40916C0238
:10C8900060E186E60E94AC3280936C0241E08DE05C
:10C8A000D81240E08091690268E183FB882780F913
:10C8B0000E940E2F9091690280FB93F99093690278
:10C8C00041E09EE0D91240E08091640260E28695EA
:10C8D00081700E940E2F9091640280FB91F99093D9
:10C8E0006402C5EFEC2ECBE0FC2EE7011FE301E074
:10C8F00086E0B82EAC2EAE18FE01449180916D02F8
:10C90000802321E009F420E068E2812F0E949176E3
:10C91000FFE0DF121DC0B09208098091F4078A1170
:10C9200017C029E048E067E28FEF810F0E94717A1B
:10C9300020E2C21619F08EE2C8120AC080916D0280
:10C94000802780936D0282E00E943B7010921D0848
:10C95000000F2196195F103769F60C94CD6E8EE1A9
:10C960009AE10E94C92E8AE080930A0994E09D15FD
:10C9700028F00E946B32F12C10E003C0FF24F394E6
:10C9800015E0E5E0FE9EE0011124C35FDD4FE0907D
:10C99000170861E479E088E00E94A47741E34F0D35
:10C9A00068E08EE10E944777D11202C02E2D01C0AF
:10C9B00020E048815981022F68E087E40E940B7AC9
:10C9C000D11214C08CE380933E014CE364EC80E010
:10C9D0000E94AF1F48815981480F511D87FD5A950C
:10C9E0005983488357FF02C01982188281E0810F62
:10C9F000D81207C063E18A810E94B21F8A8341E096
:10CA000001C040E0F11002C021E001C021E860E176
:10CA10008CE30E94611482E0810FD81205C0EE20E1
:10CA200019F02E2D03E002C020E002E04B8168E106
:10CA30008AE50E94AC328B8321E083E0810FD8121B
:10CA400020E04C8169E279E080E20E94DC2E8C8358
:10CA50001C5FD112E12CF11003C04091C70502C048
:10CA60004091C805EE2011F003E001C002E02E2D38
:10CA700068E28FE40E94AC32F11003C08093C705D6
:10CA800002C08093C805EDE0F2E08081918190932F
:10CA90006602809365028281809363028381809322
:10CAA000D30480916402948190FB80F980936402A6
:10CAB00085819681909304058093030587818093F7
:10CAC00005058085809306058091C905918590FBB9
:10CAD00087F98093C9050C94CD6E87E898E10E9490
:10CAE000C92E86E080930A09C09117086AEA7BE0A4
:10CAF00088E00E94A47721E0D11020E040916E02EE
:10CB000042954695477062E97BE088E00E94DC2E02
:10CB10008295880F807E90916E029F71982B9093E2
:10CB20006E02F1E0DF1209C064E280916F020E94A0
:10CB3000B21F80936F022C2F01C020E040916F0242
:10CB400060E186E60E94081322E0D21208C064E683
:10CB5000809170020E94B21F8093700201C0C0E0F9
:10CB60002C2F4091700268E184E50E94462F41E03D
:10CB700083E0D81240E080916E0260E282FB882759
:10CB800080F90E94302F90916E0280FB92F9909371
:10CB90006E0241E094E0D91240E080916E0268E2BA
:10CBA00083FB882780F90E94302F90916E0280FBD2
:10CBB00093F990936E0241E0E5E0DE1240E080914F
:10CBC0006E0260E3829581700E94302F90916E0218
:10CBD00080FB94F990936E020C94CD6E8FE798E1F0
:10CBE0000E94C92E85E080930A0910925601D091C7
:10CBF000060920E0D11009C043E060E08D2F0E94BB
:10CC0000A51FD82F8093060921E041E04D0F68E071
:10CC100080E00E9408138D2F0E94422E182F00E002
:10CC2000282F46E85BE068E08AE20E946D7766E6BE
:10CC30007BE088E00E94A477ED2FF0E0EE0FFF1F6D
:10CC4000E15CF74F40815181453651052CF44C3958
:10CC50005F4F24F0C2E003C0C0E001C0C1E08D2FEF
:10CC60000E947C1A811106C0CC2329F081E0D812E1
:10CC700002C002C0C0E080E0EE24E39400E0212F77
:10CC800048E168E10E944338C13011F081E0D812D8
:10CC900080E0E12C00E0212F48E160E30E9443386E
:10CCA000CC2319F081E022E0D21280E0EE24E3945C
:10CCB00001E0212F48E268E10E944338C13019F0B9
:10CCC00081E092E0D91280E0E12C01E0212F48E2DE
:10CCD00060E30E94433881E0E3E0DE1280E0E12C73
:10CCE00000E023E640E36EE10E94433881E0F4E097
:10CCF000DF1280E0E12C00E022E648E36EE10E94D2
:10CD00004338809106090E947C1A882311F08CE335
:10CD100001C08CE540E460E00E94807881E080936F
:10CD2000640961E08CE50E94C84980910609E82FFA
:10CD3000F0E0EE0FFF1FE15CF74FC081D181BE0133
:10CD40000E9454498C0189E18C9F90018D9F300D88
:10CD5000112437FF02C021503F4F532F550F550B61
:10CD6000432F60E382E70E94FB7989E1809F900175
:10CD7000819F300D112437FF02C021503F4F532FA8
:10CD8000550F550B432F68E084E50E94FB79CE01D7
:10CD9000409697FF02C0CE018F967C0175E0F59416
:10CDA000E7947A95E1F7E8016096D7FF02C0E801C1
:10CDB000AF9665E0D595C7956A95E1F7D195C19590
:10CDC000D1096C2F635E47E08CE58E0D0E94807860
:10CDD0006C2F605E47E089E58E0D0E947E78109290
:10CDE0006409DBC7F09067022F2D2F70F22EE22E20
:10CDF00081E0281741F092E0291739F0E5E02E177D
:10CE000031F0C4E005C0C6E003C0C3E001C0C7E024
:10CE100083E598E10E94C92EC0930A09D0911708B2
:10CE2000C091F40767E57BE088E00E94A477D11009
:10CE300013C08091690267E08295869587700E9491
:10CE4000B21F8295880F807E909169029F71982B06
:10CE50009093690221E001C020E04091690242956F
:10CE6000469547704F5C68E082E70E949176FF200C
:10CE700049F08DE08F0D8F70CC24C394823020F068
:10CE8000C12C02C0CC24C394F1E0DF1202C0CC2339
:10CE900011F000E001C00D2F2F2D4BE25BE060E1AF
:10CEA00084E20E946D77CC2079F167E27BE080E13B
:10CEB0000E94A47721E0D21202C0C13011F000E03C
:10CEC00001C00D2F209168022E5F49E05BE060E118
:10CED00088E40E946D7781E0D81202C0C23011F060
:10CEE00020E001C02D2F40916B0292E34902A00186
:10CEF0001124445D5E4F60E180E70E94CD79E1E05E
:10CF0000DE1267C082E01AC040916802F5E0FF12AD
:10CF100001C04F7021E0D21202C0C13011F020E0F8
:10CF200001C02D2F552747FD509502E01BE060E121
:10CF30008EE70E94CF2E81E0D81284C0809308092A
:10CF400080911C08882309F451C0C13051F018F0B9
:10CF5000C23031F12FC066E08F2D0E94B21FE82E43
:10CF600029C0CC2019F044E06EEF13C095E0F9120F
:10CF70000EC0809168024FE060E08F700E94AF1F8A
:10CF800090916802907F980F9093680213C04CE7CD
:10CF900060E0809168020E94AF1F809368020AC01F
:10CFA000CC2041F04AE06CEF80916B020E94AF1FF1
:10CFB00080936B0280916702982F9F70807F2E2D47
:10CFC0002F70822B809367029E1581F01092680269
:10CFD0000DC0E2E0DE120CC044E16CEE8091710203
:10CFE0000E94AF1F8093710221E203C0CC2051F157
:10CFF00020E240917102F5E04F02A00111244F514F
:10D000005F4F03EF1AE068E18CE40E94CF2E6AEED6
:10D010007AE080E20E94A47721E083E0D81220E049
:10D0200040916E02417060EE7AE080E20E94DC2E58
:10D0300090916E0280FB90F990936E0254E0F52E71
:10D0400018E203C042E0F42E18E195E0E912EFC0C7
:10D0500064EB7AE0812F0E94A477E090490521E0FB
:10D06000DF1020E04E2D4F716CE57AE0812F0E9499
:10D07000DC2E90914905907E980F90934905009180
:10D080006802492F552747FD50952E2D30E0421755
:10D09000530749F4402F50E034E0559547953A95B1
:10D0A000E1F7477001C040E088E0810F31E03F0DBB
:10D0B0009F7179F0933081F0953089F0973091F03D
:10D0C000993099F09B30A1F09C30A9F46CEC79E098
:10D0D00014C060E47AE011C062E37AE00EC066E258
:10D0E0007AE00BC06FEF79E008C06DEE79E005C023
:10D0F0006AED79E002C064EC79E021E0D31220E02F
:10D100000E94DC2E0F78E02EE0E18E9FE00C1124CF
:10D11000E092680290E1B92EB10E22E0C22ECF0C4F
:10D12000AE2CAA1CAA24AA1CDC1002C0CC2311F02D
:10D1300000E001C00D2F2A2D4AEB59E06B2D84E24F
:10D140000E946D77DC1002C0C13011F020E001C0F8
:10D150002D2F40914A05552747FD50956B2D8EE7A1
:10D160000E94CD7962EB79E08B2D0E94A477DC10D0
:10D1700022C081E080930809C1110FC080911C0872
:10D180008823C9F061E08A2D0E94B21F9E2D9F77EF
:10D1900081119068909368020EC0C13061F4809153
:10D1A0001C08882341F04FE761E880914A050E94FE
:10D1B000AF1F80934A0508E1B02EB10E83E0A82E80
:10D1C000AF0CE0904905E6FACC24C0F8DA1002C0B2
:10D1D000C13011F000E001C00D2F2C2D4EEA59E0B6
:10D1E0006B2D88E70E946D77DA101AC081E080937A
:10D1F0000809C11105C061E08B2D0E947E5B10C043
:10D20000C13071F480911C08882351F061E08C2DAD
:10D210000E94B21F9E2D9F7B8111906490934905BF
:10D2200084E08F0DD812B9C560E280E250C0F2E010
:10D23000EF1212C065EA79E0812F0E94A47721E005
:10D24000DF1020E04091490566E879E0812F0E94D7
:10D25000DC2E80934905A1C521E0E2129EC56CE653
:10D2600079E0812F0E94A47721E0DF1020E0409137
:10D27000490567E476E1812F0E94DC2E8093490501
:10D2800021E081E08F0DD81220E0409167024295A5
:10D29000437063E576E188E0810F0E94DC2E8370A5
:10D2A0008295807F909167029F7C982B9093670274
:10D2B00082E08F0DD81205C061E080E1810F0E94ED
:10D2C0007E5B83E08F0DD81268C560E288E1810F34
:10D2D0000E947E5B62C588E199E00E94C92E82E1CE
:10D2E00080930A0983E080930809C090F4078D2D8C
:10D2F0000E94AF5BA82EC8E0FC2E99249394DA100C
:10D3000003C0B090170801C0B12C4CE46F2D80E031
:10D310000E94477788E08A1510F448E301C041E392
:10D320004A0D6F2D85E00E9447778A2D90E0EBE053
:10D33000EA1508F00AC1F1E0CF1629F022E0C21682
:10D3400029F0E12C01C0EB2C712C02C07B2CE12CCC
:10D35000EC01CC0FDD1FCC0FDD1FC75CDA4FCC20FA
:10D3600011F000E001C00B2D2A8147E359E16F2D38
:10D370008DE00E946D778A810E94F112882E8111C2
:10D3800020C02E2D48816F2D86E30E94081318813E
:10D3900015327CF015526981812F0E940C2B9C0163
:10D3A000A2E8EA2E072D412F6F2D84E60E94AB2CB8
:10D3B00070C04981552747FD5095272D6F2D83E675
:10D3C00066C081E088120DC02E2D48816F2D86E346
:10D3D0000E941114272D49816F2D8DE40E94111494
:10D3E00058C092E089120DC02E2D48816F2D86E322
:10D3F0000E940813272D49816F2D80E50E94081394
:10D4000048C0E3E08E1223C0488147FF04C0409526
:10D41000FE2DF062EF2E552747FD50954F5F5F4F71
:10D4200004E119E02E2D6F2D89E40E94CF2E498151
:10D4300047FF04C04095272D2062722E552747FDD7
:10D4400050954F5F5F4F272D6F2D89E620C081E0FB
:10D45000C81611F020E001C02B2D48816F2D86E306
:10D460000E941114498147FF03C0409580E201C02A
:10D4700080E092E0C91202C02B2D01C020E0282BD1
:10D48000552747FD50954F5F5F4F6F2D84E60E94F3
:10D49000CD791B8117FF0CC01195E3E0CE1611F07A
:10D4A00020E001C02B2D41E26F2D89E60E9491768C
:10D4B00087EF810F843120F41F5F1C3109F419E0DC
:10D4C000F3E0CF1611F020E001C02B2D412F6F2D7E
:10D4D00089E60E94111480911C08882309F488C1F0
:10D4E000BB2009F485C121E0C216A9F0C21648F09C
:10D4F00082E0C81609F484C093E0C91609F496C006
:10D5000077C161E18A810E94B21F8A830E94F11271
:10D51000881238C16DC1E2E08E1691F0E81538F03E
:10D52000882071F0F1E08F1609F460C061C123E03A
:10D53000821609F436C184E0881609F457C058C130
:10D540006EE488810E94B21F59C0E1E0CE1609F452
:10D550009CC0F2E0CF1609F49AC0612C812CEC013A
:10D56000CC0FDD1FC80FD91FC255DB4FCC2009F4EB
:10D5700091C000E02A812F7047E359E16F2D8DE0C3
:10D580000E946D778A818F700E94F112782E882315
:10D5900009F482C021E082139BC0262D48816F2DA3
:10D5A00086E30E941114282D49816F2D8DE40E947D
:10D5B00011144A8142954F7049300CF04F5FF3E0EF
:10D5C000CF1609F4BAC020E06F2D88E60E9411142E
:10D5D00080911C08882309F40BC1BB2009F408C101
:10D5E00021E0C212ACC0E1E07E12CFC040915801F0
:10D5F000642F61952AE088810E94BE1F8883F8C04D
:10D6000092E0891609F4EBC0981540F0882009F4DF
:10D61000DAC0E1E08E1609F4D9C0EAC0F3E08F1653
:10D6200009F4E0C024E08212E3C0CDC08B8197EF03
:10D63000980F933108F48F5F9BE1980F933110F4AA
:10D64000815002C08C3121F0843E19F487EF01C073
:10D6500089E0909158014FEF490F692D691B2AE02D
:10D660000E94BE1F893021F0873F19F484EE01C06B
:10D670008CE196EF980F933108F481509CE1980F5C
:10D68000933108F48F5F8B83B3C06B2C67CF8B2CE7
:10D69000612C65CF0B2D6ECF188115327CF01552A1
:10D6A0006981812F0E940C2B9C01E2E8EE2E082D4F
:10D6B000412F6F2D84E60E94AB2C13C04981552762
:10D6C00047FD5095282D6F2D83E60E94CD7909C026
:10D6D00082E078120DC0282D49816F2D80E50E94CF
:10D6E0000813262D48816F2D86E30E94081361CF11
:10D6F000488147FF04C04095962D9062692E5527BA
:10D7000047FD50954F5F5F4F00E119E0262D6F2DCB
:10D7100089E40E94CF2E498147FF04C04095E82D3F
:10D72000E0628E2E552747FD50954F5F5F4F282DA5
:10D730006F2D8BE60E94CD793CCF2B2D45CFC216A5
:10D7400098F082E0C81699F193E0C91251C08A811D
:10D750006FE082958F700E94B21F8295807F9A81C0
:10D760009F70982B9A8344C08A816EE08F700E94CC
:10D77000B21F8F709A81907F982B9A830E94F1122A
:10D780007816B1F11882198233C07E1638F0F2E0B3
:10D790007F1621F023E0721621F02AC04EE460E0EB
:10D7A00002C043E66EEC88810E94AF1F27CF81E064
:10D7B000781661F0781638F092E0791681F0E3E09F
:10D7C0007E1681F015C04DE763E80EC04091580108
:10D7D000642F61952AE089810E94BE1F08C04EE433
:10D7E00060E002C043E66EEC89810E94AF1F89832E
:10D7F000A394F8E0FF0E20E4F21281CDCEC282E9BC
:10D8000098E10E94C92E81E180930A0983E0809308
:10D810000809A090F4078D2D0E94AF5B982E8FE031
:10D820008D15A0F0ED2DF0E0EE0FFF1FEB50F84F3F
:10D830004081518157FF02C04F5F5F4F559547951B
:10D8400044525A4F60E08EE40E94FB7980911802A6
:10D85000803819F59FE09D1540F14D2D50E0FA01FB
:10D86000E919F109EE0FFF1FEB50F84F20813181CC
:10D87000A11013C085E0849FF001859FF00D112455
:10D88000EE54FC4F8281882319F03195219531099E
:10D890003483238382E0EFD3EAD488E0C82E95E076
:10D8A000592E2AE0E22EF12C93C0E0E1DE12F5CFF2
:10D8B00089E180931B0880E80E94BD7C0E944B5345
:10D8C000ECCFE92DF0E05E9EE0015F9ED00D1124CB
:10D8D000CE54DC4FEE0FFF1FEB50F84F808191814B
:10D8E0004A812B813C81442319F0319521953109DE
:10D8F000821B930B833391050CF06EC08E3C9F4FBF
:10D900000CF46DC01DE266246394690C20E0462D82
:10D910006C2D80E00E944013412F6C2D8BE40E94FF
:10D92000477780916E0281FF5EC01DE7712EB12C9A
:10D9300044244A944C0C372C3194D91057C0AB1066
:10D9400055C02091170880911C08882309F450C005
:10D95000222309F44DC010925601822E80910805B1
:10D96000882309F453C00B811C810115110509F0AE
:10D9700041C0C801B7010E94DB8F82E0B81609F4EC
:10D9800066C093E0B91609F486C0E1E0BE1609F45A
:10D9900042C020624B815C816C2D8DE20E94CD796A
:10D9A000882059F022E048EE53E068E17CEF8B815B
:10D9B0009C810E94D51E9C838B83B39424E0B21279
:10D9C000BCCF88E08C0D803409F47EC0C82E962C24
:10D9D000F0E19F1276CF6AC0411103C0F0C141113E
:10D9E000EEC11FE790CFB4E67B2EA1CF20E0ABCFF6
:10D9F000812CB4CF90E0801791075CF091958195D0
:10DA00009109081719070CF0B4CF03C000E010E02B
:10DA1000B0CF8C01AECF18811456AB01410F511D10
:10DA200017FD5A954338FFEF5F0714F443E85FEFA3
:10DA30006C2D88E40E94CD79882009F4BECF49E19D
:10DA4000632D812F0E94AF1F8C598883B6CF8981A7
:10DA50008C59AB01480F511D87FD5A954E37510522
:10DA600014F04DE750E06C2D86E60E94CD79012B35
:10DA700031F029E048E3642D82E30E94717A882026
:10DA800009F49BCF8981472D67EE8C590E94AF1F07
:10DA90008456898392CF422F6C2D8A810E94302F29
:10DAA00091E0811101C090E09A8387CF21E0E0E10D
:10DAB000DE1220E080911B08811183C14FEF58E0F6
:10DAC0006C2D82E10E947F7768C18FEE98E00E9402
:10DAD000C92E89E180930A09C090F4078D2D0E9418
:10DAE000AF5BE82EF8E0FF2EA0E1BA2E8091D404BF
:10DAF000E11021C0D11010C010920809C091170880
:10DB000060E18F710E94B21F8F719091D404907E5A
:10DB1000982B9093D40401C0C0E04091D4044F717D
:10DB200050E0485F5F4F0FED18E02C2F6F2D8CE613
:10DB30000E94CF2E2CC18F719B2C981ACE2DD0E035
:10DB4000DE1003C082E080930809C131D1052CF4B6
:10DB5000CC0FDD1FCD52DB4F04C0CC0FDD1FC95CE5
:10DB6000DA4F10E0DE1009C0C11207C0009117089B
:10DB7000002321F062E0A62E02C000E0A12C9E143A
:10DB800008F49FC0111118C020E04E2D6F2D80E0C9
:10DB90000E944013488142954695469543702A2D30
:10DBA00067ED78E08F2D0E94DC2E8295880F880F1C
:10DBB000807C98819F7332C08881113091F580906C
:10DBC0005801982F907C903811F45FE1852E482FF2
:10DBD000440F440F459545954D314CF023EE240FED
:10DBE00040EC58E06F2D85E40E946D7705C0202F32
:10DBF0006F2D85E40E941114AA2009F4C4C060911D
:10DC0000580161958881880F880F2AE0482D8595F5
:10DC100085950E94BE1F8F739881907C982B988366
:10DC2000B2C0982F907C4981903491F447FD03C095
:10DC30004F3024F401C040E0242F01C02FE029839D
:10DC40004CEB59E16F2D88E70E946D774FE015C0CE
:10DC5000903831F5880F880F81378CF047FD04C06C
:10DC600049321CF049E201C040E049834F5F202F58
:10DC70006F2D80E60E94232A49E260E01BC04F36E8
:10DC80000CF04FE64983552747FD509540585F4FAC
:10DC9000202F6F2D88E70E94CD794FE660E80AC0FB
:10DCA000552747FD5095202F6F2D88E70E94CD798D
:10DCB0004DE763E8AA2009F466C089810E94AF1F7E
:10DCC00061C0111123C06DEB78E08F2D0E94A47705
:10DCD00020E04E2D6F2D86E10E94FD79AA2071F083
:10DCE00040915801415088812AE060E08F710E9484
:10DCF000BE1F8F719881907E982B988348814F71B9
:10DD0000202F6F2D8EE10E9411143DC088811130AB
:10DD100081F4482F4295469547702A2D6FE878E0A8
:10DD20008F2D0E94DC2E8295880F807E98819F71B6
:10DD300075CF82958695877090E04981069764F04B
:10DD4000493208F049E249834F5F202F6F2D80E66A
:10DD50000E94232A69E210C04B3F38F450E0202F84
:10DD60006F2D86E60E94CD7906C0485F202F6F2D6B
:10DD700084E50E94DB2D6FEFAA2029F0898190E0D5
:10DD80000E94B71F89831F5F133009F0EBCEE39425
:10DD900088E0F80E90E4F912A9CEDF91CF911F919F
:10DDA0000F91FF90EF90DF90CF90BF90AF909F903A
:10DDB0008F907F906F905F904F903F9008951EE7F7
:10DDC000A2CD20E07BCE1F93CF93DF93EC011AE02E
:10DDD00088810E948B380E949B3889931150C1F72B
:10DDE000DF91CF911F9108959C01265F3F4FFB016A
:10DDF0004491DC014D93CD013196A217B307C1F7D1
:10DE00000895EBE1F6E080E090E021913191820FFE
:10DE1000931F26E0E333F207C1F7089587E7EAE1AD
:10DE2000F6E0DF011D928A95E9F78BE080931A06F0
:10DE300089E1809348068AE58093490681E08093D2
:10DE40005E068CE180934B06EBE1F6E020E032E0E9
:10DE500080E093E02193319395878487938F828F1D
:10DE6000B6E0E932FB07B1F765EB7CE18BE696E0C3
:10DE7000BBDFC7DF90934606809345060895EF9277
:10DE80000F931F9361E0680F88ECE82E02EC13E01B
:10DE900028E532E042E085E199E074D621E0823C59
:10DEA000934009F020E0822F1F910F91EF90089589
:10DEB000CF93C82F22EC33E0E8E5F2E0DF01C9019F
:10DEC0001D920197E9F76AEA7CE1CF018DDF8C2F83
:10DED00090E06AE070E001960E94DB8F605D6093E5
:10DEE0005D02805D80935E0284E08093480582E05D
:10DEF00080936A0280E00E94587E8C2FCF91BFCF22
:10DF00000F931F93CF93DF93EB01042F803120F504
:10DF100061E0680F85E199E086D410E0A80160E235
:10DF200070E0CE010E9450904AE050E0BE0185E1D1
:10DF300099E0FCD40A9781F485E199E066D4C00F9A
:10DF4000D11F009749F06AE070E00E94DB8F805D8E
:10DF50008A93862F972FF5CFDF91CF911F910F9145
:10DF600008958F5F0AC461E0680F85E199E05BD492
:10DF700082EC93E0E8E5F2E0DF019C011D92215084
:10DF80003040E1F742EC53E0BF0185E199E0CEC4B7
:10DF9000FF920F931F93CF93DF93CDB7DEB76897B0
:10DFA0000FB6F894DEBF0FBECDBF01E0080F102FF3
:10DFB0001031B0F4FF24F394F10E8F2DDED38111D4
:10DFC0000DC0602F85E199E02ED461E0610F28E556
:10DFD00032E042E0CE01409685D506C01F2DE8CF45
:10DFE000103179F780E017C04FE050E0BE016F5F5D
:10DFF0007F4F85E199E034D4882349F0482FBE0152
:10E000006F5F7F4FCE014096F4D4A895EDCFCE013F
:10E0100040968ED581E068960FB6F894DEBF0FBEAD
:10E02000CDBFDF91CF911F910F91FF900895EF9297
:10E030000F931F9361E082E79CE10E94C71C80E67A
:10E040009CE10E94B71534D398ECE92E07E710E065
:10E050002AE136E041E060E085E199E093D5873739
:10E06000910521F081E59CE10E94FA1C80E01F915E
:10E070000F91EF901DCFCF93C82F8770A1F0909193
:10E080002009982B909320090E94EA1290931F096F
:10E0900080931E098C2F90E024E0959587952A9512
:10E0A000E1F780932109CF910895CF93DF9322D395
:10E0B000811102C080E02EC097D287FDFBCF60E0C7
:10E0C00085E199E0B0D387E7EAE1F6E0DF011D9250
:10E0D0008A95E9F747E750E0BF0185E199E026D44A
:10E0E0008BE696E070DE80911A068B3040F481E07A
:10E0F0008093D4018BE080931A0681E0BCDFC0914D
:10E100004506D09146067DDE21E0C817D90709F003
:10E1100020E0822FDF91CF910895EF920F931F930C
:10E12000CF93DF9310926309C0912009CC2309F4A7
:10E1300098C0909121099F5C9093630981111CC044
:10E140000E94EA1220911E0930911F09821B930B35
:10E15000883C910508F485C080912109882361F0ED
:10E16000815080932109882339F00E94EA1290930C
:10E170001F0980931E0975C01092210980910B0917
:10E1800081116FC0DC2FD470C2FD02C081E001C0DC
:10E1900083E080930B09C0FF2CC082E38093630966
:10E1A000809120098E7F8093200944E1E42E07E7C7
:10E1B00010E02AE136E041E061E18CE099E0E2D450
:10E1C0008737910519F461E180E02FC08091120931
:10E1D000823051F480912009816030C08091120911
:10E1E000823029F1D1113BC080EC9CE10E94FA1CE5
:10E1F00036C0C1FF34C083E3809363098091200956
:10E20000897F8093200934E1E32E02EC13E028E5B6
:10E2100032E042E061E18CE099E0B4D4823C93408A
:10E22000E9F68091470661E18F5FB5D218C0809111
:10E230002009D11102C0826001C08660809320094C
:10E240000E94EA12885C910990931F0980931E092D
:10E250008091B10D833019F4A8951092B10D1092F0
:10E260000B09DF91CF911F910F91EF90089580914D
:10E270002009882351F081E050DF8091B10D833077
:10E28000B1F7A8951092B10DF2CF0895EF92FF92D9
:10E290000F931F93CF93DF93C82F803108F009C1EC
:10E2A00062DE8F3F910509F010F48C2F01DE88E5C6
:10E2B00092E089DD80910005811107C0809169029B
:10E2C000869583708E5F8093000580916702982FFA
:10E2D0009295969596959370933029F09093490571
:10E2E000806C809367028091830E80648093830E9C
:10E2F0000E94EF8D80914805823008F092C010E0B6
:10E30000812F0E94F712EC0189818150843018F42A
:10E310000E94DD1289831F5F103291F7CEEAD4E0AC
:10E3200000E010E08A818F700E94F112882389F04A
:10E330008230C1F4C80181559B4F7C01FC01808172
:10E34000882339F085302CF481500E94DD12F701CA
:10E3500080838881882331F0853024F481500E94A5
:10E36000DD12888323960D5F1F4F04321105D1F60D
:10E37000C0E0D0E08E01085A1D4FF801ED5EFC4F61
:10E3800080810E94F112882391F08230E9F47801B3
:10E39000FEEEEF1AFCEFFF0AF7018081882339F0C7
:10E3A00085302CF481500E94DD12F70180830F5ECE
:10E3B0001C4FF8018081882339F085302CF481507E
:10E3C0000E94DD12F80180832496C831D10591F6B0
:10E3D00088E3E2E0F4E0AAE7B8E001900D928A95C4
:10E3E000E1F7CAE7D8E010E00EE0812F0E94DD12CD
:10E3F0008150089FD0011124AE5FBB4FFE01802FDA
:10E4000001900D928A95E1F71F5F2E96143069F7FF
:10E4100085E99CE10E94FA1C82E0809348052BDE8E
:10E4200026DF80914805833090F580E090E0FC0184
:10E43000E255FB4F2281322F3F703C3019F4207F90
:10E440002A6022832281322F3F703D3019F4207FD1
:10E450002B60228303968432910549F780E090E097
:10E460002AE03BE0FC01E559FA4F40814C3009F4C9
:10E47000208340814D3009F4308304968831910522
:10E4800089F783E08093480582E0F5DDF0DE809136
:10E490004805843070F4809175068093070582E802
:10E4A0009CE10E94FA1C84E08093480582E0E3DD51
:10E4B000DEDEEDE0F2E08091630282838091D3049E
:10E4C000838380916502909166029183808380911D
:10E4D000640281708483809105058783809106059D
:10E4E00080878091030590910405968385838091B0
:10E4F000C90587FB882780F981870E94443F0E94D5
:10E500004A3FDF91CF911F910F91FF90EF900895B7
:10E5100040E450E060E070E082E299E00C944A7BD5
:10E5200041E050E062E070E084E299E00C944A7BC4
:10E53000CF93DF931F92CDB7DEB7698390E1899FB8
:10E54000B001112441E050E0CE0101960E944A7BC7
:10E550000F90DF91CF910895CF93DF931F92CDB7A6
:10E56000DEB790E1899FB001112441E050E0CE0177
:10E5700001960E94579089810F90DF91CF91089565
:10E58000CF93DF93D82FC82F8C2FE6DF882321F07D
:10E590008C2FE2DFC82FF8CF609124098C2FC8DFC1
:10E5A000D0932409DF91CF91BBCFCF93C0912409A1
:10E5B000CC2341F08C2FD0DF80932409B1DF60E0C1
:10E5C0008C2FB6DF8C2FCF910895CF93DF9380915E
:10E5D0002409C0E0D0E0882319F02F96BDDFFBCFDF
:10E5E000CE01DF91CF910895DF92EF92FF920F93CA
:10E5F0001F93CF93DF9380E091E0E8E5F2E0DF0145
:10E600009C011D9221503040E1F7C6E2D9E0F12C87
:10E6100034E1F31205C08091240904E219E002C03C
:10E620008E01888190E0E12CDD24D394DF0C0097EB
:10E63000E9F09C01245031092C3F310530F4FC01F4
:10E64000E85AFD4F2081222361F0EE2021F060E0A6
:10E650008E2D6EDF03C0D8011C925ADF80E090E05F
:10E66000E6CFD082E82E78DF90E0E1CFF3942396D6
:10E67000B5E1FB12CDCFC4E0D0E0FE01E85AFD4F7A
:10E680008081811107C0609124098C2F51DFC093D4
:10E69000240946DF2196C115F1E0DF0771F780E01C
:10E6A000DF91CF911F910F91FF90EF90DF90089530
:10E6B000CF9380E4E2E2F9E0DF01982F1D929A9572
:10E6C000E9F796E0909322098093230980E18093F3
:10E6D000250984E0C1E0C80F6C2F2ADFCF3F11F07D
:10E6E0008C2FF8CF60E08FEF23DF84E08093240944
:10E6F000CF910ECFCF93DF9340E450E060E070E025
:10E7000082E299E00E94579080912309811103C011
:10E7100080E48093230980912209843009F5809157
:10E7200023098034E9F4C0912409DC2FCC2329F09B
:10E730008C2F12DFDC2FC82FF9CF80E8C1E0C80F83
:10E740006C2FF6DECF3F11F08C2FF8CF60E08FEF0B
:10E75000EFDE60E88D2FECDE86E080932209D8DEC4
:10E7600080912209863029F481E090912309903428
:10E7700009F080E0DF91CF91089590E0FC01EE0F69
:10E78000FF1FE80FF91FEE5DF64F81E094819111B4
:10E7900001C080E00895CF93DF9390E0EC01CC0FAF
:10E7A000DD1FC80FD91FCE5DD64F8C819D81AE81F4
:10E7B00070E0FB01EE0FFF1FE60FF71FEE5DF64F57
:10E7C0002481358146812C833D834E8384839583C8
:10E7D000A683DF91CF919CCECF9390E09C01220F36
:10E7E000331F280F391FF901EE5DF64FC481F9017F
:10E7F000EA5DF64F1082118212828ADECC2319F074
:10E800008C2FCF91BDCECF910895FC01808190E0F7
:10E81000FC01EE0FFF1FE80FF91FE95DF64F918134
:10E8200080819F700895CF93DF93FC0160831282F3
:10E83000118270E0CB01880F991F860F971FEC01A2
:10E84000CE5DD64F2C812383148215821682FC0163
:10E85000E85DF64F808182958F70DF91CF910895AA
:10E86000AF92BF92CF92DF92EF92FF920F931F93DE
:10E87000CF93DF931F92CDB7DEB78C01FC0180816F
:10E8800090E0FC01EE0FFF1FE80FF91FE95DF64F66
:10E8900080812181922F9F70F80121813281821B1A
:10E8A000930B7A018417950708F47C015B016701DB
:10E8B000C114D10421F1F8018381882301F164811D
:10E8C0006F5F648370E0F0E18F9F600D711D112414
:10E8D00041E050E0CE0101960E9457908981F501F8
:10E8E00081935F01F80184818F3028F01482838145
:10E8F00033DEF8018383F1E0CF1AD108D9CFF801D4
:10E90000818192818E0D9F1D8C199D099283818337
:10E910008E2D8C190F90DF91CF911F910F91FF9049
:10E92000EF90DF90CF90BF90AF9008957F928F923D
:10E930009F92AF92BF92CF92DF92EF92FF920F938E
:10E940001F93CF93DF934C016B018A01C0E0D0E0AD
:10E950005C0125E0A20EB11CC017D107D8F5F40167
:10E9600085818F7781F0F4014581F42FFF777F2E29
:10E970002F2F30E0C8018C1B9D0B8217930758F492
:10E98000702E7C1A08C041E050E0B501C40168DF78
:10E99000813049F31FC0E72CF12CC6018C0F9D1F5D
:10E9A00047FF06C0A70160E070E00E9450900BC0D6
:10E9B000A701BC01C40154DF871529F0FE01E80F4F
:10E9C000F11DCF0108C0CE0DDF1DF401858187192F
:10E9D0008583C2CFCE01DF91CF911F910F91FF9020
:10E9E000EF90DF90CF90BF90AF909F908F907F90EF
:10E9F0000895AF92BF92CF92DF92EF92FF920F9362
:10EA00001F93CF93DF93EC018B01D42E8B81811167
:10EA100010C089819A81892B61F4E880F12CC5DDD1
:10EA20008B83F701EE0FFF1FEE0DFF1DEE5DF64F1E
:10EA30008483CD2C8FE0A82ECC2009F43CC0EF803D
:10EA4000F8840E94EA12E81AF90AF7FE02C082E08E
:10EA500004C08B81811103C081E08E832CC09C8116
:10EA60009F3058F01C8278DD811104C09EDD682F34
:10EA70008B815EDD8B8170DD8B838B81882361F3DD
:10EA80006C819A2D961BBC2C9C1508F4B92EEB2C8E
:10EA9000F12C70E090E1899F600D711D11246F5F72
:10EAA0007F4FA701C801F6D50E0D1F1D8C818B0D60
:10EAB0008C83CB18C1CF6D2D70E06C197109298141
:10EAC0003A81260F371F3A8329838D2D8C19DF91C8
:10EAD000CF911F910F91FF90EF90DF90CF90BF905B
:10EAE000AF900895EF92FF920F931F93CF93DF9310
:10EAF000EC01F62EE42E890196DE6F2D70E0FB010D
:10EB0000EE0FFF1FE60FF71FE95DF64F1082E2944C
:10EB100030EFE322E1820E94EA12800F911F988772
:10EB20008F83DF91CF911F910F91FF90EF90089508
:10EB30001F93CF93DF93EC01888190E0FC01EE0FEF
:10EB4000FF1FE80FF91FE95DF64F898180839A81E5
:10EB50009F708181807F892B81838B81882321F025
:10EB6000FBDC182F81110AC010E0D2DC112311F058
:10EB7000812F06DDDF91CF911F91089560E08B8199
:10EB8000D7DCF3CF7F928F929F92AF92BF92CF92BA
:10EB9000DF92EF92FF920F931F93CF93DF931F9219
:10EBA000CDB7DEB76C0159012E2D30E09BDF198205
:10EBB0004501E12CF12C77247394F40181914F01EC
:10EBC0009981811108C071104CC08081811105C0EC
:10EBD000772473941BC071100AC080E09F3718F42B
:10EBE000E016F10661F5772081F0782E01C0712CD6
:10EBF000992329F19068998341E0BE016F5F7F4FAF
:10EC0000C601F7DE8130D1F026C0782E9923B9F005
:10EC100041E0BE016F5F7F4FC601EBDE8130D9F46A
:10EC20004981B701641B71096A0D7B1DC601E1DED4
:10EC30009981891719F0981B99830DC019828981D0
:10EC40008F5F8983A895FFEFEF1AFF0A0E151F0546
:10EC500008F0B3CF08C089818F778701081B11099D
:10EC600002C0872DBBCFC60163DFC8010F90DF91C3
:10EC7000CF911F910F91FF90EF90DF90CF90BF90B9
:10EC8000AF909F908F907F90089580E094E0E5E6AC
:10EC9000F9E0DF019C011D9221503040E1F7089519
:10ECA000FF920F931F93CF93DF93FA011491319644
:10ECB0007491795F769576957695DA011396FA01D7
:10ECC00032964491249FA00DB11D1124669566953E
:10ECD000669590E0F0E86F9F800D911D112420E073
:10ECE00030E060E08B59964F412F50E0671799F064
:10ECF0000A2FEC01C20FD31FFD01FE2EF01AF116F0
:10ED000020F4F490F9923196F8CFA40FB51F6F5FFD
:10ED100020583F4FEBCFDF91CF911F910F91FF9084
:10ED20000895CF93DF93382F463128F4842F880F2E
:10ED3000840F880FA9C086E0830F20FD08C021FD45
:10ED400002C090E005C09091780D96FFFACF91E057
:10ED5000A32FB0E0562F587F70E1579FA00DB11D33
:10ED60001124AB59B64F22FF43C04E3211F088E058
:10ED7000830F24ED240F2F3010F44B5211C02FEBD2
:10ED8000240F2A3110F441530BC02FE9240F2A31EC
:10ED900010F4465305C04F3511F44AE201C040E07B
:10EDA000EEE04E9F900111242952334E433311F06F
:10EDB000463311F41197825047E0F9015491379688
:10EDC000E491411102C0E0E050E02F5F3F4F9923F2
:10EDD00011F05095E095FCE0A43EBF0730F45C9341
:10EDE000ED01C058DF4FE8831196415030F74CC019
:10EDF00023FF07C0892F81958D9385E0830F31E034
:10EE000001C030E025E0429FF0011124E350F04EB4
:10EE1000677011F1AD014B5F5F4F249130E0062E1A
:10EE200002C0220F331F0A94E2F77DE0A536B70730
:10EE300018F49C9192279C93ED01C058DF4F9DE000
:10EE4000C536D90718F4988193279883119631967F
:10EE5000A417B50711F718C025E04491332311F02A
:10EE6000243041F05DE0A536B50718F491114095C6
:10EE70004C931196215031962111EFCF6DE0A536BC
:10EE8000B60710F491959C93DF91CF91089520E0FF
:10EE900048CFEF92FF920F931F93CF93DF93F62EFD
:10EEA000122F902F9071E92EFA01112379F0EE20A4
:10EEB00011F0408101C04491EF012196442331F0CB
:10EEC000202F6F2D2EDF1150FE01EFCFDF91CF915C
:10EED0001F910F91FF90EF9008950F93FA01949175
:10EEE0004F5F5F4F929F400D511D1124292FD1DF9D
:10EEF0000F9108950F9300E0CCDF0F910895FF92DA
:10EF00000F931F93CF93DF93162F022F922F9071A1
:10EF1000F92EEA01FF2011F0488102C0FE01449160
:10EF2000442361F04F3131F4185F103438F480E03D
:10EF30002196F0CF202F612FF4DEFACFDF91CF9111
:10EF40001F910F91FF900895AB0120E0682F80E0A2
:10EF5000D6CFFB01442341F09491992351F09F3186
:10EF600009F441503196F6CF20E0AF01682F80E0E0
:10EF7000C6CF089520E0C3CFFF920F931F93CF9386
:10EF8000DF93082FF62EEA0114E1180F15504C2FCD
:10EF90004F704A301CF0495C28E002C0405D20E020
:10EFA0006F2D812FBEDE84E0D695C7958A95E1F757
:10EFB0001013ECCFDF91CF911F910F91FF90089527
:10EFC000222321F09091780D96FD0895480F962FF9
:10EFD000987FE82FF0E020E1929FE00DF11D1124D1
:10EFE000EB59F64F677059F4DF018E1B982F9A0F7B
:10EFF000941720F49C9190959D93F8CF08952FEF4E
:10F0000030E002C0220F331F6A95E2F7522F232F00
:10F010008E1B982F9E0F941798F49DE0E536F90704
:10F0200018F4908195279083DF01A058BF4F9DE091
:10F03000A536B90718F49C9192279C933196E9CF95
:10F0400008952DE08536920760F4FC01208130910F
:10F050006409332319F0262B313009F02627FC01EF
:10F0600020830895262F287F6770E62FF0E0E95768
:10F07000FD4D649190E030E1239F800D911D11249E
:10F080008B59964FDECFEF92FF920F931F93CF9342
:10F09000DF93F42E47FF02C0840FF194962F987FE0
:10F0A000C82FD0E080E1989FC00DD11D1124CB590D
:10F0B000D64F6770E62FF0E0E957FD4DE490FF2052
:10F0C000B1F08DE0C536D80790F4022F10E020FF94
:10F0D00008C06E2DCE01B5DF15950795202F20684D
:10F0E00003C015950795202FFA942196E8CFDF915C
:10F0F000CF911F910F91FF90EF9008952FEFC3CF05
:10F100001F93CF93DF93142F47FF02C0640F119515
:10F11000962F987FC82FD0E080E1989FC00DD11D19
:10F120001124CB59D64F862F877099F0E82FF0E045
:10F13000E957FD4D64916195180F185017FF0DC0E8
:10F14000E12FFF27E7FDF095E157FD4DE4916E0FAC
:10F1500004C018303CF018506FEFCE0172DFC05879
:10F16000DF4FF7CF111654F4E12FFF27E7FDF0959D
:10F17000E957FD4D64916150CE0163DFDF91CF917E
:10F180001F9108953F924F925F926F927F928F925C
:10F190009F92AF92BF92CF92DF92EF92FF920F9326
:10F1A0001F93CF93DF93182FB62E802F05FF04C037
:10F1B00004FF04C002E003C000E001C001E0982F9A
:10F1C0009F77C92EE7FE04C0E1946624639401C0D2
:10F1D000612C57FF0AC050954095309521953F4FBF
:10F1E0004F4F5F4F7724739401C0712C82FF06C08C
:10F1F00098E09093650DE8E0DE2E05C096E09093D0
:10F20000650D75E0D72E86FF28C071101D0D283EB4
:10F2100083E038074105510514F01D0D05C0243663
:10F2200031054105510514F01D0D05C02A30310589
:10F23000410551050CF01D0D002381F0023031F421
:10F2400024363105410551054CF41D0D2A30310598
:10F25000410551051CF41D0D01C01D198091650D5E
:10F26000810F8093650D023011F490EFC90E882450
:10F27000839452E0A52E912CFF24E7FCF09466E0E5
:10F28000562E5B0CE82DF0E0EE16FF060CF45DC088
:10F290006AE070E0C9010E94DB8F382EEB0140E389
:10F2A000442E480E2C2D442D6B2D812F3ADD081154
:10F2B0002FC0C2FE1AC08FEF830D833008F4A394D1
:10F2C000CE016AE070E00E94DB8F823011F0843062
:10F2D000D9F484E3481204C099249394910E15C084
:10F2E00099249A94910EA39410C03EEF432E410EA0
:10F2F0008FEF810FC0FE04C047E06B2D01DF02C01D
:10F30000652DB0DE142D01C0912E209709F000E08C
:10F310009E01442737FD4095542F211531054105A5
:10F32000510581F4002331F0023059F491E0981531
:10F3300040F008C0C4FE09C0611004C080EFC80ED0
:10F3400001C000E01D1983949DCF992059F09A9433
:10F350004A2D6CE06B0D892DD1DE4A2D6DE06B0DD1
:10F36000892DCCDE772031F02C2D4DE26B2D812FB5
:10F370008D19D7DC80E0DF91CF911F910F91FF9025
:10F38000EF90DF90CF90BF90AF909F908F907F9045
:10F390006F905F904F903F900895EF920F93022FE0
:10F3A0009A01442737FD4095542FF5E0EF2EEADE11
:10F3B0000F91EF900895CF93DF93D62FC22F206245
:10F3C00050E0EBDFC7FD08C02C2F46E76D2F809182
:10F3D000650DDF91CF91A5CCDF91CF9108959091EC
:10F3E0003D0120914906921710F422E001C020E06F
:10F3F000242B492FE0CF20E0D0CFEF920F93022FA4
:10F40000005F242F30E040E050E0A2E0EA2EBADEB8
:10F410000F91EF900895DF92EF92FF920F931F9359
:10F42000CF93DF93182FE62EEA01F22E822F8470FD
:10F43000D82E22FF05C01D5F57FF0FC087E103C014
:10F4400057FF0BC08FE02F2D4DE26E2D912F981B93
:10F45000892F67DCD195C195D1092F2D20234AE34F
:10F460006E2D812F5EDC6CE370E0CE010E94DB8F9D
:10F47000462FC82FD1101E5F2F2D6E2D812FBDDF7F
:10F48000DD2011F085E101C08FE0810F202F4C2F8E
:10F490006E2DDF91CF911F910F91FF90EF90DF9034
:10F4A000ACCF0F931F93CF93DF93C82FD62F142F7A
:10F4B000022F422F25DE123030F0402F6D2F8FEFBC
:10F4C000810F8C0F1DDE6FEF6D0F600F412F8C2FA2
:10F4D00015DE412F6D2F8C2FDF91CF911F910F9152
:10F4E0000DCECF93C091640991E090936409D9DF68
:10F4F000C0936409CF9108950F931F93CF93DF9327
:10F50000182FC62FD22FE42FF0E03297053608F0DF
:10F5100004E60E9FC0010F9F900D112464E670E079
:10F520000E94DB8F062F2D2F6C2F812FDADF002317
:10F5300061F0D150DC0FCF5F1F5FCD1730F4402F4B
:10F540006C2F812FDBDDCF5FF8CFDF91CF911F9143
:10F550000F910895A998AB988BBBAD9AAD98AB9AD3
:10F56000A99A08958EEAF6DF80917A0682FF04C098
:10F5700080EAF0DF88EC03C081EAECDF80ECEADFB0
:10F580008FEAE8CFCF93C82F81E08093620981E8AA
:10F59000E1DF8C2FDFDF10926209CF910895809117
:10F5A0004806F0CFCF93DF9381E080936209AA9859
:10F5B0002AE02A95F1F700C0AA9A8CED95E0E5E0E3
:10F5C000EA95F1F7000001970097C9F7AC98C0EDF4
:10F5D000DCE1FE018491BEDF2196FCE1C73DDF073F
:10F5E000C1F7C0DFDF91CF91DACF0F931F93CF9395
:10F5F000DF9340916309442321F08091780D86FDCB
:10F600003AC081E08093620980917A0682FD02C04F
:10F6100004E001C000E010EBC5E6D9E0802F9ADFDE
:10F6200080E198DF812F96DFA998AB9AFE019E01B9
:10F6300020583F4F80818BBBAD9AAD9881818BBBA9
:10F64000AD9AAD9882818BBBAD9AAD9883818BBB0F
:10F65000AD9AAD983496E217F30761F7EF01AB9AD4
:10F66000A99A1F5F183BD1F610926209DF91CF91E2
:10F670001F910F9108954A5260E080E03FDDC1CFB5
:10F6800080917A0681FF03C083B38078089581B1A9
:10F6900082700895BF92CF92DF92EF92FF920F9304
:10F6A0001F93CF93DF937B018A01080F191FEC0191
:10F6B000E81AF90A6701CC0EDD1EC017D107C1F0A8
:10F6C000B99080910B098270E19B05C08823E1F31A
:10F6D0000E946621F6CFDFBACEBAE09A8DB3B81693
:10F6E00049F3BDBA8FB7F894E29AE19A8FBFE2CF9F
:10F6F000DF91CF911F910F91FF90EF90DF90CF900E
:10F70000BF9008958091A90D1092A90D0895FC0154
:10F7100080818F70880F611181608F709081907FE0
:10F72000982B908381818F5F81838281882351F020
:10F730009F7041F4833621F0842F80628093A90D5D
:10F74000118212828281883069F148F4813091F10E
:10F7500088F0823039F1843009F03FC023C08F3502
:10F76000C1F018F48031F1F00895813649F0823605
:10F7700071F1089580818F708F3079F581E62BC00B
:10F7800040664093A90D10923601109235018FE525
:10F7900022C08181803211F4406816C08832E9F4B9
:10F7A00080E119C09181903328F090E0959587957C
:10F7B00082831182828190E00197218130E082234F
:10F7C0009323892B51F440644093A90D08958181BE
:10F7D000803418F088E0828311820895482F909138
:10F7E000630081B1242F30E02F3031056CF4F90132
:10F7F000EE0FFF1FE20FF31FE458F24F90819F704E
:10F8000081E09F3049F52BC050E0FA013F97E93085
:10F81000F10510F5E251FF4F0C942C9084701AC042
:10F820002FDF18C0892F13C0892F8095887012C0D0
:10F8300093FF12C081B101C0809580740BC08071AC
:10F8400009C090917A0691FF02C083B3F6CF817010
:10F8500001C08072811102C080E0089581E00895A6
:10F86000CF938D3208F062C09FEF980F993018F453
:10F87000825FCF91B3CF51EE580F5330D8F491B18E
:10F88000909594705523C9F040918D064F7041506A
:10F8900021E030E0042E01C0220F0A94EAF73091F3
:10F8A0007B0D3223523041F0932B21E009F020E010
:10F8B000922F03C090E001C0932FCBEDC80FC3304F
:10F8C000E0F4DEDE91E0811190E0CC2361F18091E3
:10F8D0008D0682958F70815021E030E001C0220FAB
:10F8E0008A95EAF780917B0D8223C23009F1982B2B
:10F8F00021E009F020E0922F16C0C63019F42091C3
:10F900008F0605C0C73079F420918F0622952F709D
:10F91000215081E090E0022E01C0880F0A94EAF79E
:10F9200090917B0D982381E0911104C080E002C08A
:10F93000982FF9CFCF910895CF93C82F91DF8111E0
:10F9400007C081E08C0F8CDF882321F081E003C0A9
:10F9500080E001C082E0CF9108958F7090E08F30F9
:10F96000910551F0FC01EE0FFF1FE80FF91FE4585D
:10F97000F24F82E68283118208958F7090E08F307B
:10F98000910549F0FC01EE0FFF1FE80FF91FE45845
:10F99000F24F83E682830895EF92FF920F931F93B5
:10F9A000CF93DF938091790D90917A0D019690938A
:10F9B0007A0D8093790D8093780D96B39095809110
:10F9C000AA0D882321F0282F2877292349F4892F8D
:10F9D000807609F07DC093FD77C094FF77C080E109
:10F9E000182F166019238093AA0DCCE7DDE000E004
:10F9F00011FB662760F9402FCE0189DE0F5F169557
:10FA000023960630A9F78091170281110EC0F0B23B
:10FA1000F09480917A0686FF09C08F2D837FF82E9F
:10FA20008091800E8C70F82A01C0F12CCFE8D2E2D0
:10FA300000E010E076E0E72EEC1AFE0184914C2FF6
:10FA40004E0D8F2161E009F460E0C8018257924FAA
:10FA50005EDE21960D5F1F4F0831110571F7909101
:10FA60001D0261E0C92FC07295FF60E04EE086EA9A
:10FA70009DE04DDE86B390E0809590958E77992736
:10FA80008C2B19F089E0809355018091800E86FDC2
:10FA900002C0817402C0817082609091630092FF05
:10FAA00088609091630095FF8062989B84609C9B26
:10FAB0008064B79B806180937B0DDF91CF911F9114
:10FAC0000F91FF90EF90089588E08ACF80E088CF73
:10FAD00080E686CF929A1092980089E180939900EF
:10FAE00080919B008D7F80939B0086E080939D009A
:10FAF00080919B0087FF03C080919C00F9CF88E92B
:10FB000080939A00089581E08093AE0D8093170250
:10FB100080917A0686FFDECF089580917A0686FF6F
:10FB200010929A001092170271C790919B0095FF56
:10FB3000FCCF80939C000895E6E6FDE091898089E2
:10FB4000891749F0DF01A90FB11D8C919F5F9F704C
:10FB5000918B90E008958FEF9FEF08951F920F9281
:10FB60000FB60F9211240BB60F922F938F939F9382
:10FB7000EF93FF9380919A008F7780939A00789407
:10FB8000E091760D81E08E0F8F7090919C00209116
:10FB9000770D821731F0F0E0EA59F24F90838093AD
:10FBA000760DF89480919A00806880939A00FF9176
:10FBB000EF919F918F912F910F900BBE0F900FBEE1
:10FBC0000F901F90189595E0899FD0011124A25C99
:10FBD000BB4FCB010596FB0124912D933196E8177D
:10FBE000F907D1F708950F931F93CF93DF93182F41
:10FBF000C2E7D2E090E08881181738F0882329F016
:10FC0000903201F19F5F2A96F6CF9032D9F02FE122
:10FC100030E0291B31090AE0029FA001039F500D2B
:10FC20001124BE01CE010A960E943F90FE0111925E
:10FC30000A95E9F7188384E68A838F8188608F8329
:10FC4000CE0102C082E792E0DF91CF911F910F9128
:10FC5000089580E491E0E2E7F2E0DF019C011D926B
:10FC600021503040E1F7089588E2EEE3F4E0DF014F
:10FC70001D928A95E9F788E4E6E6F4E0DF011D923B
:10FC80008A95E9F7089590E00197FC01EE0FFF1FB8
:10FC9000E80FF91FE255FB4F6F70628340832183A9
:10FCA0000895CF93C62F9FDFFC01C183CF910895A4
:10FCB0009F92AF92BF92CF92DF92EF92FF920F93FB
:10FCC0001F93CF93DF9300D000D0CDB7DEB7182FAE
:10FCD000E0916306F0E0E35EFB4FE49184E09E2F49
:10FCE0009370A1E0B0E0AC0FBD1FA90FB11D8C93C4
:10FCF000E695E695815099F7111108C0AADF61E0F9
:10FD00008981CFDF62E08A81CCDF3AC0113041F4D3
:10FD1000EB81F0E0EE0FFF1FED52FB4F10830AC0A6
:10FD2000123089F4EB81F0E0EE0FFF1FED52FB4F34
:10FD300081EC80838091C90585FF02C080E001C00D
:10FD40008CE9818309C1133009F583DF0981802F94
:10FD50004ADFFC01EE24E394E1821EEC1283802F43
:10FD600042DF02E0FC0101831283FA808F2D3BDF2A
:10FD7000FC01E18212838F2D36DFFC0101831283A7
:10FD800063E08B818EDF64E08C8121C0143009F543
:10FD900060DFFA808F2D27DFFC0122E0E22EE18276
:10FDA0000EEC02838F2D1FDFFC0111830283FC8088
:10FDB0008F2D19DFFC01E18202838F2D14DFFC01FE
:10FDC0001183028361E089816CDF63E08B8169DFED
:10FDD000C3C0153009F092C03CDF46DF81E003DF8D
:10FDE0004AE0C42EFC01C18282E0FDDE5BE0D52E3C
:10FDF000FC01D18283E0F7DE6CE0F62EFC01F1829B
:10FE000061E084E04EDF85E0EEDEFC0103E001838B
:10FE100074E0B72EB38287E0848387818160878313
:10FE200085E0E1DEFC0101831383A8E09A2E948231
:10FE300087818160878385E0D6DEFC010183B6E09F
:10FE4000EB2EE38289E0A82EA482878181608783DC
:10FE500085E0C9DEFC0191828CE9828381E08383A5
:10FE60008781897F8460878386E0BDDEFC01A18273
:10FE70008EE1828388EF83838BE0B5DEFC01018312
:10FE800096E4A92EA282B382C4828781816087838F
:10FE90008BE0A9DEFC010183A2821383D4828781D7
:10FEA000816087838BE09FDEFC010183A282E38275
:10FEB000F48287818160878380916E028F71806276
:10FEC00080936E028FE180936F026BEA72E280E0B2
:10FED0007ADE66EA72E281E076DE61EA72E282E070
:10FEE00072DE6CE972E283E06EDE67E972E284E062
:10FEF0006ADE67E972E285E066DE2EC0163099F4AC
:10FF000086E071DEFC01118382E3828398EF9383A4
:10FF1000808786E068DEFC0111838EEC828398E0A6
:10FF20009383808719C0173021F01830A9F488E036
:10FF300001C080E158DEFC0189E0818384E6828390
:10FF400084E1838387E786838EE08093CE0488E014
:10FF50008093CC048093CD0482E00E943B700F908C
:10FF60000F900F900F90DF91CF911F910F91FF9005
:10FF7000EF90DF90CF90BF90AF909F900C9437712F
:10FF800080E49CE99BBD8ABD87B7806187BF1FBCA9
:10FF90008AE08EBD08950F931F93CF93DF93109146
:10FFA0006902129516951770882331F0A3E0BEE020
:10FFB000833021F420E103C0ABEBBDE028E0909159
:10FFC0006802990F910F920F60916B0224E6620212
:10FFD000B0011124685A7D4F0091710248EE53E040
:10FFE00004039001059F300D112428533045261B32
:10FFF000370BFD0132966D937C9340916E0241FF69
:020000021000EC
:1000000003C040E055E002C040E054E0833011F40A
:1000100018EF190FCC27DD27C41BD50B1917F0F4E7
:10002000A12FB0E0AA0FBB1FAB50B84F0D90BC91F1
:10003000A02D4A175B070CF4DA01AC17BD070CF4CE
:10004000DE01A854B44F2A1B3B0BA61BB70BB18390
:10005000A083738362831F5F3496E0CF283293E2DC
:10006000390710F428E233E231832083882331F00A
:10007000285E33403093AC0D2093AB0D1382128277
:10008000DF91CF911F910F9108951F920F920FB69C
:100090000F9211240BB60F922F933F934F938F9390
:1000A0009F93EF93FF9388B391E0892788BBE091FA
:1000B0000E01F0910F018081982F9F709F3039F0D1
:1000C00040914D0E949F402D1124415001C04FEF9F
:1000D000242F30E037BD26BD90E024E0959587952C
:1000E0002A95E1F7009731F43196F0930F01E093F0
:1000F0000E0101C08083493C40F0809167028F70FF
:10010000863011F4C09801C0C09A8091B10D816011
:100110008093B10DFF91EF919F918F914F913F91FE
:100120002F910F900BBE0F900FBE0F901F90189540
:100130001F920F920FB60F9211240BB60F922F93AE
:100140003F938F939F93EF93FF9388B391E0892719
:1001500088BBE0911001F0911101808128B539B57B
:1001600080FD03C0205E3F4F02C0205F3F4F39BD7E
:1001700028BD90E095958795009769F4CF01019689
:1001800090931101809310018181811105C087B77F
:10019000877F87BF01C080838091B10D816080938C
:1001A000B10DFF91EF919F918F913F912F910F9002
:1001B0000BBE0F900FBE0F901F901895EDE7F0E06B
:1001C0008081857E808317981F9AAAE8B0E01C92F0
:1001D00010928B0082E88C938081806280830895E6
:1001E000EDE7F0E080818F7D8083179AAAE8B0E088
:1001F0001C9210928B008AE08C93808188618083AE
:1002000008951F920F920FB60F9211240BB60F9202
:100210008F939F93EF93FF9380914B0E882321F050
:100220001F9A10924B0E04C01F9881E080934B0ED2
:10023000E0910A01F0910B018081918190938700F8
:10024000809386008091AB0D9091AC0D90938500CA
:100250008093840082819381892B11F0329608C0AB
:1002600080916E028095817080934B0EE3E0FEE0FA
:10027000F0930B01E0930A018091B10D81608093AE
:10028000B10DFF91EF919F918F910F900BBE0F9049
:100290000FBE0F901F901895E2EBFDE090819695B0
:1002A00096952781222311F096959695982B908309
:1002B00021812F5F21838085281750F0A281B3818F
:1002C0009D012F5F3F4F338322839C9310821182C5
:1002D0000895FF920F931F93CF93DF93C82F8091C0
:1002E00067028F70823069F09C2F88E0D0E0292F60
:1002F0002078D20F990F8150D1F7D07859E0F52EA0
:1003000003C048E0F42ED0E810E080E190E00C2F2C
:100310000170901302C0805F02C0BEDF80E1C6950D
:10032000CD2B1F5FF11618F0D0E8902FF0CF805F33
:10033000DF91CF911F910F91FF90AECF882339F0BD
:100340008091B80D8F5F8093B80D80E803C0109244
:10035000B80D80ECA1DF8091B80D8530C0F708950D
:10036000CF93DF93C82FE091B70DE827F0E0EE0FB1
:10037000FF1FE85DFC4D259134915091B60D40E092
:10038000242735273093B70D2093B60DD8E08C2F56
:100390008078D4DFCC0FD150D1F7DF91CF91089581
:1003A000CF9380EC79DFC6E080E876DFC150E1F7DB
:1003B00080ECCF9171CF8031E0F4E82FF0E0EE0FC8
:1003C000FF1FEB50F84F20813181C901880F991F21
:1003D000820F931F97FD0396959587959595879521
:1003E0009C5F1816190644F48E3F27E092073CF4F0
:1003F000089580E094E0089581E090E008958EEF04
:1004000097E008956F927F928F929F92AF92BF92E2
:10041000CF92DF92EF92FF920F931F93CF93DF93D0
:100420001F92CDB7DEB772EB672E7DE0772EF3011A
:100430003F018BEB9DE093838283108211821582B2
:10044000148281E0878382E08087F0906702FF2D2D
:10045000FF70FF2EF8132BC080E180934D0E80912A
:10046000AD0D86FF0DC080914905811102C080E865
:1004700005C0813011F480E901C088E98093AD0D99
:100480008091AD0D87FF05C087E1A8D9882309F4C5
:10049000BBC08091AD0D87FDBDC08BE10E94A71C44
:1004A000882309F4B7C08091AD0D8062B6C084E1A5
:1004B00080934D0E86E0F81302C08FE01EC085E5E4
:1004C00008DF809149058F5F8F758093AD0D909106
:1004D000AF0D90FF03C080688093AD0D95FF05C000
:1004E0008091AD0D80628093AD0D8091AD0DF1DEF8
:1004F00080916802EEDE80914A05EBDE05EF17E0A1
:10050000C12CD12CE12C912C35E0A32EB12C48EF3D
:10051000842EF801819191918F01880F991F880F86
:10052000991F181619061CF424E030E002C02CEFC5
:100530003FEF820F931FB5010E94DB8FF5E0CB01E7
:10054000FF1202C09C5F02C080529C4F97FD07C003
:10055000811528E092072CF08FEF97E002C080E031
:1005600090E0AA2797FDA095092C03C0880F991F3A
:10057000AA1F0A94DAF7C82AD92AEA2A8BE0890D39
:1005800089838C2DA6DECD2CDE2CEE24E981E8506B
:10059000E983E830B0F793E0990D892F8695869529
:1005A0008695992E889D900C1124F8E005311F073F
:1005B00009F0AFCF26E0F21204C080E08ADE80E0CE
:1005C00088DEF3018181A281B381882319F08FE055
:1005D0008C9304C0FD018291806F80838BEB9DE042
:1005E00090930F0180930E010F90DF91CF911F9197
:1005F0000F91FF90EF90DF90CF90BF90AF909F90C2
:100600008F907F906F9008958091AD0D8F7780933C
:10061000AD0D3FCF8091AD0D8F7D8093AD0D80915D
:10062000AD0D57DE8091680254DE05EF17E0F12C26
:100630006DE0D62EF801819191918F01D89E9001A5
:10064000D99E300D112455E0359527955A95E1F73F
:100650003E5F37FD07C02F3FF3E03F0734F4E22E43
:10066000832F06C0E12C80E003C0EE24EA9483E0EF
:100670009F2D990F990F892B2CDE8E2D2ADEF39456
:1006800026E0F212D7CF9DCFCF92DF92EF92FF926A
:100690000F931F93CF93DF93C0916702CF70809128
:1006A000660685FF04C0809154028111C4E08091E8
:1006B000AE0D8111CFEF8091B00D8C1709F468C099
:1006C000C093B00D1EBC1DBC1CBC87B7837C87BF0C
:1006D00080917D008E7F80937D008CE386BF8FE3C9
:1006E00080937C008C2F90E08730910508F050C0FB
:1006F000FC01E950FF4F0C942C9060DD41DC08C1F7
:100700005DDD88E59BE199BD88BD80EA9FE090931F
:1007100079008093780087B7886087BF80917D00DB
:10072000816080937D001FBC82E08EBD44C046DDA9
:1007300088EC90E090937900809378008CE291E0CF
:100740009DBD8CBD80EE9BEA97BD86BD87B780625C
:1007500087BF80917D00816080937D001FBC8AE10E
:100760008EBD16C0C43021F484E015DCC09803C0EF
:1007700007DC83E010DC80E593EC909387008093A6
:10078000860088E893E1909385008093840028DDBB
:10079000C23009F4BAC038F4CC2309F4B9C0C1306E
:1007A00009F0B8C008C0C33009F4B2C0C550C230A7
:1007B00008F0B0C0AAC07894F0904D0E87B7877F3C
:1007C00087BF80917D008E7F80937D00E2EBFDE00E
:1007D0008BEB9DE090931101809310018CEB9DE0D9
:1007E000938382831582148210821182168217826B
:1007F00084E080878FEF8093BB0DD2DD809168020B
:10080000AFDD4091AF0D8091490540FF0CC090E4F1
:1008100089029001112480916702869586958695BC
:100820008670822B04C020E48202C0011124842B34
:1008300097DD80E095DDE0906902E294E694A7E020
:10084000EA228F2D8170D82EF0FE02C098E0E90ECA
:10085000F8E0CF2ECE0C8E2DAEDD8C01D110185FBE
:10086000802F7EDD81E08E0DA6DDEC01D110D85FFA
:10087000E394E3949C2F9295907F812F8F70892B26
:100880006FDDCE01E4E096958795EA95E1F768DDA6
:10089000EC10E1CF80E064DDC091B60D8091B70D22
:1008A0005FDD8C2F5DDD7CDD8091B30D882319F039
:1008B00080E0F2DCF9CFE091B40DF091B50D10823B
:1008C000E8E7F0E0808191819C012854344F39BDE4
:1008D00028BD805B994B91838083C09A88E086BF56
:1008E00081E080937C0087B7886087BF80917D001E
:1008F000816080937D0080914905813011F0F394EF
:1009000001C0F12CF0924D0E05C078947BDD02C041
:1009100080E041DBDF91CF911F910F91FF90EF902D
:10092000DF90CF9008951F920F920FB60F9211246F
:100930000BB60F922F933F934F935F936F937F93D9
:100940008F939F93AF93BF93CF93DF93EF93FF93D7
:100950008CB59DB520914C0E222321F0C09A1092A7
:100960004C0E04C0C09821E020934C0EC0910C01A5
:10097000D0910D01FE01219131913BBD2ABDF09333
:100980000D01E0930C01E6E0F1E0282F31813817EA
:1009900008F481833081231708F480838A819B8146
:1009A000892BD1F48BEB9DE090930D0180930C018A
:1009B00080916E028095817080934C0E87B78F7EF8
:1009C00087BF62DE809167028F7011F0833021F45F
:1009D00087B7806187BF78948091B10D81608093E3
:1009E000B10DFF91EF91DF91CF91BF91AF919F91A9
:1009F0008F917F916F915F914F913F912F910F90C8
:100A00000BBE0F900FBE0F901F90189580916E0235
:100A10008095817080934C0E80934B0E811101C0A4
:100A2000C09A809167028F70865F8093B00D10929C
:100A3000AE0D2ACE1F920F920FB60F9211240BB655
:100A40000F922F933F934F935F936F937F938F9367
:100A50009F93AF93BF93EF93FF93809167028F7043
:100A6000813011F1863029F0853031F080E492EA4E
:100A700005C080E89EE302C080E99DE397BD86BD86
:100A800020917800309179002F3F310538F4885853
:100A90009341909379008093780007C088EC90E0B0
:100AA0009093790080937800EFDDFF91EF91BF91F3
:100AB000AF919F918F917F916F915F914F913F91F6
:100AC0002F910F900BBE0F900FBE0F901F90189597
:100AD0001F920F920FB60F9211240BB60F922F9305
:100AE0003F934F935F936F937F938F939F93AF93B6
:100AF000BF93EF93FF93809167028F7078949091EA
:100B0000B00D981769F0943059F4809154028823FD
:100B100021F08091660685FD02C0B6DD02C084E04A
:100B20003ADAFF91EF91BF91AF919F918F917F91B1
:100B30006F915F914F913F912F910F900BBE0F904E
:100B40000FBE0F901F9018958091900680FD05C0F4
:100B5000809165008B7F809365000895CF93DF932C
:100B6000EC01F2DF1C821D82188219821EA61FA6CC
:100B7000DF91CF910895F2CF21E0FC0184818111B2
:100B800001C020E0822F0895FC0121818081281B73
:100B9000277098E0921B81E0933008F480E008957C
:100BA000CF93DF93EC018C818823F1F081508C830B
:100BB0008A819B81890F8A838EA58823D1F18FA595
:100BC0009FEF980F9FA7882351F08091900680FD9A
:100BD00030C0809165008460809365002AC0B4DFD6
:100BE000809168068FA725C01B98AEDF8D81882372
:100BF00019F081508D831DC0888199818917C9F0B2
:100C000090E0FE01E80FF91F26812A8326892C83B4
:100C100026852B83268D2D8320A92EA71FA626A1EE
:100C20003FEF320F36A3211104C001968770992738
:100C30008883DF91CF910895EF92FF920F931F93D6
:100C4000CF93DF93EC01F62E142FE22E9DDF882345
:100C500009F451C08091D30181FD4DC0302F3295F0
:100C6000369536953370402F4F70333009F43FEF8F
:100C7000FF2021F080916706865FF80E80915D0667
:100C80008873803129F48BEA189F112D112402C03A
:100C9000883111F4169509C0883211F4110F05C07E
:100CA000803319F4812F880F180F288104FF0DC09D
:100CB000FA821C83ED8205FB882780F98EA71FA688
:100CC0003B8329834423B9F001C04F5FE981F0E001
:100CD000CF01019687709927281769F0EC0FFD1F47
:100CE000F682168BE68E05FB002700F900AB41501B
:100CF00046A336878983DF91CF911F910F91FF9093
:100D0000EF9008950F931F93CF93DF93EC01062F7D
:100D1000642F80915D0686958695869587703881CB
:100D200029813213F0C010E00332110508F0EBC046
:100D3000F801E250FF4F0C942C9000E326C000E332
:100D400021E0C0C002EA22E04AE064E6DAC00AE23A
:100D500022E045E06FE5CE016FDF01E22AE045E0E9
:100D60006FE5CE0169DF0AE222E045E06FE5C9C028
:100D700002EC23E04AE060E5CE015EDF02E423E01E
:100D80004AE06CE3CE0158DF00E221E065C001E2F9
:100D900021E045E066E4CE014FDF22E04FE062E370
:100DA000CE014ADF22E04FE062C002E221E045E0EE
:100DB0006EE6CE0141DF03E221E045E097C000E0AE
:100DC00025E045E062E3CE0137DF25E045E06AE556
:100DD000CE0132DF02E024E043E06EE692C003E29F
:100DE0002AE045E060E5CE0127DF01E224E145E0AD
:100DF00060E5CE0121DF03E22AE045E038C002E6EB
:100E000025E044E16AE07DC002E22AE044E062E3DA
:100E1000CE0112DF01E224E148E066E4CE010CDFFE
:100E200002E22AE048E062E3CE0106DF01E224E1CB
:100E300044E04DC00AE22AE002C002E222E345E0BB
:100E40004BC001E203C002E201C003E22AE044E138
:100E500060E057C002E122E04AE039C002E423E04A
:100E600044E16CE3CE01E8DE02EE23E044E160E51C
:100E700048C000E321E048E22AC0813009F443C0C1
:100E800000E121E04AE06BE43CC08130E1F100E1A7
:100E900021E04AE061E435C000E121E046E031C0F4
:100EA00000E3D9CF813079F100E1D5CF00E112C064
:100EB00003E303C002E301C001E323E04FE00CC001
:100EC00001E329E144E103C000E321E04EE166E4EF
:100ED00018C001E321E04AE068E713C002E321E023
:100EE0004AE06AE70EC003E321E04AE06CE709C08C
:100EF00000E520E04AE062E804C000ED20E04AE0BE
:100F000062E3CE0199DEDF91CF911F910F91089599
:100F100046E4682F85ED91E0F5CE462F682F85EDEC
:100F200091E0F0CE9091690691FF03C0862F0C945A
:100F3000C116EECFCF92DF92EF92FF920F931F93E5
:100F4000CF93DF93EC01062F142F47FF03C0842FAC
:100F50000E94C116D7FF06C0D195C195D1098AE17B
:100F60000E94C116002371F0023019F464E670E0AB
:100F700002C06AE070E0CE010E94DB8F262FC22FF4
:100F8000D72FF82E64E670E0CE010E94DB8F9B0124
:100F9000FB01EC016115710599F16A307105CCF026
:100FA0006AE070E0C9010E94DB8F6B017C01653152
:100FB00071051CF48EE68C0D05C08CE88C0D0E942A
:100FC000BD168EE60E94C116F701309769F001E068
:100FD00001C000E084E68E0F0E94C116011104C01A
:100FE000209741F18C2F0AC0209721F1CE016AE0B1
:100FF00070E0E1D79E01281B390BC901845713C04B
:1010000084570E94BD160023A9F0023079F46AE0EB
:1010100070E08F2D90E0CFD7C82F86E0860F0E941A
:10102000C1168CE88C0F0E94BD1604C086E08F0D9F
:101030000E94C11611161CF4812F0E94C116DF9167
:10104000CF911F910F91FF90EF90DF90CF90089577
:10105000863050F4E82FF0E0E657F14FCB019F7057
:101060006AE070E094D760830895CF93C82F8430EE
:1010700091F48AE09B01829FB001839F700D11243F
:1010800080914C0F882309F441C070934B0F6093FB
:101090004A0FCBE23BC0873031F580914C0F6A306C
:1010A000710510F4816001C0836080934C0F8091C2
:1010B0004C0F81FF04C0CB016AE070E068D720913B
:1010C0004A0F30914B0F121613062CF04427552768
:1010D000461B570B01C0AB01240F351F3093B50ED3
:1010E0002093B40E13C08F3F31F47093B50E60930C
:1010F000B40EC4E00BC08E3F31F47093B70E609312
:10110000B60EC5E003C08C3208F0ACC0809164021A
:10111000EC2FF0E084FD07C0EE0FFF1FE455F14F08
:10112000718360831AC0C43071F1EE0FFF1FE45564
:10113000F14F71836083C53081F42091B60E3091F8
:10114000B70E4AE0429FC001439F900D1124909337
:10115000B50E8093B40EC4E016C0C03291F48091F5
:10116000FD0482958F7090E08617970718F4681B2E
:10117000790B02C060E070E07093ED0E6093EC0EAE
:1011800071C0C730F8F4E0E9FEE04C2F50E0440FA6
:10119000551FDA01A455B14F2D913C91E40FF51F75
:1011A000468557854217530714F4378726874081B1
:1011B00051814115510519F024173507C4F53183C4
:1011C000208335C0C031D1F4862F82958F7091E095
:1011D000980F2091890E291728F4963008F096E090
:1011E0009093890E9B012F703327322F2227672F70
:1011F0007727260F371FB901CF912ACFCC30B9F40A
:10120000A091C40EB091C50E2CE330E082D620919F
:101210000005211103C021E02093000530E040E0EB
:1012200050E0DCD63093C50E2093C40E1BC0C232F2
:10123000C9F48091EE0E9091EF0E4AE0489F900124
:10124000499F300D1124260F371F45E1429FC001F1
:10125000439F900D11246BE070E099D67093F90EC6
:101260006093F80ECF9108958A3308F0815180334E
:1012700031F0893331F08E3228F080E003C087E20C
:1012800001C08BE2E82FF0E0E85DFA4D8491EDCEED
:10129000E4E0FFE09091640293FD32C090819111EF
:1012A00010C08E35D9F581E0808385818823B1F126
:1012B0001582648170E0762F66278381682B828196
:1012C000D3CF8E3511F481E014C08D3519F481E04F
:1012D000818308952181222319F0118220E682273B
:1012E000913019F4828382E004C0923021F4838328
:1012F00083E080830895848381E08583108208954C
:101300009091260F903510F483830895682F70E034
:10131000762F66278381682B84E0A7CE08951F92DD
:101320000F920FB60F9211240BB60F928F939F93CB
:10133000EF93FF93E8E2FFE08585882359F0815021
:101340008587868591E0980F9687E80FF11D80814B
:101350008CB901C05598FF91EF919F918F910F909B
:101360000BBE0F900FBE0F901F9018959EE79093A5
:10137000280F8093290FEAE2FFE083E8860F82308E
:10138000A0F082E06083E1E0E80FF0E0E85DF04F7C
:1013900040832183128213821482158216829EE773
:1013A0009783875F8093350F089560528DE7808320
:1013B000319683E0E7CF8AB1877D8AB90895549842
:1013C00057981098189A0895F6DFF9CFFC0181819B
:1013D000828310820895CF93DF93EC01842F2B81B9
:1013E0003C81260F311D3C832B839091860E9111F9
:1013F00003C054E060E102C052E064E09D819F5F61
:10140000961710F49D8313C01D8202C03595279551
:101410005A95E2F729839A81921710F4291B01C08B
:1014200020E02883622F70E020DE1C821B82DF9187
:10143000CF910895FF920F931F93CF93DF93EC0109
:101440008881873F21F148F4863FB9F589818093EF
:101450000C0F8B8180930A0F30C08D3FF9F08E3FC7
:1014600061F540E069818EE09FE0B5DF41E06A818F
:1014700084E19FE0B0DF42E06B818AE19FE0ABDF77
:101480006C81669543E080E29FE0A5DF16C089810C
:1014900080930D0F8B8180930B0F0FC019811770F4
:1014A0001D5F239603E03AE5F32E011730F489918E
:1014B000EFDEF092260F0F5FF8CF83E28093270FC5
:1014C000DF91CF911F910F91FF9008958F929F927E
:1014D000AF92BF92CF92DF92EF92FF92CF93E7E36A
:1014E000FFE04181A8E3BFE080E090E02D91BC01E6
:1014F000620F711D872F9927860F971F99277FE00D
:10150000A034B70799F78F3F910509F043C189E6E9
:101510008093270F403109F03DC18381813F41F520
:10152000F48082818330F1F028F4813069F08230D8
:10153000A1F030C1843069F0853009F02BC143E05F
:101540006F2D80E29FE012C042E06F2D8AE19FE0A4
:101550000DC06F2D70E088E288DD40E06F2D8EE0D9
:101560009FE004C041E06F2D84E19FE034DF12C1B1
:10157000811108C08FEF8093260F6481758182816D
:1015800073DE08C19FEF9093260FC480D580E6805C
:10159000F780228122952F7030E1839FC0011124B2
:1015A000282B203609F492C008F049C0213209F4F2
:1015B00074C0B8F4203109F462C050F4213009F04D
:1015C000E9C09927F7FC9A958F2D7E2D6D2D5DC072
:1015D000213109F457C0203209F0DCC0B60180E2A5
:1015E000D8C0203409F466C008F5203309F0D2C011
:1015F0008C2D90E054E0959587955A95E1F780936E
:10160000890ECC2DCF7099278F2D7E2D6D2D8C2F8F
:101610001FDDC701B601E4E196958795779567953B
:10162000EA95D1F781E08C0F13DDB4C0213409F4C1
:1016300044C0203509F0AEC0B6018CE0AAC0223803
:1016400009F447C078F42137D9F130F4203709F094
:10165000A1C0B6018DE19DC02237A9F1203809F45F
:1016600042C098C0243809F481C008F489C02039E8
:10167000F1F0213909F08EC0B6018AE28AC0C701B3
:10168000B60103C0B60187E284C02AE030E040E042
:1016900050E0C6D4B9018FEF7CC0C701B6012AE083
:1016A00030E040E050E09AD4B90186E272C0B60161
:1016B00089E26FC0B6018AE06CC0B6018BE069C0F8
:1016C000B6018EE166C0B6018FE163C0B6018DE060
:1016D00060C0C701B60124E630E040E050E0A0D48D
:1016E000B9018EEF56C0460157014EE1B694A7945A
:1016F000979487944A95D1F7C701B6019F7320E16B
:1017000037E240E050E06AD46B017C01CA01B901C4
:101710002CE330E040E050E061D4A4E6A29FF00169
:10172000A39FF00D1124E60FF71FC82DC170BF0154
:1017300081FE0EC087E199DCB60188E196DCCC23FE
:1017400019F067E570E002C065E470E089E121C04E
:101750008AE18BDCB6018BE188DCCC2319F063E5F0
:1017600070E002C06EE470E08CE113C0C701B60106
:1017700024E630E040E050E031D4B90181E109C015
:10178000C701B60128EE33E040E050E027D4B901AC
:1017900086E06BDCCF91FF90EF90DF90CF90BF9011
:1017A000AF909F908F9008951F920F920FB60F9257
:1017B00011240BB60F922F933F934F935F936F9328
:1017C0007F938F939F93AF93BF93CF93EF93FF93A9
:1017D000579878949BB18CB1C0914F0F9C7109F0D0
:1017E0008BC090914E0F9230C1F030F4992309F4E0
:1017F0003FC0913049F081C0943009F44BC048F1AA
:10180000953009F44FC079C08E3709F476C08B311A
:10181000A1F092E090934E0F13C08D3711F483E046
:1018200036C08E3769F48091860E882319F0909324
:101830004E0F62C087E39FE0FDDD10924E0F5DC04A
:10184000C33108F05AC0EC2FF0E0E95CF04F808320
:101850000DC092E090934E0FC33108F04EC0EC2FB4
:10186000F0E0E95CF04F90E298279083CF5F45C0AD
:101870008E3751F48091860E882311F082E001C0EA
:1018800081E080934E0F38C08B31B9F584E08093AE
:101890004E0F33C095E090934E0F8093850E1092BB
:1018A000840E2BC09091840E91110CC0982F9F73C1
:1018B00091F494B3906C94BB95B3807C9F73892B07
:1018C00085BB09C0913019F480931B0204C092308B
:1018D00011F4809320028091840E8F5F8093840E98
:1018E0009091850E891309C010924E0F8091830E3E
:1018F00080688093830E01C0C0E08091860E8823AB
:1019000031F0C93020F0E2DD10924E0FC0E0C093FC
:101910004F0FF894579AFF91EF91CF91BF91AF91EC
:101920009F918F917F916F915F914F913F912F91F7
:101930000F900BBE0F900FBE0F901F901895109236
:10194000C90E1092C80E1092CB0E1092CA0E1092B1
:10195000F30E1092F20E1092880E1092870E1092D3
:10196000F50E1092F40E8CE1E0E9FEE0DF011D922D
:101970008A95E9F70895CF93C82F8093860E8091BA
:101980007A0681FF23C0DBDF1098189880917A06D1
:1019900085FD0BC0C11109C0809167028F70853031
:1019A00011F487E003C087E601C080E189B9109295
:1019B000900059981AB886E0809395005F9B02C00A
:1019C0008CB1FCCF1092350F88EB8AB9CF91089576
:1019D0001F93CF93DF931F92CDB7DEB780917A0626
:1019E00081FFF8C0909167029F7081E0913009F00B
:1019F00080E09091860E8913BEDF8091270F8823A7
:101A000051F081508093270F811107C01092B30EBF
:101A10001092B20E02C080E001C081E09091260FCA
:101A2000992329F0811182E091509093260F8093A1
:101A30004D0F2091830E222309F450C080917A0625
:101A400081FF4CC08091820E882321F081508093C9
:101A5000820E44C08091350F811140C091E0392F32
:101A6000322321F48F5F990F8830C9F79095922324
:101A70009093830E843028F420E040E060E08750AB
:101A800016C0863070F48170282F30E0D901A65F2F
:101A9000B04FF901E45FF04F2C9140E060818A5033
:101AA00006C0863039F420E040E060E081EF5EDC83
:101AB00085E00FC0873091F4E8E2FFE08BE180839E
:101AC000838381E081838091860E828384E0858791
:101AD0008AE08093820E1092360F559A10918105FC
:101AE000112309F477C01330F0F48091270F882375
:101AF00009F445C01150E12FF0E0DF01AA0FBB1F30
:101B0000A455B14F2D913C91EE0FFF1FEE0FFF1F1B
:101B1000EB50FB4F4081429FC001439F900D112429
:101B200064E670E029C0133049F48091260F8823C1
:101B300031F18091EC0E9091ED0E23C081E2810F86
:101B40000E94DF2A8823D9F0AE014F5F5F4F60E02B
:101B500070E08CEF810F0E945A2A2981211108C060
:101B60002AE0AC01249FC001259F900D112409C0DB
:101B7000223039F46AE070E00AD2CB0102C080E082
:101B800090E097FF02C080E090E02091870E3091B6
:101B9000880E280F391F21315EE03507BCF0205137
:101BA0003E40E4EFFEE08081918101969183808345
:101BB000DF019C978D919C91119701968D939C9339
:101BC000BA97808191810196918380833093880EAA
:101BD0002093870E0F90DF91CF911F9108958091F0
:101BE0007A0681FF07C01092890E8091830E8F6064
:101BF0008093830E089586B380958E7708958FEF36
:101C00008ABB1BBA91E897BB9EE798BB9EE394BB47
